:020000040800F2
:10000000F8FF012001FC09089DFC09082D5F050887
:100010009DFC09089DFC09089DFC090800000000E2
:100020000000000000000000000000009DFC090826
:100030009DFC0908000000009DFC0908AD110508A1
:100040009DFC09089DFC09089DFC09089DFC090808
:100050009DFC09089DFC0908911C0408991C0408D2
:10006000A11C0408A91C0408B11C040839070000DD
:100070004D070000610700007507000089070000B8
:100080009D070000B10700009DFC09089DFC0908C0
:100090009DFC09089DFC09089DFC0908B91C040881
:1000A0009DFC0908713304089DFC090861330408AC
:1000B0008133040891330408A1330408C1150408EE
:1000C000B5150408F5150408E91504089DFC090890
:1000D0009DFC0908A5100000F91100004D13000057
:1000E000C11C04089DFC0908000000006D340408D0
:1000F000453404087D34040835340408C50700007D
:100100009DFC09089DFC0908B13304089DFC090801
:10011000A1140000F5150000C1330408813B090853
:10012000D9070000ED0700000108000015080000D5
:10013000290800009DFC09089DFC09089DFC090890
:1001400000000000000000000000000000000000AF
:100150003D08000051080000650800004917000034
:10016000291604081D1604089DFC09089DFC0908B1
:100170009DFC09089DFC09089DFC09080000000081
:100180009DFC09089DFC09089D180000F11900005C
:100190009DFC09089DFC09089DFC09089DFC0908B7
:1001A0009DFC09089DFC09089DFC09089DFC0908A7
:1001B0009DFC09089DFC09089DFC09085D160408C2
:1001C000511604089DFC09089DFC09089DFC0908BE
:1001D0009DFC0908293F09089DFC09089DFC0908A8
:1001E0009DFC09089DFC09089DFC09089DFC090867
:1001F0009DFC09089DFC09089DFC09089DFC090857
:100200009DFC09089DFC09089DFC09089DFC090846
:100210008D3404089D340408AD3404089DFC09089D
:100220009DFC09089DFC09089DFC090800000000D0
:100230009DFC09089DFC0908000000009DFC0908C0
:100240009DFC09089DFC09089DFC09089DFC090806
:100250009DFC09089DFC09089DFC09089DFC0908F6
:100260009DFC09089DFC09089DFC09089DFC0908E6
:100270009DFC09089DFC0908451B000000000000CA
:100280009DFC0908000000009DFC0908000000001A
:08029000000000009DFC0908BC
:020000040804EE
:100000004368426D30B49A61EFF31182502383F359
:1000100012884168D2B2856C0B68046D23EA05032F
:1000200023430B6082F31188436981681A68096869
:1000300022F00102D0E908541A60826A1D605C61F6
:100040005A60D0E90B429C60DA600023B0F86C2063
:1000500030BCCA620377704730B5FAB18E464FEABA
:10006000014C034600F1C005002419680C3353F815
:10007000042C43F8084C41EA0C0142EA0E02AB4260
:1000800043F80C1C43F8042CEFD1D0F8C03043EAFD
:100090000E03C0E93144C0F8C03030BD4FEA014E14
:1000A0008C46DEE710B40C4C6368002B11DD002099
:1000B00004F1080C0146DCF8AC3003F1C0025960D1
:1000C0000C339342FBD1013063680CF5867C83428C
:1000D000F1DC5DF8044B704704000020F0B5474C9C
:1000E00004EB401292F8543403B9F0BD4FF4B47CE1
:1000F000434B00264FEA401E0CFB004C9CF83A553F
:100100008CF83A6582F83A541D785A7895420DD0A9
:1001100002EB420C560003EBCC0C9CF804C00CF133
:10012000FF37012F5DD9BCF1030F55D004EB0E0052
:10013000A0F83814EFF31183902282F3128890F81C
:100140003A24DBB2B0F8381442EA4102002192B2FC
:1001500080F83A1483F311881309247883EA122370
:1001600083EA0201DCB11301C943D0F85024012411
:10017000D0F83C049BB201F00F01D2F8AC208440CF
:100180000B4302F1C000590013F4004F8BB202D1AF
:100190005168214351600C328242F4D1F0BD130109
:1001A000D0F83C44D0F8502401F00F0104F11000C5
:1001B0009BB20124D2F8AC200B43844002F1C00072
:1001C000590013F4004F8BB202D1516821435160A2
:1001D0000C329042F4D1F0BD571C07F00307AF4238
:1001E000A4D0324403EBC2030344597C00299DD0C0
:1001F00004EB0E03012283F83A2497E70400002061
:10020000201B0024704700BF024B03EB401090F806
:100210005504704704000020704700BF0A4810F8DA
:100220004C1C81B101EB410100234438490010B45A
:100230001C4650F82320063302B114608B42F8D1DB
:100240005DF8044B70477047FC1000200A4810F816
:100250004C1C81B101EB410100234438490010B42A
:100260001C4650F82320063302B114609942F8D19D
:100270005DF8044B70477047FC1000200120704768
:10028000034B00EB400003EBC00010F8330C704749
:10029000FC1000202DE9F0431D4C14F84C3CABB38E
:1002A0000022A4F144034FF0500E1A4E4FF02C0CD4
:1002B000194F154607E053F8181B01320D6014F86A
:1002C0004C1C914222DD197C0029F4D05968FE2093
:1002D0004FEA9128A8F58018B8F1520F98BF17F887
:1002E0000800EFF311888EF31288D1F824900CFBEC
:1002F00000605FFA88F809F10109C0F88C9048693C
:1003000040F00100486188F31188D4E7BDE8F0832C
:10031000FC100020201B002448190A0807EE900A50
:10032000B8EE670A704700BFBCEEC00A10EE103A84
:1003300098B27047B4224FF4A57C4FF4EB710023C0
:1003400082805522A0F802C04FF4E17C02814FF474
:100350008772C1809621828144220370A0F80AC06E
:10036000C1814382028270470346012200205A77EE
:10037000704700BF08B5D0E90B2183690B44836146
:100380000AB108469047002008BD00BF436A0246F4
:100390001B681B6A5B685B7813F0010008BF50772D
:1003A000704700BFC2628161704700BF704700BFE5
:1003B000043070470C4B93F8FC22D3F8F812024437
:1003C0000844D2B2C3F8F80283F8FC2293F8FC2266
:1003D000120605D593F8FC2282F0800283F8FC22F5
:1003E000024B01221A707047201B002400000024D9
:1003F0002DE9F84F154FD7F80053ED0A20D000260D
:10040000DFF84CA007F54179B046AC19D7F80413D2
:10041000102352466410D1F828B04846C7F83083FC
:10042000E102D8470F280BDD094B03F1100253F806
:10043000041B013107D19342F9D12546B542E4DCD2
:10044000E802BDE8F88F661CF8E700BF201B002417
:1004500040F20024184BD3F83813D3F83C238A1AFF
:10046000322A15D8D3F850238A4200D37047D3F8E4
:100470004023E2B110683231928810B44469C3F865
:10048000501322425DF8044B18BF1204826170477A
:10049000D3F840233AB193F84C031168C00792880F
:1004A00048BF12048A610022C3F8502370473231DA
:1004B000C3F85013704700BF201B0024064AD2F82F
:1004C00040333BB192F84C131A68C9079B8848BF68
:1004D0001B04936100207047201B0024044B4FF441
:1004E000007C0020D3F86033A2F800C00B60704796
:1004F000201B002400207047012070470120704716
:100500000020704700B596461A6972450CD38C4698
:1005100071448A42996938BFA2EB0E0C71445DF8B0
:1005200004EB624661F01AB85DF804FB2DE9F8436C
:1005300010F08CFE224F4FF0000C05464FF48678E9
:10054000204E7968002930DD00231C4608FB037229
:10055000013392F805218B4244EA0204F6D144EAC1
:100560000C0C5FFA8CF97368C3F30803D3B9EFF38B
:100570001183BBB914F092FD431BB3F5FA6FCCBFE6
:100580004FF0000C04F0010CBCF1000FD9D1B9F10F
:10059000000F04D00C4B93F89023542A08D04846FF
:1005A000BDE8F88310F026FEE6E7E1460024DAE72E
:1005B000B3F8982348460132A3F89823BDE8F8839E
:1005C0000400002000ED00E0201B00242DE9F04F86
:1005D000BD4D87B02B781BB9012007B0BDE8F08F67
:1005E0006B68BA4A002BD2F8387318DD05F108049D
:1005F0000020B749D4F8F430BFF34F8F03F5907261
:10060000C1F85C3220339342FAD1BFF34F8FBFF36E
:100610006F8F01306B6804F586749842EADBAD4B4E
:10062000AD4EA3FB0723AD4FDFF8C8A25B09A7F1CE
:100630007C0BA6FB0326F60806EB8606A3EB460614
:10064000F3B207EB8606059307F538730293002390
:100650009946DBF864344B4540F30F81DAF81830E3
:10066000DAF80480D3E93D5410F0F0FD0122049043
:1006700002FA08F39A4901936118944B05EB410182
:1006800093F8A40393F890331A46039305EB4003C1
:10069000542A00F04181019A994240F24481B3F812
:1006A00000C01CEA020F00F04D81B3F802C01CEA42
:1006B000020F00F04A81B3F804C01CEA020F00F0F8
:1006C0004781B3F806C008331CEA020FE4D1019257
:1006D000A3EB050E99424FEA6E0E40F22481A4EB83
:1006E0000E04452C28BF452403EB4404A34280F0AC
:1006F0001F8100259C46019AA84629460196188824
:100700001040884214D158881040814240F0D78070
:1007100098881040814240F0D480D8880833104037
:10072000814206D19C4207D9188810408842EAD0FD
:1007300002339C4200F2A880B8F1110F019E40F2F2
:10074000F780D8F1150200F1F3806649049C4B68EC
:100750009E455E4BD3F8A80338BFC1F804E0231AC6
:10076000002B13DB604B03449C4200F2F680574899
:10077000C0F8A8334B68052B40F2ED80053BDBB297
:10078000524880F8A4334FF0FF334B6042B105FA72
:1007900002F2C8F11408012505FA08F848EA020532
:1007A000524BC5F3C43203EB8202506D05F01F02B9
:1007B00003EB8202516DC5F34412C5F3842503EBAC
:1007C000820203EB850541EA0031536D41EA0311D2
:1007D0006B6D41EA032181EA112383EA131303F0CD
:1007E0000F030F2B40F08880B1F5803F80F08480AC
:1007F000039B0909542B05D1344AB2F894330133D1
:10080000A2F89433DBF86433B1F5606F03F10103B0
:10081000CBF8643300F0B380029B998197F858308D
:10082000059883420CD0B2683B689B1A3B607B689A
:10083000326B9B1A7B600023B360336387F85800E8
:100840003B6801333B60B3680133B3604FF6FF731D
:10085000994205D17B6801337B60336B013333638D
:10086000029B09F101095C375C361433B9F1080FBA
:100870000AF1200A02937FF4ECAE012301208BF8E9
:10088000603407B0BDE8F08FA3EB0C0C184833F8C8
:10089000021C4FEA6C0C11400CF1010C80FB0C6047
:1008A000A0EBEC704FF0010C0128B8BF012085408F
:1008B000804401380CFA00F09C4605431FE70433DE
:1008C00037E7063335E700BF04000020201B002473
:1008D00000ED00E01F85EB51CDCCCCCC7811002091
:1008E000C7FFFF7F0000002420A1070048190A0865
:1008F000565555553C040020039B542B33D0DBF850
:1009000064330133CBF86433DBF860334FF6FF71A7
:100910000133CBF8603381E7204A9942A2F89A0369
:10092000019A3FF6BCAE18B101381C4B83F8A40302
:10093000039B542B94D1194AB2F896330133A2F891
:1009400096338DE702330192C2E604330192BFE68B
:1009500006330192BCE6002312E704980F4B0530E2
:10096000C3F8A80306E70D4AB2F894330133A2F89E
:100970009433DBF864330133CBF86433C4E7074ABC
:10098000537803EB430302EBC3034B445B7C0D2B17
:100990007FF442AF8023029A93773FE7201B002425
:1009A00010B5044660F05CF80146204689B2BDE807
:1009B0001040FFF793BB00BF00EB400010B5084CA0
:1009C00004EBC00414ED0F7A54ED0E7AE7EE007AD2
:1009D000B0EE670A60F044F854F8443C186010BD6B
:1009E000FC100020F8B5264B1A785B789A4242D169
:1009F000244E7368002B23DD002506F10800224CED
:100A00002F46D0F8AC30BFF34F8F03F1E002C4F8AB
:100A1000683220339342FAD1BFF34F8FBFF36F8F09
:100A2000337813B1037F012B20D0426901357168FF
:100A300000F586701368A94243F001031360E0DCFF
:100A400010F004FC114BD3F86844002C0DDD03F2C8
:100A50006C4303EBC4041968083333F8042CC868EA
:100A60009C4242EA0002CA60F5D1F8BD80F8FC70F1
:100A7000FFF7C6FAD9E759F077FC0028B8D1F8BDDE
:100A8000201B00240400002000ED00E0FC100020EA
:100A90004FF0B042F8B5D2F88030D2F888502B40F1
:100AA00003EA0005C2F888507DB1084F0126B5FA67
:100AB00085F4C4F11F0407EB840306FA04F4D3F8A9
:100AC000AC0303689847A543F1D1F8BD201B00246F
:100AD0000269C3682DE9F04712EA03092AD00546E6
:100AE0000E464FF000474FF00008B9FA89F327FA95
:100AF00003F21B3BD24309EA02092A61042B16D8F0
:100B0000DFE803F03B30251A0300B36A002B3FD027
:100B100003F1FF3AC6F828801FFA8AFA746A34B1E2
:100B200023682046514698476468002CF8D1B9F1F3
:100B3000000FDAD1BDE8F08770680028F7D0696B44
:100B4000036889B29847B9F1000FCED1F2E7B068D7
:100B50000028ECD0A96B036889B29847B9F1000F5F
:100B6000C3D1E7E7F0680028E1D0E96B036889B2F8
:100B70009847B9F1000FB8D1DCE730690028D6D02A
:100B8000296C036889B29847B9F1000FADD1D1E75C
:100B9000E96A1FFA81FAC1E78069B4304FF044BCBA
:100BA00038B590F828300446012B04D0407F40B17E
:100BB0000023637738BD406A03681A7B9AB9637F64
:100BC0000BB9012038BD0A4D022305F1200205F1C1
:100BD00040010FF00FF895F8213003F0010383F086
:100BE00001006377E6E71B6A002BE8D0002038BDE0
:100BF00040F20024F8B5144E044690F8281006F18F
:100C00002007437F012904D00BB100236377012023
:100C1000F8BD606A01680D7B85B9002BF7D002230F
:100C20003A460A490EF0E6FF96F8213003F0010338
:100C30006377002BEBD094F82810E3E70A6A002AC8
:100C4000E8D1002BE3D0EAE740F2002480F2002450
:100C5000F0B511F0010583B00AD190F82860044680
:100C6000012E07D0C368B3F1807F01D90123237718
:100C700003B0F0BD0A4B476AD3F88C040FF02EF98D
:100C8000E368B880B3F1807FF2D9B7212A463846AD
:100C900033468DF8041001A926770EF0ABFFE7E785
:100CA000201B002470B5002394B00546224C069307
:100CB00002200B9304F120021093139311930192DD
:100CC0001E4E6A6A04960E4600940290CDE90E33D9
:100CD00001238DF80C3007938DF820308DF83430D7
:100CE0008DF848302B7F002B14BF052304230C9371
:100CF00004F140030593124B0993A4F120030A93D6
:100D000010685DF06FFD2B7FA3B1A4F18002330E5C
:100D10001E3C82F86130320C6946330AA67022709C
:100D20006370686A0EF0ACFF6B6A18685DF05AFD7C
:100D300014B070BD1F3CEEE7C0F200248D03040820
:100D40006903040810B594B0044650220649684669
:100D500060F004FC6946606A0EF092FF636A1868EE
:100D60005DF040FD14B010BD1C1A0A082DE9F843CF
:100D70001F46436A04468846186891465DF032FD76
:100D8000237F002B3BD0A0690523264D264EAB6365
:100D9000030EE23606F8013CB070030C000A012F86
:100DA000337070704FF00000D8F800306B64D9F8E1
:100DB0000030EB642363E86527D0022F1DD1D9F8FA
:100DC000042068651344D8F8041085F850002A669A
:100DD0000122A9652363154B85F86420AB66144B8B
:100DE000617F03F11402606A002914BF194611469D
:100DF0000EF046FFE36A7BB1206BBDE8F883094D36
:100E00000423A0690B4EAB63C6E7084B85F850700E
:100E1000A86528666B65E2E7636A18685DF0E2FC26
:100E2000EAE700BF0000002440F200247503040834
:100E30000800002421F3002400B583B081610192F1
:100E400001A9049A00930123C2626A46FFF78EFF4C
:100E500003B05DF804FB00BF2DE9F0439846436AF8
:100E600095B0054618680E46344C91465DF0BAFCC4
:100E70000223334A0027029304F59073049204F589
:100E80008072009304F5A073297F019301230592DA
:100E90008DF80C300697002937D08DF8343004F5E2
:100EA00081748DF84830330ECDF82C9004F8013C55
:100EB00005238DF82070CDF8308013970793CDE986
:100EC0000977CDE90E77CDE91077330CA6701D4F69
:100ED000360A23706670D7F88C040EF0FFFF6C6A38
:100EE0006B7FA0803BBB05A920460EF0C9FE6B6A54
:100EF00018685DF077FCD7F890040EF0EFFF6B6A8E
:100F00009880404615B0BDE8F0838DF8343004F287
:100F100001148DF848300423CDF82C908DF8201062
:100F2000CDF8308013910793CDE90911CDE90E1169
:100F3000CDE91011C9E76946D6E700BF40F20024A9
:100F40008D030408201B00242DE9F843DDF82080E0
:100F50000F4616460021202204461D4660F072FB13
:100F6000B8F1000F0CD0D8F80030B8F80A20E381AF
:100F70001B0C2382D8F804306282E3821B0C23838B
:100F800038465DF03DFFF30619D4431EB8B107EBB8
:100F9000000C01E0013B12D31CF801EDBEF12E0F55
:100FA000F8D1C01A03F10109421EB944032AA8BFAF
:100FB0000322082BA8BF082390461A4606E00828FB
:100FC0000246B9464FF00008A8BF08224FF0203370
:100FD000394620462360636060F0C0FA04F10803DC
:100FE0001748424649462081A072184660F0B6FA7A
:100FF00004F1FF3C0346E21D1CF8011FA1F1610E44
:101000002039BEF1190F98BF8CF800106245F3D15A
:10101000184604F10B0110F8013BA3F16102203BDB
:10102000192A98BF00F8013C8842F4D1182365833F
:101030002D0CE6722373099BA582E361BDE8F8835A
:10104000202020002DE9F04FDFF88C9487B0D9F8EC
:101050003803C9F83C03002B00F0DA80134415462E
:1010600001F1200601F5FE77DFF870A403931FE07D
:10107000002D63D0D9F86C23AA4200F0CD80D9F8B6
:101080006823AA4200F00281D9E9DC21AA424CD8A7
:10109000A94200F2CF81691A184657F06DFE01355A
:1010A000039B06F5007607F500779D4200F0B080BF
:1010B000D9F87843A6F12003AC42D9D82C1BD9F833
:1010C0008883E208D8F8301004F0070402328A421C
:1010D00003D3D8F838108A420DD9414610460593FB
:1010E000049257F019FE8046DDE90423002800F041
:1010F000C181C9F8880398F80410002940F03F81A5
:10110000D8F828B0BBF1000F00F0AD811846D8F830
:1011100030304FF40071D21AD8F80C3004EBC20210
:1011200003EB42224346D847B9E7A942B3D9184650
:101130004FF40072002160F085FAB0E74FF40072BE
:101140002946184660F07EFA80220346D94886F880
:101150009E210C2286F8A221D9F86813D9F86023C1
:101160008142C3F8C611C3F8CA2100F36881D24B8B
:10117000013AD24C83FB0103C81784FB01C40B4422
:10118000C0EB6313C0EB2430CD4C84FB03C4C3EB32
:10119000831C86F8A1018010A1EB0C011C4420F0F7
:1011A0003F000131014386F8A011D917C1EBE411CA
:1011B0000B4486F89F31BF4B9A4200F34C81BE4BE3
:1011C000BE4883FB0213D11780FB02401344C1EBDE
:1011D0006313C1EB2031BA4880FB0340C3EB831497
:1011E00086F8A5118910121B184421F03F01013225
:1011F0000A4386F8A421DA17C2EBE010034486F80C
:10120000A331552386F8DE31AA2386F8DF3146E77D
:10121000002007B0BDE8F08F4FF0FF320024A6F1A8
:101220001C00049383F8EC21214683F8ED2183F818
:10123000EE2183F8EF2152221A705A7061229A70BF
:1012400083F8E7214122DA7083F8E621722283F8DD
:10125000E42183F8E521D9F88023C3F8E8214FF48D
:10126000F07260F0EFF9049B5522C6F8D041C6F841
:10127000D441C6F8D84183F8FE216FF0550283F8B7
:10128000FC4183F8FD4183F8FF2108E78D4C0021E4
:101290004FF40072184660F0D5F903464FF0000C89
:1012A000022203CC46F8191CEB2146F81D0C08203D
:1012B00006F8201C582106F81F1C902106F81E1C59
:1012C000F8211A7383F80BC006F8130C9A7383F88D
:1012D0000FC006F8102C06F80B1C83F82C20D9F848
:1012E0006813D9F8602383F819C0521A83F81BC019
:1012F00083F81DC01A6283F81EC083F81FC083F8EC
:101300002DC083F82EC083F82FC0D9E9DC12521A01
:1013100080215A623F221A764FF0FF329A763E229F
:101320001A77012283F8302083F831C086F8201024
:101330002921654B86F82210942186F8260086F82C
:1013400023100E21614A86F824100D2186F82510FD
:10135000552186F8DE11AA2186F8DF1103CBC6F8E5
:101360002B101988C6F827009B78A6F82F1086F84E
:10137000313003CAC6F83200C6F836108FE64FF493
:1013800000721846002160F05DF9D8F8402003464D
:10139000002C76D1002A00F0A380D8F8303011223A
:1013A0004B49CDE90044FFF7CFFDD8F840301A6C27
:1013B000002A00F0A1801B6BCDE9004411224549B1
:1013C00030464FF4E07BFFF7BFFD06F12003D8F86D
:1013D0004480B8F1000F3FF462AE03F120049B4457
:1013E000049523464446984610E05CF81C1B0025F3
:1013F000236BCDE900C5FFF7A7FDABEB0803A46C99
:1014000008F12008002C18BF1F2B51D92379A446BE
:1014100004F11C0E1122A8F12000002BE5D1627905
:101420002569236B42F021022168CDE900E5FFF731
:101430008BFDE2E7A91A184657F09EFC2FE6FF2322
:10144000013A86F89F3186F8A13186F8A031194B10
:101450009A427FF7B4AEFF2386F8A33186F8A53110
:1014600086F8A431CDE6594618464FF4007260F074
:10147000E9F814E6A6F1240343F804AF9F42FBD138
:101480000DE6002AD8F844800CBF01220222C2EBEC
:101490000414B8F1000F3FF402AE4246013C926CD6
:1014A000002C01DD002AF9D190464FF4007B90E733
:1014B000049DF4E5FF03FB00832008829755454116
:1014C0008180808038AB0A0844AB0A0850AB0A0818
:1014D00030AB0A0834AB0A08201B0024DEADBEEF97
:1014E00023460822D9F864134FF4F07BCDE9004479
:1014F000FFF72AFD33466AE72346CDE900445DE75E
:1015000010B4294C94F88C346BB3D4F894249042E2
:1015100035D0012B27D0D4F87025824237D0022B4A
:1015200021D0D4F84C26904233D0032B1BD0D4F8D2
:10153000282790422FD0042B15D0D4F804289042AD
:101540002BD0052B0FD0D4F8E028904227D0062BC3
:1015500009D0D4F8BC29904223D0072B03D0D4F86B
:10156000982A824211D0DC22591C02FB034284F8E3
:101570008C14C2F8940418465DF8044B704700239D
:10158000DBB25DF8044B184670470723F8E70123E8
:10159000F6E70223F4E70323F2E70423F0E7052349
:1015A000EEE70623ECE700BFFC10002000207047A8
:1015B000704700BF014850F005BA00BFCC1F00249F
:1015C000084810B4D0F8AC34D0F8E04499691A68EF
:1015D0002CB1234600F2AC405DF8044B18475DF88F
:1015E000044B7047201B0024014850F0EBB900BFAA
:1015F00030200024084810B4D0F81035D0F8444505
:1016000099691A682CB1234600F5A2605DF8044B75
:1016100018475DF8044B7047201B0024014850F028
:10162000D1B900BF94200024084810B4D0F8743514
:10163000D0F8A84599691A682CB1234600F2745075
:101640005DF8044B18475DF8044B7047201B0024DD
:10165000014850F0B7B900BFF8200024084810B482
:10166000D0F8D835D0F80C4699691A682CB12346C1
:1016700000F5BB605DF8044B18475DF8044B7047FC
:10168000201B002403282DE9F04FD4BF0027012799
:1016900083B0B0F1FF3F08BF47F001078DF8073076
:1016A000002F40F0C5809D4E6423054603FB006378
:1016B000D3F8AC04002800F0BC8093F8ED44202C53
:1016C00040F0CB8093F8EC44012C00F0C68001245C
:1016D0009346D6F8248683F8EC4406E0D6F8243600
:1016E000A3EB0803192B00F2A880836913F40043CD
:1016F000F4D14FF0640A4FF021094FF0010C4FF084
:10170000400E0AFB05FA864A06EB0A0484F8ED94BB
:1017100001FA0CF984F8EEE4C4F8E034C4F8F034CB
:10172000A4F8D6C44368134043EA41037D498A4480
:101730007D4919430DF10703C4F8D0344160414697
:10174000504658F0ADFE002840F0CB80D4F8AC14E1
:10175000C1F828B006E0D6F82436A3EB08030A2B1C
:1017600000F2B2808A6912F08002F4D0642202FB97
:101770000562B2F8D6349BB2FF2B78D8B2F8D634D3
:101780006A489BB2A2F8D434DBB24A6849EA034300
:101790000240134343F000734B60642404FB056470
:1017A00005E0B4F8D6349BB2002B00F0A18041468E
:1017B000504658F075FE00284FD1D4F8D034D4F8F4
:1017C000AC2413F8010BB4F8D4149062C4F8D034EC
:1017D0000139B4F8D63489B2013BA4F8D4149BB2D1
:1017E000A4F8D634B4F8D6349BB20029D9D1002B52
:1017F000D7D0916911F0800109D1D6F82436A3EB36
:1018000008030A2B4FD8916911F08001F5D0B4F884
:10181000D6349BB2FF2B36D9536844490B40444918
:1018200043EA09031943FF23A4F8D4345160B8E70D
:101830000027384603B0BDE8F08F64232021002242
:1018400003FB0565D5F8F03485F8EC240B43C5F8A7
:10185000F03485F8ED1485F8EE24B6F828363846CD
:1018600001339BB2A6F8283603B0BDE8F08F4B6871
:101870002E4803402E4843EA09031843FF23A2F8E9
:10188000D434486089E7B4F8D63428489BB251680C
:10189000A4F8D434DBB2014049EA03430B4343F0DC
:1018A000007353607DE7642303FB0565D5F8F034CE
:1018B00085F8EC1443F02003C5F8F034202385F8B4
:1018C000ED3485F8EE14C8E76423202003FB05639C
:1018D000D3F8F0140143C3F8F01483F8ED0483F84F
:1018E000EE246423002203FB056585F8EC24B4E7AD
:1018F0004146504658F0FEFD0028AED1D4F8AC3435
:1019000020210C4D0127D9615A682A405A6084F879
:10191000ED1484F8EC0484F8EE048AE7201B00241C
:10192000009800FCCC1F002400200181009C00FCDA
:101930000000FF0100E800FE114A037A0168D35C51
:1019400010B4CC58CA1824F00104CC501368DB073B
:10195000FCD4037D1F2B09D9203B20225DF8044BCA
:1019600002FA03F343F01803CB60704720225DF8BE
:10197000044B02FA03F343F018038B60704700BF77
:1019800054AC0A08F8B507680646D7E90454A061C4
:101990002B7D1F2B49D9203B2022286802FA03F314
:1019A00043F01803C360237D1F2B48D92022203B1E
:1019B00002FA03F3226843F01803D360636800223D
:1019C00069680A601A601A6842F010021A60BA69FF
:1019D000297A5AF0CDFBFA69217A20685AF0C8FBBF
:1019E00033682E681A6A5B6891685868184A024022
:1019F00020680A4317495A602A7A8D5C725942F06E
:101A000001027251227A895C425842F0010242502E
:101A10009A6842F440429A601A6842F001021A60E1
:101A20001A6842F400721A60F8BD2022286802FA8F
:101A300003F343F018038360237D1F2BB6D82022C5
:101A400002FA03F3226843F018039360B6E700BF7D
:101A50000000FFFF54AC0A0810B1036882889A6145
:101A6000704700BF18B1838802681B0493617047F8
:101A700008B51D200EF0CEFD08B183794BB11E20B4
:101A80000EF0C8FD08B1837903B108BD5523C380AA
:101A900008BD5523C380F2E7D3B20F2B2AD84FF0ED
:101AA000000C10B46346144C04E001332A2B1DD003
:101AB00014F803CF6045F8D194F801C08C45F4D1F7
:101AC0000E4C03EB43030E4902EB420C23445DF83A
:101AD000044B01EB8C0201F1800093F8263100EBFE
:101AE0008C00C2F8883082F88030704700205DF8A2
:101AF000044B7047002070476C1A0A0848190A08FE
:101B00000000002410B40C4C002304F22C6C01E003
:101B1000152B0CD003EB430201331CF80210814259
:101B2000F6D122445DF8044B92F92E0670474FF02F
:101B3000FF305DF8044B7047201B002430B40023B5
:101B4000114C124D04E001331A2B1AD054F8085FDF
:101B5000A842F8D125798D42F5D10D4C02EB420512
:101B60000C4904EBC30301EB850201F1800093F8FB
:101B7000A93100EB8500C2F8883082F8803030BC93
:101B80007047002030BC7047EC1A0A080000014082
:101B900048190A0800000024F0B1002310B50446DB
:101BA0000E4894F804E000F22C6C01E0152B11D0E3
:101BB00003EB430201331CF802107145F6D10244D5
:101BC0006179206892F92E26D3B20F2B02D8BDE896
:101BD0001040B3E7002010BD00207047201B0024F8
:101BE0000138074B074A00EBC00003EB8000D0F838
:101BF000400190420CBFA020A12058F0F3BE00BFCE
:101C0000000000240000024001382DE9E84100EB0B
:101C1000C000134D1E46134B05EB800590460F4642
:101C2000D5F8400198420CBFA020A12058F0DAFE60
:101C3000B5F956014FEA9811C5F85071C5F85861C9
:101C400058F0A0FEB5F95631002B07DB03F01F005A
:101C500001225B090449824041F82320BDE8E88164
:101C6000000000240000024000E100E0800AA0F52E
:101C70008010522806D8044B1B5C0D2B02D8034A57
:101C8000D05670470020704748190A0844AC0A082B
:101C90000120FEF7FDBE00BF0220FEF7F9BE00BF27
:101CA0000420FEF7F5BE00BF0820FEF7F1BE00BF1E
:101CB0001020FEF7EDBE00BF4FF47870FEF7E8BECF
:101CC0004FF47C40FEF7E4BE30B1036882881B69A4
:101CD0001A4214BF01200020704700BF70B50C46A7
:101CE00086B00546164640B101680E4B0E4A0B44BD
:101CF0009B0A02EB4303B3F8740258F073FE04F03E
:101D00001303AA8801A90293C4F341132868C4F3FA
:101D1000810401920596CDE903344FF00DFD06B024
:101D200070BD00BF0000FEA748190A0800B1D5E742
:101D300070472DE9F84FC34F6423044603FB00733B
:101D4000D3F89464002E00F06D81D3F89CA4BAF10E
:101D5000000F04D09AF80630002B40F06381642312
:101D600003FB0473D3F8A0541DB1AB79002B40F0F2
:101D70005981631CDBB2BAF1000F04D015228AF836
:101D800007308AF8062015B11622EB71AA714FF0C0
:101D90006409308B58F026FE294609FB04F95046A9
:101DA0005CF024FD504607EB090898F8A63498F833
:101DB000A424002B14BF3E211E21FFF7B7FF98F883
:101DC000A6342846A04D002B98F8A5244D44DFF8F2
:101DD000989214BF3E211E21FFF7A8FF4C2200213C
:101DE00028465FF02FFCD8F89434984A5B689342F9
:101DF000C8F8AC34DFF8748240F0168150F000F976
:101E0000D9F82030C3F302139FED917A9FED915AD8
:101E1000B0EE084A4344F7EE003A4FF0000E40F2AD
:101E2000145893F8883203F01F03D840642307EE58
:101E3000900A03FB0473F8EE677AB3F8A894C7EE30
:101E4000275A07EE909A9FED847AF8EEE77AC7EE6C
:101E5000274ADFED827AB0EE007AE5EE877AA5EECA
:101E6000875A25EE844A37EE856A74EEE72AB9F57B
:101E7000C87F0EF1010CD5BF642332234FF4967056
:101E8000782007EE90CAD8BF4FF4167A0344C8BF33
:101E90004FF4827AB8EEE77AD8BF414607EE903A1F
:101EA000C8BF4FF4FA7127EE257A01EB0A03F8EE6A
:101EB000E76A86EE873A73EE636AFCEEE67A17EE1F
:101EC000902A07EE90AAB8EEE73A07EE903AF8EEBD
:101ED000E77A23EE243AC3EE276A36EEC53A72EE6D
:101EE000E66AC3EE077A77EEE37AFCEEE77A17EE5E
:101EF000901AC6EE877A77EEE37AFCEEE77A17EE71
:101F0000903A03F1020A0AEB010BF0EE466A07EE83
:101F100090BAF8EE677AE7EE276AF4EEE64AF1EE59
:101F200010FA00F388805FFA82FABAF10F0F00F21C
:101F30008480323807EE900AF8EEE77A77EEC47ABA
:101F4000C7EE876AFCEEE67A17EE900A5FFA80FA2F
:101F5000BAF10F0F71D81FFA81FABAF1FF0F6CD8DE
:101F60001FFA83FABAF1FF0F67D812054AEA0E7317
:101F700002F07F620004134300F47F00384A0343F9
:101F800002EA01210B43642000FB04740027284669
:101F9000C4F8B0340123C4F8B474C4F8B834C4F835
:101FA000BC74C4F8C074C4F8C874C4F8CC745BF0D2
:101FB00035F894F8ED34202BD9B21AD194F8EC34DA
:101FC000012B16D0242384F8ED34D4F8AC341A68ED
:101FD00022F001021A601A6822F480521A601A680C
:101FE0001A601A6842F001021A6084F8ED1484F84D
:101FF000EC740021F07E58F0C5FCF37E0124194DED
:102000005A0903F01F03002104FA03F345F82230B4
:10201000B07E58F0B7FCB37E5A0903F01F039C4012
:1020200045F82240BDE8F88F4FF0EAFFD9F81C30A0
:10203000E8E6E6461BE7013165E7BCF10F0FF8D192
:102040000023A0E7201B0024CC1F0024001C005804
:10205000286B6E4E00001643002474490000704245
:1020600000FFFF0000E100E00044025848190A08A0
:102070002DE9F843B14C04EB0017D7F86C36002B70
:1020800000F0BF8005460601B7F8760658F0AAFCB6
:10209000B7F87636012103F01F025B09023B01FA13
:1020A00002F2082B0FD8DFE813F008011001180125
:1020B000200128010900300138014001A04BD96FEF
:1020C00021EA0202DA67A319013593F87006EDB22E
:1020D0000EF0A0FA074610B11223C5718371A3193F
:1020E00093F871060EF096FA814610B11323C5716C
:1020F0008371A31993F872060EF08CFA804610B122
:102100001423C5718371344448462E2194F87426F3
:10211000FFF70CFE94F875260E214046FFF706FEE9
:1021200094F873262E213846FFF700FED4F86C365B
:1021300084491A688B4222F001021A6063D0824AF5
:10214000934200F08F8002F58062934279D17C4AFD
:10215000D2F8901041F40041C2F89010D2F89010DB
:1021600021F40041C2F89010DA6842F00042DA60CF
:102170009A6822F4F0729A601A68D60741D47349BB
:102180009D68D1F89823D1F8A04344EA0200D1F821
:10219000882310436E4A2A401043D1F89423986054
:1021A000DD68D1F88403ED007BD50243D1F88C03C0
:1021B000DE68B4F5800F42EA0002D1F89003654D65
:1021C00042EA0002D1F89C0305EA060542EA000251
:1021D000D1F8800300F4C02600F4006042EA060251
:1021E00042EA0502DA601A6822F4006242EA00025A
:1021F0001A6002D1D1F8A4231A641A6D22F00102E8
:102200001A65BDE8F8834E4AD2F8981041F480511F
:10221000C2F89810D2F8981021F48051C2F89810A2
:102220004D4A9342A0D1464AD2F89C1041F0200179
:10223000C2F89C10D2F89C1021F02001C2F89C102A
:1022400092E7464A93421BD13D4AD2F8981041F496
:102250000051C2F89810D2F8981021F40051C2F839
:10226000981081E7364AD2F8901041F48041C2F8C4
:102270009010D2F8901021F48041C2F89010CFE76E
:10228000374A9342CCD12E4AD2F8981041F48011AB
:10229000C2F89810D2F8981021F48011C2F8981062
:1022A00062E7B2F1806F80D1B0F5800F7FF47DAF2F
:1022B0001D6845F480551D6077E7214BD3F89810D1
:1022C00021EA0202C3F89820FDE61D4BD3F89010D6
:1022D00021EA0202C3F89020F5E6194BD3F89410D6
:1022E00021EA0202C3F89420EDE6154BD3F88010E2
:1022F00021EA0202C3F88020E5E6114BD3F88410EE
:1023000021EA0202C3F88420DDE60D4BD3F88C10DD
:1023100021EA0202C3F88C20D5E6094BD3F88810D5
:1023200021EA0202C3F88820CDE6054BD3F89C10C1
:1023300021EA0202C3F89C20C5E600BF201B00244E
:1023400000440258003001400038004000000024E2
:10235000E0FFBF8FFFFF39D8001400580034014060
:102360000050014008B10022B8E470470E4B70B530
:10237000D3F86464002E14DD0C4C002503E0B54254
:1023800004F120040DD0237F0135002BF7D0E06845
:1023900000220028F3D0217D2034FFF79FFCB542B6
:1023A000F1D1012070BD00BFFC1000203C040020D2
:1023B000F8B590F8EE311C09013C062C0FD81B4EE5
:1023C000054603F00F0306EB4402B2F8B80240FAE8
:1023D00003F2D20703D595F8F971012F01D001203E
:1023E000F8BD07FA03F33444013B18405DF034FABA
:1023F00094F8C82213180E4A02EBC30152F8332096
:102400008B8810691840EBD0002395F8EF2108461F
:10241000022185F8F931FFF761FCD5F850213846E3
:10242000136843F008031360F8BD00BF48190A0899
:10243000EC210024014B53F8200070475040005815
:10244000014B43F8201070475040005819481A4B70
:1024500001681A4A41F4807130B4016082B0D3F847
:10246000F410FF24CA2041F48031C3F8F410D3F8EB
:10247000F41001F4803101915321019D54625062A6
:102480005162D3F8D030DB010CD40D4B00210D4A42
:1024900043F8041B9342FBD1084B0B4A1A6502B068
:1024A00030BC7047126D084B9A42EED102B030BC7E
:1024B000704700BF004802580044025800400058CE
:1024C000544000586C40005831666542F0B50446EF
:1024D000D0F85C01454B83B0A16804F5967204F115
:1024E000E0070E68C1B220F0FF0001921039A3FB93
:1024F0000131090959F08CFED4F81C110023019A0E
:10250000012984F8203118D0042916D0102958D078
:10251000402912D0B1F5807F56D0B1F5806F53D0ED
:10252000B1F5805F58D0B1F5803F4FF03C030CBF50
:102530006FF0080C6FF4006C01E06FF0080C06F10E
:1025400018053046E95801EA0C01E950D4F81C118D
:1025500059F0FEFAD4F81C31012B16D0042B14D0FC
:10256000102B0FD0402B10D0B3F5807F30D0B3F5B7
:10257000806F2DD0B3F5805F32D0B3F5803F06F188
:10258000540502D04FF4006100E008212B683A4660
:10259000D4F85C010B4340212B60C4F8E810C1B2B1
:1025A000124B20F0FF001039A3FB0131090959F04B
:1025B000DFFDD4F85C21136843F01003136003B00F
:1025C000F0BD6FF4006CBAE76FF0080C0423B6E7B7
:1025D00006F11C050821D9E76FF4006C0423AEE76F
:1025E00006F11C054FF40061D0E700BFABAAAAAA10
:1025F0002DE9F04FDFF848B185B09BF8004024B9D1
:102600000124204605B0BDE8F08F474BD3F838537E
:102610000EF01CFE454A92F8B83B002B00F0BC813E
:10262000434B02F17C070BF5A7640026A3FB0513BF
:10263000404D5B09A5FB0315ED0805EB8505A3EBF4
:102640004505D2F87C3BC31A0193EBB207EB850535
:10265000029302F557730093019A002A04DBD4F821
:102660002431934200F37C814FF4B47303FB06B32F
:1026700093F85836002B00F0C080D4F85C11A368A2
:102680002D481A68CBB221F0FF01103BA0FB0303D9
:102690002A481B09C35C19444B68A1891FFA83FEB1
:1026A000D368CEF1160E23EA0103BEF1070FD36003
:1026B00040F2A3801D4A0121D2F864338A460133D7
:1026C000C2F864330022D4F8643190469C460393E8
:1026D0005CF8049B48461DE0DCF80090B8F1140F4C
:1026E000A9EB000348462DDC13F1080948BF03F1AC
:1026F00017094FEA291308EB291803F1FF390131B3
:1027000002FA03F30CF1040C0AFA09F28E4542EACC
:10271000030217D38E45DFD8C8F11503DCF800009B
:102720004FF01508E9E700BF201B0024FC10002033
:102730001F85EB51CDCCCCCCABAAAAAA54AC0A08CD
:1027400004000020B8F1150F40F000819649C2F353
:102750008423C2F3441001EB830301EB8000D3F820
:10276000D032D0F8D0021B0243EA001302F01F005F
:10277000C2F3C43201EB800001EB8202D0F8D01228
:10278000D2F8D0220B4343EA023383EA132282EACF
:10279000121202F00F020F2A40F0D880C3F30F1379
:1027A0004FF6FF72934200F0D180B3F5606F00F0F6
:1027B000DC80009A938197F85820029882420CD0CE
:1027C000A9683A68521A3A607A68296B521A7A6094
:1027D0000022AA602A6387F858003A6801323A60FA
:1027E000AA680132AA604FF6FF72934205D17B6856
:1027F00001337B602B6B01332B63009B204601363A
:102800005C3714335C3504F5B4740093FFF75EFE57
:10281000664B93F8B83BB3423FF71EAF63480121C4
:10282000002280F86014C0F87C2B002B3FF4E8AE47
:102830009BF81026DBF8540612F0020FDBF8402557
:1028400011680A6A0CBF024342EA8002012B0A6245
:102850003FF4D6AE9BF87827DBF8BC0712F0020FE6
:10286000DBF8A82611680A6A0CBF024342EA80021C
:10287000022B0A623FF4C4AE9BF8E028DBF824097F
:1028800012F0020FDBF8102811680A6A0CBF02432D
:1028900042EA8002032B0A623FF4B2AE9BF8482A58
:1028A000DBF88C0A12F0020FDBF8782911680A6A4B
:1028B0000CBF024342EA8002042B0A623FF4A0AE3E
:1028C0009BF8B02BDBF8F40B12F0020FDBF8E02AD8
:1028D00011680A6A0CBF024342EA8002052B0A62B1
:1028E0003FF48EAE9BF8182DDBF85C0D12F0020F52
:1028F000DBF8482C11680A6A0CBF024342EA8002E6
:10290000062B0A623FF47CAE9BF8802EDBF8C40EE7
:1029100012F0020FDBF8B02D11680A6A0CBF0243F7
:1029200042EA8002082B0A627FF46AAE9BF8E83F15
:10293000DBF8182F13F0020F1D4B1268D96A136AC7
:1029400014BF43EA81030B43136259E6174AD2F8D6
:1029500060330133C2F86033B6B14FF6FF732AE734
:102960000024204605B0BDE8F08F12494A7802EBFA
:10297000420201EBC2023244527C0D2A7FF419AFAD
:10298000802200998A7716E7039958220A485EF058
:10299000E5FD4FF6FF730EE704490122C1F87C3BC9
:1029A00081F860242DE600BF48190A08FC100020B9
:1029B00004100020201B002404150020D0F8501122
:1029C0002422F8B5C0F8D02104460A6800238068A4
:1029D00004F5A87522F001020A600B604B608B6061
:1029E00094F805C0C4F8D83184F8CC31C4F8D0319B
:1029F000C4F86831C4F8D431C4F87031C4F8643113
:102A00004FEA8C23B44A03F48053C4F85401914232
:102A1000C4F858314FEA0C3303F40053C4F85C3166
:102A20004FEA0C2303F48063C4F8603100F0AE81F8
:102A3000237913F0010002D00422C4F8642113F0BA
:102A4000020305D0D4F8642142F00802C4F86421DE
:102A50001CF0010F0DD048B1D4F8782142F00202E9
:102A6000C4F878214FF48032C4F88021002B40F064
:102A700081819A4B03F12C0053F8042B944200F00F
:102A80003F819842F8D11CF0080F40F04F81D4F8F4
:102A9000D031002B00F09C8124232846C4F8D0318B
:102AA0000B6823F001030B604FF08CFE012815D05A
:102AB000D4F87831002B40F09181D4F85031284679
:102AC0005A6822F490425A609A6822F02A029A6068
:102AD0001A6842F001021A6059F098FC2379DA076B
:102AE0006DD5D4F82C21002A00F05F810023D4F8A2
:102AF000341104F13C06E2634FF48062C4F8B8106C
:102B00003046E264C4E91133C4E91433C4E918332C
:102B1000C4E91A334FF48033E3654FF48073A3653F
:102B20005AF0CAFA30464EF009F9D4F8D431C4F854
:102B3000C861202B65673DD1E368626999B2CAB369
:102B4000B1FA81F04009A9B394F8CCC1BCF1010FEE
:102B500030D02227C4F8D80194F870C0C4F8D471DA
:102B60005F4FA4F8AC110121A7675E4F8C45C4F8F4
:102B7000A821E7675C4FC4F88C0084F8CC11C4F836
:102B800088700ED094F8717084F87010012FD4F80A
:102B9000501100F02B814FF4006384F87000C4F8EA
:102BA0009030102100222023C4F8D81184F8CC21C1
:102BB000C4F8D031E26B23795268C4F844219B07F2
:102BC00040F18880D4F83021002A00F0E38000230F
:102BD000D4F8381104F1B406C4F8B420C4F8C030F5
:102BE0004022C4F8D0303046C4E93233C4E9363329
:102BF000C4E938334FF48033C4F8D4304FF48063E1
:102C0000C4E92E12C4F8C4305AF056FA30464EF0D9
:102C100095F8002840F0B980D4F8B420334B3448FC
:102C20003449824218BF9A42C4F8C461C4F8EC50D7
:102C300000F160000CBF012300232F4C8A4208BF23
:102C400043F001033031A24208BF43F00103603476
:102C50008A4208BF43F001033031824208BF43F08B
:102C6000010300F568708A4208BF43F0010301F5D3
:102C70005C71A24208BF43F0010304F568748A4204
:102C800008BF43F001033031824208BF43F0010323
:102C900060308A4208BF43F001033031A24208BFCE
:102CA00043F001038A4208BF43F0010330318242FE
:102CB00008BF43F001038A4208BF43F001033BB958
:102CC0000E4BD31AB3FA83F35B09002B00F0A780F5
:102CD00000235360F8BD00BF000C0058BC1C00204E
:102CE000C9D20808FDD2080801D308081000024024
:102CF000280002404000024058000240B804024050
:102D0000002C3FF4C0AE94F8F831002B3FF4BBAE7A
:102D1000D4F878311CF0080F43F00803C4F8783178
:102D20004FF40043C4F888313FF4B1AED4F8D03149
:102D3000002B50D024232846C4F8D0310B6823F050
:102D400001030B604FF03EFD01283FF4C7AED4F8FD
:102D50007831002B46D1D4F8503128465A6822F4F5
:102D600090425A609A6822F022029A609A6842F071
:102D70000802ACE6D4F8783143F00103C4F87831A6
:102D80004FF40033C4F87C3173E6FEE70423C4F843
:102D900074314DE6D4F8DC311A6842F080021A60D2
:102DA0001A6842F040021A60F8BDD4F8DC211168BC
:102DB00041F480711160916841F0010191601168E6
:102DC00041F020011160116841F010011160F6E638
:102DD00084F8CC3160E684F8CC31ABE728464FF07C
:102DE000CDFF6AE628464FF0C9FFB4E79BB2243115
:102DF00030464EF0C3F900287FF4D3AED4F85031FA
:102E000084F8CC011A6842F480721A609A6842F021
:102E100001029A609A6842F040029A60CAE65360E2
:102E2000F8BD00BFF8B50446EFF31185502383F3D6
:102E30001288D0F830311B6803F001031BB1EDB2EA
:102E400085F31188F8BDD0F8D021D0F8D4110A4309
:102E500002F02102212AF2D0D0E909218A424FD082
:102E60004BD800691A46431A9BB2A262002284F82A
:102E7000E021D4F8D021202AE1D1A2695118DED076
:102E8000B3FA83F25209002BD9D094F8CC0101286F
:102E9000D5D02120A4F8A6314FF0010CC4F8D821D8
:102EA000C4F8D001D4F8C401C4F8A011A4F8A43126
:102EB00084F8CCC170B31D4E90F834E0C6631C4E4C
:102EC000E645026506641B4EC6640CD090F835607A
:102ED000D4F85071664580F834C015D04FF40063C3
:102EE00080F834204365102100222023C4F8D81133
:102EF00084F8CC21C4F8D031A1E7531A9BB2B4E7CF
:102F0000012380F8E0319AE707F128024EF036F904
:102F10000028E8D1D4F8503100224021196284F809
:102F2000CC219A6842F080029A6088E7A1D2080812
:102F3000C5D2080801D308082DE9F8434D4C04EB2D
:102F40008004D4F8C04B002C44D0D4F8E8511F467C
:102F5000494B0646A1602046236090466B68C4F842
:102F6000DC31AB6B63616B6BA361EB8FE360AB8FA9
:102F70002361424BC4F8E4310DF0FAFE6B68A88D72
:102F8000C4F85031002863D194F8EE010DF042FBF3
:102F9000022117F00802034694F8EC9184F8F91125
:102FA0001BD060B317F0510F4FF00B0206F1010672
:102FB00014BF0A211A2117F0410FC671827114BF84
:102FC0004023202394F8EF211943FEF787FED4F81D
:102FD0002C314BB32046BDE8F88318F0020F0ED019
:102FE00068B14FF00B0C3B0680F806C006F1010CEF
:102FF00080F807C02FD494F8EF21FEF76FFE484603
:103000000DF008FB0028E2D018F0010FDFD00C22F1
:1030100001360221C671827194F8ED21FEF75EFE41
:10302000D4F82C31002BD5D195F8321095F830001A
:10303000890957F0A7FC95F830300122104903F0B8
:103040001F005B098240204641F82320BDE8F88339
:1030500057F0C8FC98E7D4F850714FF0010C2021CC
:103060003B6823F008033B6084F8F9C1FEF736FEA5
:10307000C5E700BFFC100020981C0A08B123040813
:1030800000E100E0BFF34F8F0549064BCA6802F428
:10309000E0621343CB60BFF34F8F00BFFDE700BF7B
:1030A00000ED00E00400FA051C481D4AC1681D4BF4
:1030B00010B44FF6FF0485B021401B4C0A43C26098
:1030C000D3F8D010D3F8DC20C4F84C1A42F00052E8
:1030D000C3F8DC20D3F8DC2002F000520192019A00
:1030E000D3F8DC2042F08042C3F8DC20D3F8DC20A7
:1030F00002F080420292029AD3F8DC2042F00042B1
:10310000C3F8DC20D3F8DC3003F000430393039BC7
:1031100005B05DF8044B0EF021B800BF00ED00E0F3
:103120000005FA0500440258201B002408B51D487C
:103130000023C0F88430BFF34F8F436923F48033FA
:103140004361BFF34F8FD0F8803043F6E074C3F390
:103150004E3CC3F3C90E4FEA4C1C0CEA0401734603
:1031600041EA8372013BC0F874225A1CF8D1ACF1D9
:10317000200C1CF1200FF0D1BFF34F8FBFF36F8FE6
:10318000BFF34F8FBFF36F8F4369002223F40033E7
:103190004361C0F85022BFF34F8FBFF36F8F72B6F9
:1031A000FFF770FF00ED00E003689B0AA3F58013B2
:1031B000522B57D870B53E4C14F803C0BCF10D0F1C
:1031C0004FD840798508002951D04FEA900E4C2401
:1031D00038480CEB8C0304FB0C040CEB4303D4F8D1
:1031E000506A02242B4404FA0EFEF46800EB8305B7
:1031F0004EEA0404A966AA67F460EFF31184502331
:1032000083F312882C2303FB0CF3C1184A6E52B3CC
:10321000131DC1F88820284A2C21284D01FB0CF1F0
:1032200005EB010E14310A4452F8041B19B1196060
:1032300052F8043C04339645F6D10022E4B21A60F9
:1032400084F311882C2303FB0C03D3F888302BB3B1
:103250004C2303FB0C00D0F8502AD36843F0010341
:10326000D36070BD7047144A24331344D4E7114827
:103270004C23022403FB0C0304FA05FED3F8506A26
:103280000CEB8C03F4680CEB430324EA0E042B4490
:10329000F46000EB8304A166A267AEE74C2303FB56
:1032A0000C00D0F8502AD36823F00103D36070BD1E
:1032B00048190A08201B0024841B0024A81B002492
:1032C00003689B0AA3F58013522B00D97047144A58
:1032D000D35C0D2BFAD84FF04C0C10B4114C79B9CB
:1032E000417902220CFB03405DF8044B21FA02F302
:1032F000D0F8501A9A40CB6823EA0203CB6070479B
:10330000417902220CFB03405DF8044B21FA02F3E1
:10331000D0F8501A02FA03F3CA681343CB6070471F
:1033200048190A08201B002403689B0AA3F5801390
:10333000522B10D8084AD25C0D2A0CD840790223AF
:1033400006494FF04C0CD8400CFB02128340D2F8D7
:10335000502ADB431361704748190A08201B0024D8
:1033600001490248FDF7B4BB841B00240000014062
:1033700001490248FDF7ACBB841B0024000001405A
:1033800002494FF08040FDF7A3BB00BFB01B0024F3
:1033900001490248FDF79CBBDC1B002400040040EF
:1033A00001490248FDF794BB081C002400080040B6
:1033B00001490248FDF78CBB341C0024000C00407E
:1033C0002DE9F843194E3569F3681D4010D04FF0D0
:1033D0000047DFF85C80B5FA85F227FA02F31F2A6E
:1033E0006FEA030305EA0305336103D0002DF2D130
:1033F000BDE8F883D8F86831A3B103F1FF390023A1
:103400001FFA89F9C8F86831D8F86441002CEDD06A
:1034100023682046494698476468002CF8D1002D5F
:10342000D9D1E5E7F16A1FFA81F9EDE70010004014
:10343000201B002401490248FDF74ABBB81C0024A8
:103440000004014010B5064C064804F5CC71FDF7A8
:103450003FFB04F5F8710448BDE81040FDF738BBA8
:10346000201B002400040140001C004001490248C8
:10347000FDF72EBBE41C002400180040014902485F
:10348000FDF726BB3C1D00240020004001490248F6
:10349000FDF71EBB681D00240040014001490248A1
:1034A000FDF716BB941D0024004401400149024869
:1034B000FDF70EBBC01D0024004801402DE9F0417E
:1034C0004FF425728EB000217B485EF0BBF87B4B39
:1034D0007B4E4FF08041D3F8F02006F68415374636
:1034E00042F00102DFF8E08106F66814C3F8F0202C
:1034F000D3F8F02002F001020092009AD3F8E820FD
:1035000042F00102C3F8E820D3F8E82002F00102FB
:103510000192019AD3F8E82042F00202C3F8E820B1
:10352000D3F8E82002F002020292029AD3F8E820CF
:1035300042F00402C3F8E820D3F8E82002F00402C5
:103540000392039AD3F8E82042F00802C3F8E82077
:10355000D3F8E82002F008020492049AD3F8E82095
:1035600042F01002C3F8E820D3F8E82002F010027D
:103570000592059AD3F8E82042F02002C3F8E8202B
:10358000D3F8E82002F020020692069AD3F8F02041
:1035900042F00202C3F8F020D3F8F02002F0020259
:1035A0000792079AD3F8E82042F04002C3F8E820D7
:1035B000D3F8E82002F040020892089AD3F8E820F5
:1035C00042F08002C3F8E820D3F8E82002F080023D
:1035D0000992099AD3F8E82042F48072C3F8E820EF
:1035E000D3F8E82002F480720A920A9AD3F8F02005
:1035F00042F48032C3F8F020D3F8F02002F4803295
:103600000B920B9AD3F8F02042F40032C3F8F0206A
:10361000D3F8F02002F400320C920C9AD3F8F02088
:1036200042F48022C3F8F020D3F8F03003F4802372
:103630000D930D9B4246002301E054F83320914244
:103640000BD00133112BF8D11C37002057F0CAF9E9
:10365000AF420CD057F81C1CECE71A4A1C3702EB9F
:10366000C303B3F8080D57F0BDF9AF42F2D14FF0E4
:103670008041154F154C3A46002301E054F83320A1
:1036800091420BD00133112BF8D11C36002057F09A
:10369000A9F9AE420CD056F81C1CECE7094A1C36BE
:1036A00002EBC303B3F8080D57F09CF9AE42F2D118
:1036B0000EB0BDE8F08100BF841B00240044025816
:1036C000E41C0A0848190A08000001404C260A08B0
:1036D000800AA0F5801052280DD8074B1A5C0D2ADD
:1036E00009D8064B4C2101FB0233D3F8502A13684A
:1036F00043F001031360704748190A08201B002497
:1037000038B590F83DE08446BEF1020F5FFA8EF0C6
:1037100018D014469CF83D20012A02D102228CF8D0
:103720003D200C290DD8DFE801F05D0C0C0C290CB4
:103730000C0C430C0C0C0E004032214628464DF078
:103740001DFD002038BDDCF83050334AEA63334AAF
:10375000EA6495F83420012AF3D00121DCF8002036
:1037600085F8341095F835100129E5D000234FF481
:103770000062184685F834306A6538BDDCF8285098
:10378000254AEA63254AEA6495F83420012AD8D00C
:103790000121DCF8002085F8341095F83510012956
:1037A000E4D13832214628464DF0E8FC002038BDEF
:1037B000DCF82C50184AEA63184AEA6495F8342079
:1037C000012ABED00121DCF8002085F8341095F8DC
:1037D00035100129CAD13C32214628464DF0CEFC95
:1037E000002038BDDCF824500B49DCF80020E963E8
:1037F0000A49E96495F834100129A2D0012185F81D
:10380000341095F835100129B0D1343221462846BC
:103810004DF0B4FC002038BD41D20808E9D10808B9
:103820001F4B984210B50ED003F5806398420AD022
:103830001C4A03F58043984218BF904203D003F519
:10384000806398421BD14EF0DBFB174B1749DC69B4
:10385000DA69C4F3022CC2F3022201EB0C0393F8E1
:10386000883203F01F03D8400F4B11491B69C3F383
:10387000C03342EAC303CB5C03FB00F010BD4EF043
:10388000BFFB094B0949DC69DA69C4F30214C2F3CE
:1038900002120B1993F8883203F01F03D840E3E7B4
:1038A00000000140004001400044025848190A0845
:1038B00030AC0A082DE9F04FB34B91B00024DFF88B
:1038C000F0820193B14BA3F68C5BB14E0025DFF87B
:1038D000BC92B30AA3F58013522B57D81BF80330C0
:1038E0000D2B53D818F90370AA4B93F8D63E012B31
:1038F00040F01081012F3FD14FF0000A5146384669
:1039000012F09AF912F020FA90F800C0BCF1000F02
:1039100018BFBCF1540F14BF4FF0010C4FF0000C56
:1039200040F0F4800AF1040A1FFA8AFABAF1100F83
:10393000E4D1002C00F0B580934A00210DE01BF883
:1039400003300D2B10D818F90330BB420FD00131D2
:1039500002F58672A14280F2A080906803689B0AFB
:10396000A3F58013522BEAD90023BB42EFD1437950
:1039700099F805009842EAD10135082D14D059F87C
:103980001C6FB30AA3F58013522BA7D9814B93F870
:10399000D63E012BF0D001220027022BACD1002A09
:1039A000AAD00135082DEAD1019B013403F58673B5
:1039B000042C019389D1784F0026DFF8F8B1774BBA
:1039C000D3F86434B34265DDD7F80C80B8F1000F4A
:1039D00060D0734BB8F804105D68D8F800003B7CE9
:1039E000002DDFF8D4C10193B1FA81F38444C3F10F
:1039F0001F0902934FEA9C2C40F3A980624A0024DD
:103A000005E0013402F58672AC4200F09D80136837
:103A10006345F6D14FF486735B4A03FB0424019B94
:103A20000322C7F8049001363B744FEA4903C7F8F4
:103A30000C8002FA03FCBC6188F80620012288F899
:103A4000076002FA03F5A36C43EA0C03A364236D39
:103A50002B432365524B1B78002B60D0636D02FA19
:103A600009F943EA0903636581611FFA89F1D4F812
:103A7000AC00FCF7F1FA20462037FCF7C1FA01232D
:103A8000082E0BF1180B07F8043C07F8033C0BF861
:103A9000073C94D111B0BDE8F08FBCF1000F7FF46A
:103AA0006BAFD9F8080000223E4B04E001320C3322
:103AB000102A00F02A8359688842F7D152B2304662
:103AC00099F80510FEF73AF8374A40680023516824
:103AD0000133884217D0102B02F12402F7D14FF0A6
:103AE000FF3303EBC303314A02EB830393F85C31EA
:103AF000002B7FF441AF254BC5EBC50503EB8505D6
:103B0000019B9D6050E7DBB2013BEAE7002C7FF4AC
:103B100013AF31E7B7F1080218BF01223DE7029D5C
:103B20004FEA014C02FA09F1C5F12F0589B202FAF8
:103B300005F51A46636D2B436365C0F818C0D4F8C9
:103B4000AC00FCF789FA96E7032C00F3E9804FF408
:103B50008673134A03FB05231869002800F0C1820D
:103B60005422C3F808C00CF1010C0E4C83F810214C
:103B700083F811C16B1C0A4A53600022054B93F86D
:103B8000ED3E039383681EE00C000020D4260A0853
:103B900000040140201B00243C040020FC100020F5
:103BA00004000020800000244001002400000024C4
:103BB00044AC0A08B81000200000FEA701320C3403
:103BC000102A00F0A28261688B42F7D1417952B28B
:103BD0000068FDF7B3FF4FF48672B14BDFF804A322
:103BE00002FB0532D0E90141C2E9074100225146FA
:103BF0004B6801329C4217D0102A01F12401F7D101
:103C0000A84BA94693F83821002A00F05C82A64808
:103C1000A649A74AA74BC0F8101CC0F8082CC0F84A
:103C2000183C11B0BDE8F08FD2B24FF48671013A62
:103C300001FB05F39B4902EBC202049301EB8202F4
:103C40009749194492F85C31B1F810010593002BA3
:103C5000DDD1049CA2F85C01974BA210086903FB1C
:103C600002F2964B0068C2EBC20C02EBC20203EBFD
:103C70004C1C03F5607303EB4212D8F80030C1F816
:103C8000B4C0C1F8FC203322CB60C1F8B8208C222C
:103C9000C1F80021FFF7C4FD894B1C19039B062BBB
:103CA00000F00E82072B874B874908BF1946874BC8
:103CB000874A18BF1A464FF48673B0FBF2F2B0FB86
:103CC000F1F1013A7648013903FB050392B2A3F8FA
:103CD000BC10A3F87420226600220393A4F8582095
:103CE0006266E265049A02F1580100F1080211448B
:103CF0001A69106858F0A8F8039B1A6910680392B3
:103D0000036843F08003036053790C2B0DD8DFE880
:103D100003F06F0C0C0C670C0C0C5E0C0C0C5500BB
:103D200003236C4A82F8EC3E71E74FF486735C4AD9
:103D300003FB052359694FF0600C02680023CDF89E
:103D400020C04FF4807C0A9322F00102CDF838C0E5
:103D50004FF0010C0D930F930223CDF824C04FF0C8
:103D60000A0CCDE90BC3026008AA57F0F1FE4C4BD8
:103D70004FF4867202FB0532039B526919680023D7
:103D8000012A3DD0042A3BD0102A00F0AF81402AFE
:103D900036D0B2F5807F00F0AC81B2F5806F00F0D4
:103DA000A881B2F5805F00F0A981B2F5803F4FF0A5
:103DB0003C030CBF08224FF4006222E04FF48673EC
:103DC000374A4FF4805103FB05235961B3E74FF4A1
:103DD0008673334A4FF4807103FB05235961AAE7C8
:103DE0004FF486732E4A102103FB05235961A2E785
:103DF0004FF486732A4A012103FB052359619AE790
:103E0000082201F1180050F803C042EA0C02C25027
:103E1000039B1879002840F03E81214B4FF48672B5
:103E200002FB053200231069D1690068026842F084
:103E300001020260DAF804200133914200F0278188
:103E4000102B0AF1240AF5D14FF0FF33154A03EB8A
:103E5000C30302EB8303D3F840011F4B98420CBF0E
:103E6000A020A12056F0BEFD0D4A4FF4867303FB3F
:103E700005231A6951790C2900F20681174B03EBCF
:103E80004103B3F86CCED2F800E04FF48673044AD5
:103E90001349704603FB0523A3F818C000232AE04A
:103EA0000400002000000024FC10002069D8040851
:103EB00065D8040871D804086B4CA407E0430124BA
:103EC0000C0000201055220044950800D0DD0600AB
:103ED00040771B00201B00240000024048190A08FC
:103EE0006815002040010024904200F00581013354
:103EF000042B00F0078151F83320002AF4D1844AC2
:103F000086461046D2F868240132C0F8682400EBD7
:103F1000C302DB00C2F86CE41944059823469022E2
:103F2000B1F804E0DFF804A24CEA0E0CA1F804C0DA
:103F30007849FDF769FE4FF48673774A4FF4403EA7
:103F400040214FF4805C03FB05250023E8690268EB
:103F500042F010020260026842F014020260C4E9FA
:103F60001F33C4E92733C4E929334FF480632A6A35
:103F7000C4F898E0C4F88430A167C4F89420D5F858
:103F8000B820C4F89020C2B220F0FF00103AAAFB7B
:103F90000231EA68049B1832C4F888C04FF4804CA0
:103FA0000909226703F170025C4B1A44D5F8B4305A
:103FB000C4F88CC0636758F0DBF8E869049B4FF4E1
:103FC0000031D0F800E04FF4006C03F1B802534B1D
:103FD000C4F820E0D0F814E01A440023C4F824E028
:103FE000D0F804E0C4F828E0D0F808E0C4F82CE0E9
:103FF000D0F80CE0C4F8C830C4F830E0C4E930337D
:10400000C4E93933C4E93B332B6AC4F8E0100393A5
:104010004FF48063C4F8CC30039BC4F8DC30D5F88F
:104020000031C4F8D830C3B220F0FF00103BAAFB27
:104030000331EB68C4F8D0C010330909C4F8B830B4
:10404000D5F8FC3003934FF48043C4F8D430039B7D
:10405000C4F8BC3058F08CF8EB69B8F804101A6852
:10406000D8F8000062635A69A2635A68E2639A68EA
:104070002264DA6862641A6842F010021A601A68F0
:1040800042F014021A60CAE44FF0000CFBE6DBB207
:104090000593013BDAE607910CF0BCFA079906900C
:1040A00048B1039B0221DA79FDF718FE069B5422E2
:1040B000DA80039B19684B6C43F400434B64ACE615
:1040C0001749184AF7E5144A4FF4867808FB09287F
:1040D00098F8111198F8102183F8391183F83821D4
:1040E00095E50223104A82F8EC3E90E54FF4006219
:1040F00087E60822042384E6DB000DE74FF4006224
:1041000004237EE600239B88FFDE00235B68FFDE3E
:10411000FC10002001000000040000200C00002022
:10412000882A1100A0BB0D00201B0024ABAAAAAA5C
:104130002DE9F04F00228FB02F21074611F05CFED1
:10414000D0B1B04C06464379D0F80080A4F838349A
:10415000FDF722FD80B1456875B1DFF8E0B20022BD
:1041600059464B68013224319D4210D0102AF8D1B3
:10417000A54B93F838211AB100200FB0BDE8F08F9D
:104180002F21104683F8392183F83811F5E7D2B290
:10419000DFF874A2013A02EBC2020AEB820292F843
:1041A0005C91B9F1000FE7D12F2183684046C4F834
:1041B000EC83A2F85C110393FFF732FB934A904221
:1041C00080F0FF8001234A46029340460192FFF7A8
:1041D00027FB029B019A8E49C4F8F023B0FBF3F24F
:1041E000120A0020A1FB02328A4BC4F8FC03110919
:1041F000C4F8F4031209A3FB0131C4F8F8234A08F8
:10420000A4F8F02E5200A4F8EE2E94F8292402F01F
:10421000FF01002A00F0E38002227F49D4F8EC037A
:1042200084F829244EF0F4F90122384684F8342425
:1042300084F82A2484F82B2484F82C2484F82D2450
:1042400084F82E2484F82F2484F8302484F8312430
:1042500084F8322484F8332484F829240CF0DAF921
:10426000C4F8F40E28B12F21C1804E21F279FDF758
:1042700035FD6A4A0021039BC4F8041FC4F8FC3EC4
:10428000C4F8141FC4F81C1FC4F8241FC4F8281F46
:10429000D2F8D800C4F8F85E40F00100C2F8D800A7
:1042A000D2F8D80000F0010005900598D2F8D800A7
:1042B00040F00200C2F8D800D2F8D82002F0020282
:1042C0000692069A4022C4F8002F4FF48062C4F888
:1042D000082F4FF48052C4F80C2F4FF48042C4F8DA
:1042E000102F4FF40032C4F8182F0322C4F8202FE7
:1042F00094F838240C2A75D8494901EB4202B2F8E7
:10430000887EB846083747485946002204EB870C98
:10431000CCF8EC03A0F60C30C4F8300F486801323A
:104320002431854264D0102AF8D14FF0FF3202EBDD
:10433000C2020AEB820A3C4ADAF8400190420CBF02
:10434000A020A12056F04EFB0022DBF80410013221
:104350000BF1240B8D4248D0102AF6D104EB8707CD
:104360004846434660223149FDF74EFCD7F8EC033E
:104370004CF0E4FC00287FF4FFAE60210C90B37990
:10438000079159000D90DB00089001F002010B909D
:1043900003F00803B4F838242548CDE9091307A928
:1043A00055F058FC00287FF4E7AEB379B4F8381420
:1043B0009B071F481FD54EF0B7F9B0FA80F04009AF
:1043C000DBE64046FFF72CFA1A4A1B490244A1FBE0
:1043D0000232920D013A92B2531C0293F5E684F830
:1043E000281419E788460F468CE75FFA82F9B5E78B
:1043F000D2B2013A9BE74EF081F8B0FA80F0400962
:10440000BBE600BF201B002400000024006CDC027F
:10441000598B4F01ABAAAAAA101F002400440258CE
:1044200048190A08182A0024000002409D010000D3
:104430000C1F002400366E01819F5E16400100248F
:10444000830AA3F58013522B00D970472DE9F04160
:1044500015460F4AD65C0D2E17D80E4C4FF04C085F
:10446000013908FB064789B2C7F85C1AFFF7D8F98B
:1044700007F65421B0FBF5F2013AD7F8500AC7F815
:10448000542ABDE8F0414EF0C3B8BDE8F08100BF4A
:1044900048190A08201B0024830AA3F58013522B15
:1044A0006BD82DE9F0411646794A84B0D75C0D2FC0
:1044B00060D8DFF804824C25044605FB0785D5F853
:1044C000503A834256D00139C5F8500A89B2C5F82E
:1044D0005C1AFFF7A5F90023B0FBF6F2C5F8603AC5
:1044E000013AC5F8583AC5F8643A95F88D3AC5F8D6
:1044F000542A03F0FF02002B40D04C23654903FBF4
:10450000078503FB07110223D5F8500A85F88D3A79
:1045100004314EF07DF8012385F8983A85F88E3AFB
:1045200085F88F3A85F8903A85F8913A85F8923A6D
:1045300085F8933A85F8943A85F8953A85F8963A4D
:1045400085F8973A85F88D3A534B9C4219D0B4F1CF
:10455000804F16D0A3F57C439C4212D003F58063B4
:104560009C420ED003F580639C426CD003F57843E7
:104570009C4268D004B0BDE8F081704785F88C2A71
:10458000BBE74C234FF48051002203FB07830091CB
:1045900093F88C1A03920129CDE90122EAD0022175
:1045A000D3F8500A012483F88D1A3C4985682940C4
:1045B000816083F88D4A83F88C2A4C22002302FB09
:1045C00007820293CDE9003392F88C3A012BD1D0C7
:1045D000D2F8503A0221304882F88D1A83425A6844
:1045E00099682CD000F58060834228D022F07002B8
:1045F0002B485A602B4A934218BFB3F1804F0CBF2F
:1046000001220022834208BF42F0010200F58060CF
:10461000834208BF42F0010212B9234A934202D1F9
:1046200021F0800199604C230121002203FB0787C0
:1046300087F88D1A87F88C2A04B0BDE8F0811B48F2
:1046400010405860ECE700214FF48053CDE9003171
:104650004C2303FB078393F88C2A012ACDE902112E
:1046600088D0D3F8500A022283F88D2A0B4A856835
:104670002A4082600E4A83F88C1A0121944283F802
:104680008D1A9AD00B4B9C427FF474AF95E700BF14
:1046900048190A0870250024000001408800CEFF58
:1046A0000008004000040040001800408FFF0FFF8A
:1046B00000040140000C0040201B00242DE9F04FB5
:1046C0000546086889B00C464FEA902CBDF8488032
:1046D000ACF5801C9DF84CA0BCF1520F69D8DFF8F6
:1046E000EC9019F80C700D2F63D807EBC706DFF8B4
:1046F000E0B0194607EB4606FFF7CEFE23680BEB4A
:1047000086066179A279BAF1000F55D194469B0AC9
:10471000A3F58013522B25D819F803000D2821D8B2
:1047200000EBC0030A4601A9CDF8088000EB430066
:104730004FEA4C034FEACC0C03F002030BEB800072
:1047400003930CF008034FF4807C049360230193DF
:104750004FF40073CDE906C30023059355F07AFAB0
:104760006179A2799307304629D54DF0DDFF154BCD
:104770004C2202FB073797F88D3A012B10D1022308
:10478000D7F8502A87F88D3A0F4B91680B40062BCB
:1047900006D0B3F5803F03D0136843F001031360E4
:1047A0002168637901F1340269600021D018286022
:1047B000D15009B0BDE8F08F82F0010CA7E74DF0B1
:1047C0009DFED4E7201B00240700010048190A08B9
:1047D0007025002470B504460068830AA3F5801391
:1047E000522B03D82B4DEE5C0D2E00D970BDFFF778
:1047F00053FE294B4C2202FB063696F88D3A012BCC
:1048000013D021680023254A254801E050F83320C1
:1048100091421CD00133112BF8D10121002056F018
:10482000B1F8204B01221A6070BD0223D6F8502A3D
:1048300086F88D3A1C4B91680B40062BE1D0B3F5FE
:10484000803FDED0136843F001031360D9E705EB26
:10485000C3030121134D93F80A4D204656F092F8F8
:1048600004F01F03012162091B2C01FA03F345F830
:10487000223006D1192056F085F84FF000732B60D6
:1048800070BD2E2CB2D12C2056F07CF84FF4805302
:104890006B6070BD48190A08201B0024000001400D
:1048A0004C260A0800E100E00700010070B5154C35
:1048B00082B094F88A3403F0FF05002BF9D1012669
:1048C00094F8703F84F88A640BB902B070BD0E4A48
:1048D000B4F88814138A14320C480191FEF710FFC3
:1048E0000199034618B184F88A5402B070BDD4F817
:1048F0003C4432460548636202B0BDE870405AF05D
:10490000A3B900BF201B0024A0F600245C1F0024D4
:1049100038B5264C94F8743F012B12D1042894BF6B
:10492000002301236BB904EB40000D4694F88C1F63
:10493000C4F8A03FB4F88E2FB0F8963FB4F8920FA9
:1049400001B138BD07EE902AD4F8842F9FED180AE4
:10495000B8EEE77ADFED177A27EE277A07EE902A8E
:104960006422F8EE676A02FB03F307EE903A02FB5B
:10497000003366EE806AB8EEE76A07EE903AF8EE2A
:10498000E77A27EE067A87EE270A20EE260A5CF001
:1049900067F8D4F87C2FB4F8903F1060D4F838133F
:1049A00019442944C4F8A41F38BD00BF201B0024AB
:1049B000CA269B3E0AD7233C2DE9F043BDB0BFF386
:1049C0005F8FA34A0020516A0346044621F48031D8
:1049D00051620146C2F89400C2F898300133C2F81F
:1049E0009C10112BC2F8A010F6D10523C2F8943008
:1049F000536A43F480335362BFF34F8FBFF36F8F1B
:104A00009448954A9549121A5CF0A8FD9448954A35
:104A10009549121A5CF0A2FD944AD368042B00F069
:104A2000FD8005D8012B00F08183022B00F07783F5
:104A3000874A00238E4C0120D2F888108D4E41F415
:104A400070018D4DC2F8881020602361216841F00B
:104A500080012160216801432160216841F4803197
:104A60002160216841F480512160A361E3612362E8
:104A7000A362E36223636363A363E3632364636406
:104A8000216821F4802121607C492366C1F8080156
:104A90004FF000614FF6FF00794B9160D168014003
:104AA0000B43D3604DF08AFAA36902460F20C3F38B
:104AB0000323A169334493F8883203F01F0322FAD9
:104AC00003F3C5F8D0334BF043FC6E4AD36813F0C0
:104AD000040FD36840F0A4806B4B0021694A039116
:104AE000D96A21F00101D962DB6A03F00103039363
:104AF000936943F440439361936903F44043039300
:104B0000039B93699B04FCD54C2200210DA85F4CAC
:104B10005CF098FD5E4A42F203031268B3EB124F59
:104B20004FF00003079304F1140318BF1C46E2681A
:104B3000002A4FD0544B5349D86A20F00100D86264
:104B4000DB6A03F0010307938B6923F440431343AB
:104B50008B618B6903F440430793079B494A936930
:104B60009F04FCD5424B4FF440314A484FF00108B6
:104B7000D3F8E020002742F08002C3F8E020D3F809
:104B8000E03003F080030693069B0323816108A9AC
:104B900008930B93CDE909874CF0CEFD02230DA8B5
:104BA000CDF834801E97CDE91633A3781893A388E7
:104BB0001993A3791A93E3791B93237A1C9323699E
:104BC0001D934FF480330E934CF03AFF03283BD0F3
:104BD00098B1FEE72B4A2C4B916941F44041916119
:104BE000926902F440420792DA6A42F00102DA6204
:104BF000DB6A03F001030793AFE7274B1A6812F053
:104C00000E0F4DD11A6822F00F0242F002021A6014
:104C10001B6803F00F03022B42D0FEE7D46007E7C6
:104C200023F007031D4C43F00203D360D4F824168D
:104C300006E0D4F824365B1AB3F57A7F3FF64CAF22
:104C400053689804F5D547E772B6FEF71BFA00BF24
:104C500000ED00E00000000050470000D03E0B08CF
:104C60000000002004000020BFAC0B08504000589A
:104C70000044025848190A0800000024008000512E
:104C80000003FA050048025800040058A803002455
:104C90000010005C001C025800200052201B002461
:104CA0006E4A936903F070033F2B05D8936923F094
:104CB000700343F040039361684AD36903F07003C3
:104CC0003F2B05D8D36923F0700343F04003D36131
:104CD000624AD36903F4E063B3F5806F05D2D36908
:104CE00023F4E06343F48063D3615C4A136A03F006
:104CF00070033F2B05D8136A23F0700343F0400381
:104D00001362564B9A69140705D49A6922F00F0270
:104D100042F008029A61514A936923F470639361E7
:104D2000136898017FF579AF136941F288304C4CD4
:104D300023F0070343F003031361D4F8241605E0BE
:104D4000D4F824365B1A834200F2A181136903F080
:104D50003803182BF4D1936903F00F03082B05D9FE
:104D6000936923F00F0343F0080393613D4A1368EE
:104D700003F00F03022B0BD9136823F00F0343F04A
:104D800002031360136803F00F03022B7FF445AF97
:104D9000324A936903F07003402B05D9936923F0DD
:104DA000700343F0400393612C4AD36903F070030E
:104DB000402B05D9D36923F0700343F04003D3613E
:104DC000264AD36903F4E063B3F5806F05D9D3694C
:104DD00023F4E06343F48063D361204A136A03F051
:104DE0007003402B00F24B811C4F4DF0E7F8034657
:104DF000D5F8D403BA69B969C2F30322164496F808
:104E0000882202F01F02D340C5F8D0334BF0A0FA3D
:104E1000002840F03D811023149016900DA80D93AA
:104E20004CF00EFE002840F029813B680E4943F00B
:104E300080033B60D7F8F43043F00203C7F8F43046
:104E4000D7F8F43003F002030293029B0A6A074B7F
:104E500042F001020A62D4F824160CE00044025821
:104E6000201B0024002000520004005800E204002F
:104E7000013B3FF4E9AED4F824269142F8D0D4F8AF
:104E80002426D4F824369B1A0A2BFAD94FF480230F
:104E9000B14C0DA84FF000080D934FF440130326BA
:104EA00002272E9357F0B0FBD4F8EC300DA843F056
:104EB0000203C4F8EC30D4F8EC3003F002030193A1
:104EC000019BD4F8943043F00203C4F89430D4F832
:104ED000943023F00203C4F89430A04B1A6841F2D6
:104EE0000303B3EB124F9E4B9E4A38BF1A469E4BAC
:104EF0005A601A6822F47C5242F400521A601A680E
:104F000042F060021A600D96CDE92A8857F07CFBCA
:104F10004FF4E0430DA8CDF8E0800D93CDE924884F
:104F200057F072FB18230DA8CDF8B4800D93CDF87F
:104F3000C88057F069FB4FF400230DA80D934FF480
:104F40000033359357F060FBD4F8E03008A9874868
:104F500043F00103C4F8E030D4F8E030CDF83080FD
:104F600003F001030593059B4FF48073CDE90A8696
:104F7000CDE908374CF0E0FB236908A97C4823F011
:104F8000FE7343F088732361D4F8E03043F00403E8
:104F9000C4F8E030D4F8E030099703F004030B962E
:104FA000CDF8288004934FF40073049A0893CDF849
:104FB00030804CF0C1FB236923F07E4343F0FC4377
:104FC00023614CF0FBFF6B4B6B4A4146C5F8D003A5
:104FD0001846D21A5CF036FB6848694A6949121AC9
:104FE0005CF0BCFABFF35F8F674D4646674C012704
:104FF0006B6A23F480336B62C5F8948023E0002A47
:1050000044D0D4F80080637A103414F8061C1B06D0
:1050100043EA017343EA420314F8052C43EA82434E
:1050200014F8042C43EA424314F8032CC5F89860A2
:10503000013643EA0243C5F89C80032E43F0010386
:10504000C5F8A03025D06368227A002BD7D0D4F8D9
:105050000080002AD7D128F01F09A3EB0903202BD9
:1050600038BF2023184699465CF072FA431E07FAAF
:1050700003F2914518BF0346DAB2C4E7FEE7136AAC
:1050800023F0700343F040031362ADE6FEE7C4E58E
:10509000C3E50523C5F894306B6A43F480336B6233
:1050A000BFF34F8FBFF36F8FBFF34F8FBFF36F8F80
:1050B0000022C5F85022BFF34F8FBFF36F8F6B698B
:1050C00043F400336B61BFF34F8FBFF36F8FC5F8AD
:1050D0008420BFF34F8FD5F8805043F6E0762A49FD
:1050E000C5F34E34C5F3C905640104EA06002B4636
:1050F00040EA8372013BC1F86022F9D2203C14F1EE
:10510000200FF2D1BFF34F8F4B6943F480334B61D3
:10511000BFF34F8FBFF36F8F3DB0BDE8F083042125
:105120000320FDF78DF972B6FDF7ACFF02200A4BA4
:105130001749D060D3F8F4200243C3F8F420D3F821
:10514000F43003400D930D9AD1F8003883F30888AA
:10515000D1F804389847FEE7004402580010005C7C
:105160007FBB22307FBB2200008400400000025839
:105170000008025820F60024A0F6002440F2002483
:1051800020F60024C3AC0B0800ED00E0D803002497
:105190000090F01F0548D0F8043323B1DB6A13B147
:1051A00000F5417018470248704700BF201B0024DB
:1051B000EC270A0810B5174CD4F8A83F1B883BB958
:1051C000002384F8B43F84F8FC32C4F8F83210BDF0
:1051D000D4F8AC2F002AF3DD012A08D0D4F8B03F70
:1051E00059880123A4F8B61F84F8B83FE8E7D4F83B
:1051F000B01F8A8849880132521A9A42F1D100229E
:10520000D4F8043304F541701B69C4F8302398477F
:10521000D6E700BF201B00240748D0F8003313B1A5
:1052200090F8B83F0BB100207047D0F8043300F578
:1052300041705B68184700BF201B0024174B10B457
:10524000174C93F8FC222244C0E9002493F8FC0296
:1052500093F8B42F824217D893F8FC02824206D307
:1052600000235DF8044B1846C1E90033704793F8FA
:10527000FC32002A5DF8044BC3F180030CBF01200F
:1052800002204A600B60704793F8FC420023012023
:10529000121B5DF8044BC1E900237047201B00245A
:1052A00020F600240F4B93F8FC2293F8B40F93F8E8
:1052B000FC22904293F8FC220FD8904204D3D3F8FA
:1052C000F83200201844704793F8FC22D3F8F832E3
:1052D000C2F18002104418447047801AD3F8F832A3
:1052E00018447047201B002410B51B4C84B01B4B86
:1052F00094F8FC220393134494F8B41F029394F897
:10530000FC32994294F8FC3214D899420AD294F8AB
:10531000FC320191C3F180030093C9B901223F2BF4
:105320000ED868B994F8FC02401AB0FA80F040092F
:1053300004B010BD0022CB1A019201220093EEE7C7
:105340006946002302A859F02DFC94F8B41FE9E740
:105350000B440222E3E700BF201B002420F60024B8
:105360002DE9F043164685B000293BD0451E284C58
:10537000DFF8A4804FF000096F180DE094F8FC32BC
:1053800008468B4294F8FC321CD9C3F180031844C0
:105390003F281AD8AF4225D094F8B40F15F8013F32
:1053A000411C08F80030C9B20B0684F8B41FE5D5DB
:1053B000002094F8FC3284F8B49F01468B4294F8A4
:1053C000FC32E2D8C01A3F28E4D994F8FC328B4270
:1053D000E0D0104B1B78002BDCD00020FFF784FFBF
:1053E000AF42D9D1694602A8FFF728FFDDE90032B4
:1053F00013443F2B00D910B905B0BDE8F083024635
:10540000334602A859F0CEFB05B0BDE8F08300BFDB
:10541000201B00240000002420F6002430B585B0B5
:10542000694602A8FFF70AFF58B9094C04F541750F
:10543000D4F8043328465B6898470028F8D005B0B4
:1054400030BD0246012302A859F0ACFBEDE700BFD6
:10545000201B002470B5114C16460A4682B0D4F8C1
:10546000003381190546994294F8B41F88BF1E1A6B
:1054700094F8FC32994203D00192FFF7CFFF019AD2
:10548000002033462946C4F83003D4F80403846A64
:105490000348A44602B0BDE870406047201B0024CA
:1054A000241E00248C461346014662461846D1E766
:1054B00038B5244C002204F6BC701346C4F800230F
:1054C00002461178063202292BD00133062BF8D17F
:1054D0000022D4F80433C4F8B02FF3B1DA6AE2B191
:1054E00019489047D4F8B03FC4F8A80FA3B1598821
:1054F0009A884368521A02FB0333C4F80033FAF760
:1055000077FF94F8FC32054694F8B42F9A4201D004
:10551000FFF784FFC4F8F85238BD0C4BC4F8A83F1D
:1055200038BD03EB4303D4F8042300EB4303C4F872
:10553000B03F12B1D26A002AD2D1044A1046C4F850
:10554000A82FD4E7201B0024241E0024EC270A08DF
:1055500010B50A4CD4F804335B6A13B104F54170FA
:105560009847D4F8F832D4F8A82F013B5288134456
:1055700052421340C4F8F83210BD00BF201B002473
:105580002DE9F043384E93B0FFF714FEFFF790FF7C
:1055900096F8FC3296F8B42F9A4201D0FFF73EFFFE
:1055A0000025D6F80073C6F8F85297B16C46DFF8BC
:1055B000BC802A4641462046203501F07DFE20462B
:1055C00059F01EFC012201462046FFF7C9FEAF42FA
:1055D000EFD896F8FC3296F8B42F9A4201D0FFF734
:1055E0001DFFD6F8A83F9B7B012B36D096F8FC32E6
:1055F00096F8B42F9A4201D0FFF710FF0020C6F8AA
:10560000F8026FB380466C46DFF86090054601E013
:10561000AF421CD92A46494609A801F04DFE212275
:10562000002120465CF00EF8202221462846FFF794
:1056300011FF2022064609A9204620355CF02FF9EB
:1056400008B9202EE4D0AF4208F10108E2D8B8FA38
:1056500088F0400913B0BDE8F083FFF779FFC5E794
:10566000012013B0BDE8F083201B00245CAB0A08C6
:10567000F0B583B04EF074FB214B292203F5805422
:10568000A3F82A27A3F83227D4F8982212B10022CF
:10569000C4F89822D4F8A02212B10022C4F8A022A3
:1056A000184E0027012506F5816283F8E07F84F813
:1056B0007C52C4F8942255F003FB06F224430DF10A
:1056C0000600ADF80670C4F89832D6F85034984702
:1056D0000D4BC4F8A00293F8CD31AB4202D028465E
:1056E00003B0F0BD06F25C46D4F8BC02C4F8B86260
:1056F00057F06AFC054B384683F82370F0E700BF8B
:10570000201B002400000024182C002400ED00E0E1
:105710000A4B93F87C0418B9094B93F8D0017047F1
:10572000084AD1680329F7D105494FF0010C81F8E7
:10573000D0C10021D16083F87C14704700000024A0
:10574000182C0024504000580321044608B5084690
:10575000FCF776FE72B6104BD3E9760350EA0302EB
:105760000AD1002211460420FCF76AFE11460520EA
:10577000FCF766FEFDF786FC084A21B24EF660246F
:10578000D2F8382304FB01F1121843F100038A1800
:1057900043EBE171E7E700BF182C0024201B002435
:1057A0000021032008B5FCF74BFE72B6FDF76AFC3A
:1057B000184CD4F8E02194F8E60108B54AB1116814
:1057C000938809690B40F8B9003B18BF0123002BEF
:1057D000F4D114200FF002FF00BFD4F8E03163B120
:1057E000196894F8E6219B8809690B4042B9003B8F
:1057F00018BF01230BB1FFF7D3FFFAF72BFEEBE73E
:10580000B3FA83F35B09F5E7B3FA83F35B09002B83
:10581000D4D1DEE7182C00242DE9F04F00218BB005
:1058200041F62C72AF485BF00DFF0420FCF702FE3E
:1058300001460520FCF7FEFD51EA000340F04381DC
:10584000A94B0393039BE422A849A648D3F8B0448C
:105850005BF084FEA34BC3E907445C621E461C67F1
:10586000C3F8B440C3F8B840C3F8BC40C3E91A4415
:1058700055F038F9FFF71CFE002108460AF05AFFE0
:10588000FAF7B6FDB0F1000940F38C810024984D81
:10589000984B06F1E4082746A24605F5F47B964EA0
:1058A0000294019304E00AF5006AD14540F3AC800C
:1058B000019AD2F83833C2F83C33FAF7CBFD2022F4
:1058C00059465046FFF7C6FD12228C4958465BF0F8
:1058D000E6FF0028E7D1574521D0029B5A1C03EB75
:1058E0004301874B029203EB8103864918460493D8
:1058F00001F0E2FC4246049B42F84C3BD8F81C30D5
:10590000C8F80C70AAEB0707C8E908330123C8F8E8
:1059100008307D4BC8E90477C8F828309046039BCF
:1059200057461222D3F8B034C8F81C30A918335D9A
:10593000013291F8E81199420BD00024202AF5D1C8
:1059400020375946B945384654DBFFF783FD00221E
:10595000ECE70134152CF1D1D0196C492022FFF766
:1059600079FD00230A2209A96848CDF824B001F086
:105970002DFE0746099800230A22013009A9099043
:1059800001F024FE0790002309980A2209A901309A
:10599000099001F01BFE0690002309980A2209A92C
:1059A0000130099001F012FE059009A90998002321
:1059B0000A220130099001F009FE049000230998A1
:1059C0000A2219460130099001F000FE97B1DDE985
:1059D000063243EA4211049B5A01059B42EAC32264
:1059E00042EA6003A7F2BC7241EA422243EA024360
:1059F000C8F81C30029B642B00F0F88057460AF56B
:105A0000006AD1453FF754AF029A642A00F0C5807E
:105A1000BA4500F0C2800C23394CAAEB070602F10C
:105A2000010A03FB024437495246374D204601F034
:105A300043FC029AC8F80040131DD8F81C20C8F88F
:105A40000C70CDF808A0C8F82850C8E90822012237
:105A5000C8E90466C8F808204C220021DFF8B480A9
:105A6000012702FB03F61F4B9C1920465BF0EAFD61
:105A70004C22002120465BF0E5FD1A4B039A43F8C7
:105A80000680029BD2F8B0240433A760A56262624C
:105A9000C4E90499C4E907224FEA4902B2F1805FE0
:105AA000C0F281800F4B9D6835B91A461B791BB136
:105AB0001368002B40F0A380002108460BB0BDE81E
:105AC000F04F0AF037BE4FF47A72002359F05CFEB3
:105AD0000F4B40F26D11022440F2B2720D46B0FB42
:105AE000F3F321E0783300240000002400280A08A2
:105AF000182C0024201B0024A0AB0A087CAB0A0849
:105B0000202E002490AB0A08A5540408002E00247F
:105B100080510100B8AB0A0801325B1A12F003048D
:105B20000CBF4FF4B77129469942F5DD8549002C29
:105B30005FD003910399D1F88014994200F39280C9
:105B4000814D01245B1A55F8041F01349942F9DD97
:105B50000133A2F2BC72039D43EA44133C2443EA9E
:105B600042237A4AB0FBF2F102FB11024FF461606A
:105B7000B2FBF0F100FB11221C20C5F88404B2FB3B
:105B8000F4F004FB1022521042EA401242EAC12211
:105B900042EA0343C5F8B03454E6029AD31C32BB40
:105BA000032379E703234C220021DFF8B481012687
:105BB00002FB03F4664B02271D1928465BF042FDE9
:105BC0004C22002128465BF03DFD614B039A43F8CF
:105BD0000480C9F10063D2F8B024B3406F71AE60A5
:105BE0006A62C5E90722C5E904335BE76723594DBB
:105BF00032E70C4603911D21C4F884149AE7294624
:105C00002E461564D563C2E91155D46C02F14C03DC
:105C100054B39C68481E1E648442DE63C3E9116667
:105C200012D0481C844216D08C427FF445AF0846FF
:105C300000283FF441AF116CCC6B0134CC63196484
:105C4000936401461A46E0E700293FF435AF8842E5
:105C500053F80C2CECD1117900293FF42DAF53648B
:105C60001A64EEE7012473E739490222264611E05F
:105C7000CB6B0A635B01C1E9046657D003F6FF777B
:105C8000531E03EB17335A1C0135C1E90D3351F88C
:105C90004C0FC8B10B79002BEAD108690A630028C0
:105CA00048D1531E10464F694863002F40D007F675
:105CB000FF7703EB1733201A8B635A1C0135C41886
:105CC00051F84C0F0028E5D123483E22013BC0F893
:105CD00080433F24C0F868234022990F0190C0F808
:105CE0008C53C0F87C33C0E9DB421C4AC0F8642303
:105CF0009A002BB340F2FF10121841F10001520A32
:105D000042EAC15202F140010198114C0A44C0F824
:105D1000741302EBC303C0F878235902C0F8603350
:105D2000DA0DC0E9E144C0E9D612C5E61346AAE798
:105D30001346C0E700F6FF70531E03EB1030B2E7C6
:105D40000122DFE7000000248004002480510100CC
:105D500078330024A5540408201B0024D4AB0A087F
:105D6000C8AB0A0843F2010C43F2011101220023DF
:105D7000A0F800C04FF6057CC18006210273827036
:105D80000272C38103824382A0F814C081757047F8
:105D9000FF22034600F11E01F0B5DA70053303F867
:105DA000012C8B42F9D1124B4FF0FF3C47261625B0
:105DB00003F11E0764464FF0150E00220AE093F926
:105DC0000620063393F801E09D78DE7893F90440CD
:105DD00093F905C002EB82029F4200EB020100F83A
:105DE00002E04D708E70CC7081F804C0E7D1F0BD38
:105DF0002C330A084FF0000C01210222032380F803
:105E000005C08171C2710372704700BF0023022276
:105E1000037043708370C3700271704740F22E4C60
:105E20004FF4F07100230722A0F81EC04FF4FA6C63
:105E300001804FF47A714371A0F820C040F2262C03
:105E400041844FF4F5618371438240F20123A0F84D
:105E50001CC041F2101C818441F21231838240F255
:105E60000343A0F808C04FF00E0C41810221C38209
:105E700040F20563827080F826C041748276038305
:105E8000704700BF8388C3F30B039342A8BF134638
:105E900070B51D460C461A46064680685BF05EFBF0
:105EA0006219084B9442B56908D0074814F8011BE1
:105EB00000FB03F3A24283EA0103F7D101202B6028
:105EC00070BD00BFC59D1C819301000100230370BC
:105ED00043708370C37070470023037043708370F6
:105EE000C3707047002201234FF04D0C8121427096
:105EF00080F800C08270C270017143718371C371F8
:105F0000704700BFFF232822437002708370C37064
:105F1000704700BF002306214FF47A7201700373AB
:105F2000C0E90123704700BF00230372704700BF20
:105F300037230370704700BF0023FF22411C10B5B8
:105F400000F8132001F8132001330B2BF8D10C4B70
:105F50004FF0FF31002203F11B048C4605E013F9DA
:105F600002CC13F9011C13F8032C033300EB420E8F
:105F700000F812C09C428EF80110F0D110BD00BF95
:105F800053330A0802224FF0100C0123FF21427004
:105F900080F800C04FF0000C0271C2710272827270
:105FA000032280F802C04FF0110CC272372280F831
:105FB00003C04FF0120C02734C2280F806C04FF061
:105FC000130CC273552280F809C04FF0040C827480
:105FD0001F22437143738173037480F811C0C3742B
:105FE000017583754275C175704700BF4FF0FF336F
:105FF0000722436003608360C360037402717047CB
:1060000003230370704700BF002303704370C37005
:1060100083700371704700BF704700BFDFED277AC0
:10602000B4EEE70AF1EE10FA0CDDDFED256A9FED24
:10603000257AF0EE407A30EE660AF4EEC77AF1EE99
:1060400010FAF6DCDFED207AB4EEE70AF1EE10FA92
:106050000CD5DFED1B6A9FED1D7AF0EE407A30EE35
:10606000260AF4EEC77AF1EE10FAF6D4DFED187ACC
:10607000B4EEE70AF1EE10FA14DDDFED107A37EE38
:10608000C00A60EE006A9FED136A9FED137ADFEDA0
:10609000137AA6EE867A20EE266AE6EE877AA6EED8
:1060A000270A7047DFED0E7AB4EEE70AF1EE10FA38
:1060B000E7D5DFED057A37EEC00AE2E7DB0F4940AE
:1060C000DB0FC940E4CB1641DB0F49C0E4CB16C15E
:1060D000DB0FC93F92E741B99730083C15A82ABEAB
:1060E000DB0FC9BF2DE9F047089F002B0E46054680
:1060F0003C4614BF4FF030094FF0200914F8011B43
:1061000041B3002A2CDD234600E0B2B113F8010BA5
:106110009046013A0028F8D1A8F102086AB1C246B7
:1061200049462846B04753460AF1FF3A002BF7DCB0
:1061300028EAE8723978013249B1D71B2846B047BE
:10614000E01914F8011B0029F8D1BDE8F0871046CA
:10615000BDE8F087002A02F1FF38E0DC0846F4E7EA
:106160000022EAE703685A1C02601970704700BFFA
:10617000024B186803681B68184700BFA852002428
:10618000884230B54FF001043AD301FB04F4B0FB70
:10619000F4FC8C45F9D2BCB102BB06E0A14203F885
:1061A000015B11D81446B0FBF2FCBCF1090F0CF1F5
:1061B00057050CF1300E04FB1C00B4FBF1F2EDDCD2
:1061C000A14203F801EBEDD900221A7030BDA142C3
:1061D00003F8015BF8D81446B0FBF2FCBCF1090FE0
:1061E0000CF137050CF1300E04FB1C00B4FBF1F28E
:1061F000EDDCA14203F801EBEDD900221A7030BDAD
:106200008446002AEAD1D0E7002870B503DA2D23AE
:10621000404201F8013B092886464FF0010307DDA3
:1062200003EB83035B00B0FBF3F2092AF8D8A3B1B8
:106230000F4CA4FB0320BEFBF3FCBCF1090F4FEA9B
:10624000D0000CF130060CF1570503FB1CEE07D80B
:10625000092B01F8016B0346EBD800230B7070BDCE
:10626000092B01F8015B0346E3D800230B7070BDD6
:10627000CDCCCCCC0378092B01D0202B05D110F844
:10628000013F202BFBD0092BF9D02D2B00F0A9804A
:106290002B2B75D0B7EE000AA3F13002D1B2092939
:1062A00077D8F2EE046ADFED5F7A07EE102A10F875
:1062B000013FB8EEC77AA3F13002D1B2A7EEA67AB9
:1062C0000929F0EE477AF0D92E2B66D003F0DF03D0
:1062D000452B40F0838010B442782D2A00F0968040
:1062E0002B2A00F08380A2F130030130092B00F249
:1062F00084800024002303EB830302EB430310F8A4
:10630000012FA2F13001303B0929F4D9B3F59A7F6E
:106310001A46B7EE007A28BF4FF49A72072B09D9B4
:106320001346DFED416A083B27EE267A072BFAD8A1
:1063300002F00702DAB1F2EE046A012A27EE267AA9
:1063400015D0022A27EE267A11D0032A27EE267AC4
:106350000DD0042A27EE267A09D0053A27EE267AB0
:1063600005D027EE267A012A18BF27EE267A002CC0
:1063700045D0C7EE877A5DF8044B20EE270A7047B8
:106380004378B7EE000A0130A3F13002D1B20929F7
:1063900087D92E2BDFED237A98D143780130A3F1F2
:1063A0003002D1B2092991D8B2EE047AF0EE475A00
:1063B00006EE902A10F8013FB8EEE66AA3F130022B
:1063C000D1B2C6EE076A092927EE257A77EEA67ABA
:1063D000EED903F0DF03452B3FF47DAF20EE270A13
:1063E00070474378BFEE000A013055E782780230EB
:1063F000A2F13003092B7FF67CAFB7EE007A67EE8F
:10640000877A5DF8044B20EE270A704782780230C5
:10641000A2F13003092B01D801246BE7B7EE007A13
:10642000A7E700BF0000000020BCBE4CF0B5067915
:1064300006F0E003402B03D145794FF0FF3406E02E
:10644000602B4FF00105F8D1447905FA04F40023DC
:10645000012006F00706AB4200D1F0BD052E0FD893
:10646000DFE806F00308101D242448B1C85CD75C9F
:1064700078400FE020B1C856D756C71B7842784104
:106480000133E8E70028FBD031F8130032F813702D
:10649000784080B220420CBF01200020F0E70028A5
:1064A000EED031F9130032F91370E6E70028E7D097
:1064B00051F8230052F82370DAE7037903F0180348
:1064C000102B1DD004D82BB1082B06D0002070470C
:1064D000182BFBD1B0F80B007047114BB0F80B0034
:1064E00093F90030591C09D10E4B1B7903EB830241
:1064F00003EBC20300EB830080B27047DBB2F5E729
:10650000074BB0F80B0093F901305A1C06D1054B2C
:106510005B79C3EB031300EB4300EDE7DBB2F8E775
:10652000B4040024A85200240022104B30B5944635
:106530004FF4487403F1120596460260828002EB24
:106540004202AB4200EB420100F812E081F801C0C8
:10655000DA788C808A7008D093F90620063393F895
:1065600001E093F802C09C88E9E730BD6C330A086B
:10657000092917D0B1FA81F35B0999B10139036098
:106580004B0001F0030103F00802C1EB011193007D
:10659000C1EB0111A3EB92038900C3EB03138180CC
:1065A0009B004380704700BF442203230270437066
:1065B000704700BF43F6017200234FF4007C4FF494
:1065C000917142800122A0F800C0C1800381438103
:1065D0008381C281704700BF4FF0010C2C21022241
:1065E000002380F800C041708270C370704700BF04
:1065F000144B1522144910B5044618681B79206203
:1066000004F1250084F824305BF05DF90F4B4FF066
:10661000010E1A7D84F83AE012B984F83B2010BDCF
:1066200003F1180CBCE80F0020606160A260E36019
:10663000BCE80F0084F83BE020616161A261E36186
:1066400010BD00BF60AC0A0868AC0A08A85200245C
:1066500010B50021382204465AF0F4FF0C4A0921F3
:106660000C480123226141F61E6C0B4A21720B4932
:10667000A373E161214684F82130A4F826C0C4E95F
:106680000502074A0748A262BDE810402FF05CBA35
:106690006400DC051A046C070019750343080E003A
:1066A0001E7D010178AC0A08B5EEC00ADFED357A2F
:1066B0000023F1EE10FA70B5C8BF30EE270A86B09D
:1066C000D8BF30EE670ADFED307A054603A90293A2
:1066D0006E4620EE270ACDE90033FDEEC07A17EEB4
:1066E000904A84EAE470A0EBE4704FF07BFD002C4C
:1066F00003A8ACBF20232D238DF8003058F080FB79
:10670000012829D0022833D003281DD003A9304600
:106710005BF090F8304658F073FB0446314628464B
:10672000033CE4B222465AF019FF002328462B55B9
:1067300058F066FB2E22431C31192A54E8185BF0EE
:1067400095F8284606B070BD302303A930468DF871
:1067500001305BF06FF8DDE743F23002302303A92C
:106760003046ADF801208DF803305BF063F8D1E7D7
:1067700043F2300303A93046ADF801305BF05AF81C
:10678000C8E700BF6F12033A00007A4409F012BA5A
:1067900013B568B14C1E14F8011F21B902B0BDE851
:1067A000104009F01BBA019009F004FA0198F2E7D1
:1067B00002B010BD202108B55BF04BF8034618B1BC
:1067C0001A780130202AF9D0184608BDF8B5E8B18A
:1067D0000138114ACB43C60002EBC00003F00103AD
:1067E00090F83C5090F83D7083EA0504A7420DD024
:1067F000806B40B10768AB420CBF10230023808838
:1068000000FA03F3BB61324482F83D40CB0701D468
:10681000FCF78CFCF8BD00BFA85200242DE9F34121
:106820000023124D044600EB8106114F05F8583F36
:10683000B44203D10F4802B0BDE8F0813946284682
:106840004FF000085AF0F6FF214668465BF00EF85C
:10685000202168465AF0FDFF28B9694628460434CD
:106860005AF0E8FFE4E780F80080F1E7A85200243E
:106870001FFE0A0800530024014BD86F3CF042BEB3
:10688000A8520024704700BF084B024608498B42BB
:106890000AD2184602E01C30884205D20388C3F3AE
:1068A0000B039A42F7D170470020704728860B08E7
:1068B000908F0B0870B50546B0F80900FFF7E4FFAC
:1068C000064B0446284693F88060FFF7F6FD16B1A4
:1068D000E368184470BDA368FBE700BFA85200241A
:1068E00038B505460C46FFF7E5FF2B7903F0E002CB
:1068F00003F00703602A2AD1052B0CD8DFE803F048
:10690000030B0F0B1B1B6A79012393400278DBB248
:1069100014B11343037038BD22EA0303FAE76A791E
:106920000123934002889BB214B113430380F2E722
:1069300022EA0303FAE701236A7903FA02F2036801
:1069400014B113430360E6E723EA0203FAE7052BD9
:10695000E1D8DFE803F00303050507070470DAE771
:106960000480D8E70460D6E770B585880B460446F6
:106970000021C5F30B0518462A465AF063FE6169EB
:10698000084A0346914202D3074A914205D319B1FE
:106990001846BDE87040084770BD2A46BDE8704003
:1069A0005AF0DCBD908F0B08A3910B0838B5064C4C
:1069B000064DAC4206D2A16820461C34FFF7D4FF36
:1069C000AC42F8D338BD00BF28860B08908F0B0867
:1069D0000A4491421AD001F1FF3C41F2210100B575
:1069E00002F1FF3E1CF8012F082380EA022010F478
:1069F000004F4FEA400281EA40000CBF90B280B2E3
:106A0000013BF4D1E645EDD15DF804FB7047F8B5E4
:106A1000164D6B78BE2B26D1AC1C154F0222294691
:106A20004FF6FF70FFF7D4FF22884AB1A618BE4286
:106A300019D2052A17D921463446FFF7C9FFF3E7D3
:106A400021460222FFF7C4FF0222A1180634FFF7F5
:106A5000BFFF084B641BA3F8824041F60F53C31AD3
:106A600058425841F8BD0020FCE700BF0000020872
:106A700000000408A85200240823484010F0800FAA
:106A80004FEA400182EA40000CBFC8B2C0B2013BED
:106A9000F4D1704730B505688D421AD901F1FF3E37
:106AA0006C1E00231EF801CF082183EA0C0313F0AB
:106AB000800F4FEA430C82EA43030CBF5FFA8CF36A
:106AC000DBB20139F3D17445ECD16A1C02602B7042
:106AD00030BD00236A1C02602B7030BD9FED067A2A
:106AE000F7EE007A60EE870A20EE800A70EE277AD1
:106AF00080EE270A704700BFDB0FC94007EE101A6F
:106B0000DFED7E7AB8EE477A27EE000A60EE277A4C
:106B1000BDEEE77A17EE103A2033402B00F2DC800E
:106B20009FED777AB4EEC70AB0EE677AF1EE10FA0D
:106B30000CDDDFED745A9FED746AF0EE476A37EEB4
:106B4000657AF4EEC66AF1EE10FAF6DCDFED6F6AF4
:106B5000B4EEE67AF1EE10FA0CD5DFED6A5A9FED4D
:106B60006C6AF0EE476A37EE257AF4EEC66AF1EE0B
:106B700010FAF6D4DFED676AB4EEE67AF1EE10FAB9
:106B800040F39680DFED646A36EEC77A27EE075A47
:106B90009FED624A9FED626AF7EE005ADFED616A8F
:106BA000A5EE046ADFED604A27EE054AE5EE066AC7
:106BB000A4EE267AF0EE656AE7EE245AE7EE646A00
:106BC00086EEA54A9FED537A77EE877ABDEEE77A97
:106BD00017EE103A2033402B77D89FED547AB4EE5D
:106BE000C70AF1EE10FA0CDD9FED466ADFED466A4A
:106BF000B0EE677A77EEC67AB4EEE67AF1EE10FA86
:106C0000F6DC9FED427AF4EEC77AF1EE10FA0CD57D
:106C10009FED3C6ADFED3E6AB0EE677A77EE867AEA
:106C2000B4EEE67AF1EE10FAF6D49FED3A7AF4EE8D
:106C3000C77AF1EE10FA54DD9FED377A77EE677A76
:106C400067EEA74ADFED353A9FED355AB7EE006A99
:106C5000DFED346AB6EE007AA4EEA35A27EEA43A2A
:106C6000F8EE003AE4EE856AE3EE267A36EE676ADD
:106C700067EEA37A26EE077AB7EE005A002380ED7E
:106C8000044A8361C5EE256A436180ED095A0362B7
:106C9000C36126EE877A26EE866A66EEA77A80EDD5
:106CA000007A80ED016A80ED027AC0ED037A7047C8
:106CB000DFED1F6AB4EEE67AF1EE10FA7FF566AF0B
:106CC000DFED126A36EEC77A60E7B6EE007ADFEDE6
:106CD000197AB7EE006ACFE7B7EE004AF0EE445AF1
:106CE00070E79FED137AF4EEC77AF1EE10FAA7D5AC
:106CF0009FED067A77EE677AA2E700BF27D4D236F7
:106D00000024F448DB0FC940E4CB1641DB0F49C037
:106D1000E4CB16C1DB0FC93FDB0F494092E741B915
:106D20009730083C15A82ABEF304353F0024744868
:106D3000DB0FC9BF000000009FED2E7A70EE077ACE
:106D4000FDEEE76A16EE903A2033402B4FD8B4EEB2
:106D5000C70AF1EE10FA0CDD9FED276ADFED276A16
:106D6000B0EE677A77EEC67AB4EEE67AF1EE10FA14
:106D7000F6DC9FED237AF4EEC77AF1EE10FA0CD52B
:106D80009FED1D6ADFED1F6AB0EE677A77EE867AB7
:106D9000B4EEE67AF1EE10FAF6D49FED167AF4EE40
:106DA000C77AF1EE10FA16DD9FED177A77EE677A63
:106DB00027EEA76ADFED155ADFED156A9FED157A0C
:106DC000E6EE256A67EE865AA6EE267AE5EE877A23
:106DD000B0EE670A70479FED107AF4EEC77AF1EED5
:106DE00010FAE5D59FED067A77EE677AE0E79FED3A
:106DF0000B0A7047DB0FC93FDB0FC940E4CB1641DC
:106E0000DB0F49C0E4CB16C1DB0F494092E741B923
:106E10009730083C15A82ABEDB0FC9BF0000000050
:106E2000B0EEC07AF0EEE06A86FE876AB5EE406AA0
:106E3000F1EE10FA3DD0C6FEC75AC5EE867ADFEDF8
:106E40001E2ADFED1E3ADFED1E4A9FED1E5A9FED12
:106E50001E3AB7EE006A9FED1D4ADFED1D5AE7EEC0
:106E6000E23AA7EE834AE7EEA34AA7EE846AA7EECA
:106E7000A45AE7EE855AC5EE867AF4EEC76AF1EEBB
:106E800010FA03D59FED137A77EE677AF5EEC00A14
:106E9000F1EE10FA03D59FED107A77EE677AB5EE32
:106EA000C00AF1EE10FA48BFF1EE677AB0EE670A59
:106EB0007047DFED077AE0E739094E3DE3B59E3EC6
:106EC00088FA163E45FE7F3F99FB243F69A2163E95
:106ED000A7DFA834DB0FC93FDB0F49409FED4D0A08
:106EE00090ED005A35EE000A08B5FDEEC07A17EEB7
:106EF000903A2033402B7BD8FFF790F8F0EE403AE1
:106F0000FDEEC57A17EE903A2033402B7FD8B0EED5
:106F1000450AFFF783F8B0EE405AD0ED014A9FEDE5
:106F20003D0A34EE800AFDEEC07A17EE903A203327
:106F3000402B69D8FFF772F8F0EE405AFDEEE47A84
:106F400017EE903A2033402B5BD8B0EE640AFFF77F
:106F500065F8F0EE404A90ED023A9FED2E0A33EECE
:106F6000000AFDEEC07A17EE903A2033402B45D848
:106F7000FFF754F8B0EE404AFDEEC37A17EE903AB0
:106F80002033402B37D8B0EE430AFFF747F8F0EE36
:106F9000407A27EEA36AC1ED024A24EE233A24EE9A
:106FA000057A67EE856A24EE254A65EEE77A25EED6
:106FB000655AF0EE462A81ED004A65EEA35AC1ED0E
:106FC000017AF0EE433A81ED055AE7EE242AA6EE67
:106FD000247AC1ED085AE6EEE43AE3EE646AC1EDC4
:106FE000032A81ED077AC1ED043AC1ED066A08BDB6
:106FF000DFED093A84E7DFED087ACAE79FED064A3C
:10700000BAE7DFED054AA6E7DFED035A96E79FED05
:10701000025A82E7DB0FC93F000000002DE9F04370
:107020001D4689B0531C0F4603931178002900F0C8
:107030000D8100240646A04608E030460134B847DA
:10704000039A531C0393117800293CD02529F4D1CD
:10705000931CCDE903385078302800F08980A0F1E6
:1070600030034FF00009DBB2092B40F28C806C2812
:107070002DD0782800F29180572817D9A0F1580315
:10708000202B00F28A80DFE803F0BB88888888889C
:10709000888888888896B588888888888888888835
:1070A0009E888888888A88A38888BB0058B125284C
:1070B00073D125213046B847039A0134531C0393FA
:1070C00011780029C2D1204609B0BDE8F083039BA6
:1070D0005A1C03921B78782BB3D8572B58D9A3F19D
:1070E00058012029ADD801A050F821F019720408E8
:1070F0004370040843700408437004084370040894
:107100004370040843700408437004084370040883
:107110004370040843700408B771040841720408FE
:107120004370040843700408437004084370040863
:107130004370040843700408437004084370040853
:1071400043700408C97104084370040843700408BC
:1071500043700408437004089F71040843700408D6
:10716000317204084370040843700408197204085B
:10717000D31C4FF0010903939078A0F13003DBB2E8
:10718000092B3FF674AF04AA03A951F047FE6EE73E
:10719000002B98D0252B8CD053E7039A51E755F854
:1071A000040B0023049A394600903046FEF79AFFFC
:1071B000039A044445E755F8041B30460134C9B22C
:1071C000B847039A3DE7039A55F8043B1C6038E73B
:1071D00005AB00220A2155F8040BFEF7D1FF05AAE2
:1071E0004B46394630460092049AFEF77BFF039ADD
:1071F000044426E705A955F8040BFFF705F8EEE768
:10720000A0F1580205AB102155F8040BB2FA82F236
:107210005209FEF7B5FFE2E7A3F15802102105ABD2
:1072200055F8040BB2FA82F25209FEF7A9FFD6E72D
:1072300005AB00220A2155F8040BFEF7A1FFCEE7AB
:1072400005A955F8040BFEF7DFFFC8E70C463AE73F
:1072500073B5144C06460D460192D4F88400C0B1B3
:107260001149FFF795FA3146D4F88400FFF790FAF8
:107270000E49D4F88400FFF78BFA0D49019B2A468A
:10728000D4F88400FFF7CAFE0A49D4F88400FFF757
:107290007FFA94F8883013B1012384F8893002B062
:1072A00070BD00BFA8520024B0EE0A08ADF20A0873
:1072B0008D670408BDEE0A080EB400B584B0084915
:1072C00005AB019001A853F8042B0393FFF7A6FE2A
:1072D000019B00221A7004B05DF804EB03B0704704
:1072E0006561040800232DE9F0411C4682B0074681
:1072F000038021460134384636F026F9082CF8D1AF
:10730000002307F1FC06DFF8608087F8EA301D46AD
:10731000C7F8EC30C7F8F030C7F8F430C7F8F830E9
:107320001F462A46414601A83446FFF7C5FF0322FF
:1073300001A911F8013B5BB1013A04F8013BF8D116
:10734000013504362770082DEBD102B0BDE8F0817D
:1073500001352046202114445AF074F9082D06F115
:1073600004062770DDD1F0E784AC0A08F7B5114EAA
:10737000074600230C46304615460F498A3600F86A
:107380008A3F04EB45050D4B002F08BF19460C4FF3
:107390005AF050FAAC4202D10A4803B0F0BD394667
:1073A00034F8022B6846FFF787FF694630465AF0EB
:1073B00041FAEFE7A8520024C1EE0A08CAEE0A0813
:1073C000D3EE0A0832530024F7B500230B4E0446CF
:1073D00000EB41050A4F06F8BB3FAC4202D1094819
:1073E00003B0F0BD394634F8022B6846FFF764FF5E
:1073F000694630465AF01EFAEFE700BFA852002453
:10740000333B0B0863530024F8B54E1E054601F1CB
:107410001F04054F16F8012F284639460235FFF79D
:107420004BFFA642F6D1F8BDD8EE0A0803685A1CF5
:1074300002601970090A03685A1C026019707047CB
:1074400002681146531C0360D31C11F802CB016083
:107450005178036093781B0443EA0123111D43EA2A
:107460000C030160D07843EA00607047A0F130035C
:10747000092B07D920F02000413819288CBF0020A3
:107480000120704701207047303809288CBF002048
:1074900001207047413819288CBF00200120704717
:1074A000613819288CBF00200120704720280BD09C
:1074B000092809D00A2807D00D2805D00B38012843
:1074C0008CBF00200120704701207047A0F14103CC
:1074D000192B98BF20307047A0F16103192B98BF7A
:1074E0002038704710B56FF000440246044404E0B1
:1074F000B3EB0E0015D1A24214D012F8013BA3F158
:107500004100192811F8010BA0F1410C98BF20335C
:1075100000F1200EBCF1190FEAD91B1A04D1002882
:10752000E9D110BD002010BD184610BD02B384463D
:1075300010B5841804E0B3EB0E0014D1A44513D0A9
:107540001CF8013B11F8010BA3F1410200F1200EE0
:10755000192AA0F1410298BF2033192AEBD91B1A2E
:1075600004D10028EAD110BD002010BD184610BD7E
:107570001046704770B5044608460D4657F040FC6B
:10758000064602E014F8013F43B120463246294640
:10759000FFF7CCFF0028F5D1204670BD1C462046E1
:1075A00070BD38B507490546FFF7E4FF041E0649DC
:1075B000284618BF0124FFF7DDFF08B144F002049C
:1075C000204638BDDDEE0A0805050B082DE9F0411F
:1075D000064686469EF800C070460EF1010EBCF1CC
:1075E000200FF7D0BCF1090FF4D0BCF10A0FACF1B9
:1075F0000B05EFD0ACF10D04B4FA84F46409002C4F
:10760000E8D1012DE6D9BCF12B0F3DD0BCF12D0FF7
:1076100039D0102A86463DD04FF0FF359046B5FB55
:10762000F2F502FB05F7FF43FFB20EF1010E002059
:1076300010E0ACF1300C5FFA8CFC944512DA854214
:10764000764602D334D1674532D21C404FF0FF302A
:107650001EF801CBBCF1390FEBD94CF0200CBCF17A
:10766000600F0BD801B10E602CB3B0F1004F2BD9D5
:10767000DB0729D54FF00040BDE8F081ACF1570C95
:107680005FFA8CFCD9E70124102A00F1010E90F872
:1076900001C0C1D1BCF1300F19D04FF0FF354FF010
:1076A0001008B5FBF2F502FB05F7FF43FFB2BCE79C
:1076B00008FB00C0CCE70028DEDA13F0010F18BF8A
:1076C0006FF00040BDE8F0814042BDE8F0819EF8D7
:1076D00001C00EF10106ACF141056046192D01D83B
:1076E0000CF1200078280BD04FF0FF354FF0100838
:1076F000B646B5FBF2F502FB05F7FF43FFB294E790
:1077000010229EF802C06FF070450EF1020E0F2796
:1077100090468AE701230A22002157E770B50D46FB
:107720001446FFF747F80646A0B1FFF7F3FF40F60F
:1077300034039842A8BF1846B0F5617FB8BF4FF434
:107740006170A0F561731920B3FBF0F32B702378FF
:10775000013323703046FFF72DF80646A0B1FFF73E
:10776000D9FF40F634039842A8BF1846B0F5617FB0
:10777000B8BF4FF46170A0F561731920B3FBF0F34B
:107780006B70237801332370304670BD2DE9F041D2
:1077900017461E4605464FF47A7200233846314696
:1077A000454C57F0F1FF4549454A0144454882FBA5
:1077B00001C34FEAE17C0B44CCEB631382FB03C2B1
:1077C0004FEAE37C1A44CCEB621284FB02C44FEA1A
:1077D000E27CCCEBA40C80FB0C404FEAEC74C4EBD5
:1077E000E010C3EB0314A1EB8401A971C2EB0211F9
:1077F000A3EB81036B710CEB4C03A2EBC30240F2D1
:10780000B55303FB10CC80002A71BCF5896F45DAB3
:1078100040F2DA239C4548DCBCF5B77F2A4BB4BF65
:107820000022012202EB42014FEA420803EBC103AE
:1078300091B2B3F86E3008EB020E244C04EBCE0488
:107840004FF00B0E163401E034F8023D634520DDA5
:10785000BEF1010EF8D11C4B42444FF0010E03EB78
:10786000C202B2F8583000F5FA600CF1010C4FF486
:107870007A7285F802E00844ACEB030C3146002331
:107880002880384685F803C057F07EFF2A81BDE87E
:10789000F0810EF1010E5FFA8EFEE4E7032140F263
:1078A00096534FF006080A46C5E7022140F22943E5
:1078B0004FF004080A46BEE7ABAAAA2A80BC92C7CA
:1078C0008988888873B06D162C330A0884330A08B7
:1078D00008B50D4BD3E9002352EA030C0AD1014647
:1078E000002340F2011218460B804A808B808B7176
:1078F0000B8108BD054909688A1843F10003FFF7A9
:1079000045FF012008BD00BFF02D0024581E0024B3
:1079100090420B462DE9F041B0FBF2F604461546C5
:1079200008D2124A05FB16441846135D00F8013BC5
:10793000BDE8F0819642B6FBF2F706D20B4A05FB92
:107940001767D15D03F8011BECE7BA42B7FBF2F809
:1079500007D905FB1878054A12F8081003F8011B2F
:10796000EDE74046FFF7D4FF0346F2E78CAC0A0888
:1079700030B5684C83B0B4F8F033B3F57A7F03D9EF
:107980004FF47A73A4F8F033B4F8F233B3F57A7F96
:1079900003D94FF47A73A4F8F233B4F8F403B0F5D2
:1079A0007A7F04D94FF47A731846A4F8F433B4F804
:1079B000F613B1F57A7F03D900231946A4F8F633FC
:1079C000B4F8F823B2F57A7F04D94FF47A731A46E3
:1079D000A4F8F833B4F8FA33B3F57A7F02D9002368
:1079E000A4F8FA33884202D80021A4F8F413934291
:1079F00002D30023A4F8F833B4F80624B4F808340A
:107A00009A4202D90023A4F80634434B1B8803B3DF
:107A1000424DAA78062A43D8414901EB820191EDF3
:107A20002E0A2979002940D194F8101407EE903AD3
:107A3000AB7907EE101AF8EEE77AF8EEC76A86EE31
:107A4000A77A0BB130EE000AB4EEC70AF1EE10FAD5
:107A500030DC6379032B14D8C3EB0313314A02EBF8
:107A600043022379032BC4F8182412D803EB8301B3
:107A70002D4A03EBC10302EB8303C4F81C3403B0AB
:107A800030BD0023274A63712379C4F81824032BDF
:107A9000ECD90022244B2271C4F81C3403B030BD51
:107AA00029799FED220A0029BED0042A21D8002A74
:107AB000CFD021E067EE807ABCEEE77A8DED017AD7
:107AC0009DF8042007EE102AB8EEC77AF4EEC77AC4
:107AD000F1EE10FA01DD0132D2B2CAB1102AA8BF0C
:107AE0001022D2B28A42134638BF0B4684F81034B3
:107AF000AFE7053A032AACD9F7EE007A87EE800AA1
:107B000058F0AEFF2B88984228BF18462880A0E77F
:107B10000122E6E7A8520024241D0020E4290024C5
:107B20002C330A088C530024045400246F120338A9
:107B30002DE9F04FAA4E85B096F8203400AFA3F19E
:107B40001702022A00F2BB82A64BBB60DFF8B4A288
:107B50004FF0000896F838140AF190095446DFF8FF
:107B6000A8B2A14D34E010F0010C4ED1142A00F05F
:107B7000A2824308820803F0773302F033321344C1
:107B8000C208C31A02F011329B1A03EB131303F05D
:107B90000F33ABFB03E2D209C2EB02229A1A830332
:107BA00002D5012A00F08782012A0ED9082A00F2A4
:107BB0008282BCF1000F01D0284206D1F96056F054
:107BC000EBFBF968002800F076820C344C4521D09C
:107BD00094F904202068A2F11E03DBB2012BC2D865
:107BE000A27920F04100E3794FF0000C022A2060D6
:107BF000A8BF0222022BA8BF0223A271E371237A3D
:107C0000022BA8BF02232372B3E708F101085FFA31
:107C100088F8AEE708F1FF38B8F1020F00F24B82A6
:107C20000024022086F8FC4415F058F896F8003538
:107C3000022B00F0EE82002800F061836B4B4FF4C2
:107C40007A7E96F8F1854FF0000C03F5247B5A8874
:107C5000B2F57A7FB3F8462088BFA3F802E0B2F508
:107C60007A7F9A8888BFA3F846E0B2F57A7FDA88EF
:107C700088BFA3F804E0B2F57A7F02D90022A3F806
:107C800006C099889142B3F85A10B3F85C2098BFA7
:107C9000A3F804C0914293F86B2002F1FF3288BF31
:107CA000A3F85AC0632A03D94FF0640283F86B200B
:107CB00093F86C2003F1660019460132D2B2092A0A
:107CC0004FF0000288BF83F86CC08D7A013210F843
:107CD000014B0631A54238BF00F801CC032AF4D18C
:107CE000B8F1010F03F1A40318BF03F81FCC5B45E3
:107CF000ADD13F4B9B78042B00F0D4822BB93C4A8A
:107D00001388B3F5F07F00F2F881FFF731FE3948B0
:107D100096F80B16FEF72CFC0E3096F81916FEF7A7
:107D200027FCB6F82626B6F824361343B6F82826DC
:107D300013431BB213B10123A6F82A36D6F8E03557
:107D40002D4A1A40002A00F0E982D90700F1538237
:107D50005A0440F1D6812949D6F8E4250B400A405F
:107D6000C6F8E035C6F8E425180440F11182002277
:107D700086F83F2486F84F24D90440F1148296F8FF
:107D80003736022B02D1012386F83736DFF870B080
:107D90005B460BF1780402E00633A3420CD01A785C
:107DA000072AF9D19978DA78914202D35A79002AD0
:107DB000F2D0072023F0C0FB00234FF4806086F848
:107DC000FC3414F08BFF002800F086820C4DA8468E
:107DD00098F8051029B398F8000000B35B4618E046
:107DE000A85200242C330A08BC02020004540024C8
:107DF000E4290024B458002409600002F6DFFFFDE6
:107E0000E4580024105700248180808006339C426F
:107E100007D01A788A42F9D15A79002AF6D023F08D
:107E20008BFB08F106084445D2D1B84B93F802B059
:107E3000BBF1080F00F00B8296F8F135D6F8E42577
:107E4000A3F10103C2F3C031B3FA83F386F8B71686
:107E50005B0986F8B43696F8F235A3F10103B3FA5C
:107E600083F35B0986F8BA3696F8ED33032B02D913
:107E7000002386F8ED33A649D6F8E0350A400B40DA
:107E8000B17CC6F8E425C6F8E035002900F0EB81A6
:107E9000B6F8D036002B40F0F281D6F8D43613F085
:107EA0007F4F02D00023C6F8D436D6F8DC36994A84
:107EB0001A401AB140F20223C6F8DC3696F8D836DA
:107EC000013B042B02D9012386F8D836ABF1050B10
:107ED000914BBBF1030F93F890B540F27781BBF162
:107EE000000F20D00023FB60884B6FF007017C60FF
:107EF000C91A03F108080C4604E004EB08035B45CB
:107F000080F01C8118F8010B0028F6D00DF05CFE03
:107F10000028F2D083799B07EFD5FB6801227C68AB
:107F2000002B40F01181794B9B7913B10023774AE4
:107F30009371B6F8E63613F00C0F03D1C3F30313B5
:107F4000022B03D94FF42063A6F8E636B6F8E836DC
:107F500013F00C0F03D1C3F30313022B03D940F624
:107F60000123A6F8E83696F8592796F865379A421D
:107F700000F2368196F8583796F864279A4204D270
:107F8000002386F85837A6F85C3796F85A2796F8F3
:107F90004E389A4202D9002386F85A375F49FC606E
:107FA00001F1780BBC6811F8013C4FF0030803EBBA
:107FB0004303234493F88CE293F88DC293F88E0226
:107FC0000B461A787245A8BF724603F8012B5A79FE
:107FD0006245A8BF62465A719A788242A8BF02469B
:107FE000B8F101089A70ECD11E318B45DBD1D6F87F
:107FF0006024FC68002A00F04C810020012102E08E
:108000000635AC420ED02B78282BF9D16B7804338F
:1080100001FA03F31342F3D0063522EA03020120EA
:10802000AC42F0D108B1C6F860243D4D05F108041A
:108030002B4613F8012B072A00F293809C42F8D1BB
:10804000EB4688B0FF2120226B46184659F0FAFA19
:108050003349034611F8012B53F82200013040F058
:1080600087808C4243F82220F4D1B6F8EA25DD4619
:10807000B6F8E8359A4202D32A4BC6F8E835FF2312
:10808000294986F880389AF90430142B05D0DAF89B
:10809000002031EA020200F002810AF10C0ACA450E
:1080A000F1D1224B5A79022A01D100225A71143798
:1080B000BD46BDE8F08F1E4814F0C8FDB0E51D4A6E
:1080C0001146BA60DA0001EBC30393F8D41021B172
:1080D000D3F8D830002B00F0FB80BB68134493F832
:1080E000D520002A3FF432AD93F8B431002B7FF451
:1080F0002DAD182386F8203428E54FF4F073138053
:1081000003E61D0740F180800B4925E6E4290024A1
:10811000FFDFFFFDFDFDFFFF241D00208F53002426
:10812000F7290024AE014A0101000200E02D0024DD
:10813000105700242C330A08FE9FFFFDFB68002225
:108140007C68002B3FF4EFAE7A494B7C002B7FF428
:10815000F0AE4B79012B3FF4E6AE002A7FF4E3AE9C
:10816000E7E6EB4688B02022FF21684659F06AFA1C
:1081700005F8018B08F10108B8F1080F3FF475AF5D
:1081800005F8018B08F10108B8F1080FF0D16CE790
:1081900096F83F24002A00F0AC800022D90486F82B
:1081A0004F243FF5ECAD1A067FF5E9AD96F8203483
:1081B000182B06D801229A405F4B1340002B7FF406
:1081C000DEADDFF888B10BF17804F5E50023594AFC
:1081D0001371BBF1000F00F09F800123FB6083E669
:1081E000002296F8583786F85927002B3FF4CDAE79
:1081F000A6F85C27C0E65149D6F8E4250B400A40B2
:10820000C6F8E035C6F8E4259C047FF5ADAD4C49D1
:10821000A2E500283FF412AD4A4B4FF0FF0C90F955
:10822000045096F84D1503F1900093F90820AA42E6
:1082300004D10139012483F808C0C9B20C33834248
:10824000F3D1002C3FF4FAAC86F84D15F6E41A464B
:108250009B79002B3FF4F0AD537C012B7FF4ECAD08
:1082600002235374E8E538490B430A43C6F8E03566
:10827000B6F8D036C6F8E425002B3FF40EAE96F8DB
:10828000CC060DF0A1FC00287FF407AEA6F8D006BE
:1082900003E6282023F050F9D6F86024ADE686F8EE
:1082A0008038FEE6D6F8E035224A23F48053C6F83B
:1082B000E035D6F8E43523F48053C6F8E435538C22
:1082C000B3F57A7FBFF421AD4FF47A7353841CE584
:1082D000172386F8203400E7D6F8E03523F0006352
:1082E000C6F8E035D6F8E43523F00063C6F8E43587
:1082F0006CE542F2010213427FF44FAF3CE5D6F841
:10830000E025D6F8E43522F0800223F08003C6F899
:10831000E025C6F8E43591E45A4615E7D6F8E42599
:1083200043F0080342F00802C6F8E035C6F8E42539
:108330000BE500BFE429002400410001F79FFFFD89
:10834000F6BFFFFDF857002420063700E45800244C
:108350002DE9F04F864E83B096F88438013B012B0F
:1083600040F2F480D6F8B8284FF0010A814BDFF8CC
:10837000288202F2DC524345C6F8B8284CD29B460C
:108380007D4B7E4D9F1C7C4B5988002900F0C3809B
:108390007A18AA4234BF00200120052998BF40F076
:1083A0000100002840F0B780BBF800003C46C0F355
:1083B0000B000BE0118814460A44002900F0AB8042
:1083C000AA4280F0A880052940F2A58061888142F8
:1083D000F0D161798B07EDD123885846DBF808107E
:1083E00094F804900193FEF7BFFABBF80010B9EBC4
:1083F000113F00F098804FF0000ABBF804100BF119
:108400001C0B5BF8140CC1F30B014FF0C3FE5BF8BF
:10841000042CC3451060B6D3D6F8E035584DC6F8E5
:10842000E435FFF785FB3379A5F17801554C03EB73
:10843000830203EBC2037279C2EB021205EB8303E2
:1084400001EB4202C6F81C34C6F8182422F0A4FA44
:108450004FF0FF33D6F81C0463602BF01DF923F0B6
:10846000BDF805F59C6305F5AB6102E00633994262
:1084700063D01A78002AF9D19D78D878854202D342
:1084800058790028F2D096F834366421227203EB32
:10849000830303EB83039B00632BD8BF6423C6F8DD
:1084A000B038B6F8383601FB03F3632B4ADD1A46C1
:1084B000C6F8B43800233449C6F8CC28C6F8B83812
:1084C000C6F8BC38C6F8C038C6F8C438C6F8C838CC
:1084D000A6F8D03886F8D2382C4BC1F8C0362DF02B
:1084E000DDFC96F8D618B6F8D40825F02BFA3BF048
:1084F000B5F818F07BF896F88438013B012B2FD99A
:10850000234B012250461B6886F8D128C6F8B8389C
:1085100003B0BDE8F08FDBF8081058464FF0000AB2
:10852000FEF722FA69E7019BA11D58469A1FFDF745
:10853000A9FC00287FF461AF5DE7F27C003A18BF28
:108540000122A0E70A46C6F8B418B3E708F07EFE99
:10855000104B0222034486F8A828C6F8A43801E785
:1085600008F074FE0223C6F8A40886F8A838C7E706
:10857000A852002428860B08000002080000040806
:1085800004540024B4040024241D0020CC580024EA
:10859000581E002460E31600908F0B0838B50122A6
:1085A0001C4B032805461C4C83F8C82620D96A1C9E
:1085B00000231A490220D2B24FF0140E5200402A72
:1085C00028BF4022C854023301EB030C9A420CF836
:1085D00001ECF7D8FF2D4FF0FF034FF00E0008BF5E
:1085E0000222224482F8D838BDE8384016F0A2BDF5
:1085F00000EB800004F5AE73257105EBC00003EBC2
:108600008000C4F81C042BF047F829F08DFF2AF0F5
:108610005FF8CCE7241D0020A8520024805B0024D2
:10862000054B0121D3F81C2983F8191942F40012D3
:10863000C3F81C29704700BFA85200240368C3F385
:10864000100230B5044687B00D463ABB2021039294
:10865000CDE901220122CDE9042103F17841B1F5F0
:10866000801F0DD2029203F17843694601A85B0C8A
:10867000039348F047FF88B14FF0FF3007B030BD9B
:10868000A3F10162B2F5801F04D20222A3F5801388
:108690000292E8E705200DF041F9FBE72946206842
:1086A0004FF01AFD18B9236820332360E6E76FF016
:1086B0000100E3E72DE9F041694F92B03B78B12B1F
:1086C0007AD1FEF7A4F980F00104E4B2654B04F01E
:1086D0000104654DB3F89B32644EADF80030B542ED
:1086E0006CD3002C00F0B9803022002106A858F08D
:1086F000A9FF5F4B0497DB1B05935E4BDA68D40739
:108700006BD45C4BD3F80C21D0076FD40123002528
:108710000222694604A88DF840300F9556F0CCF837
:10872000022269464FF6FF704F4FFEF751F904469B
:10873000B74265D30025022201A904A8ADF8045070
:1087400056F0BAF8022201A92046FEF741F940BAD4
:10875000022202A9C043ADF8080004A856F0ACF804
:108760000E9878B106ABC0F120022946184458F0A3
:1087700069FF0F9818B906A904A8FFF75FFF002347
:108780000F900E939DF840300F987BB1394BDA680B
:1087900042F00102DA60DA68D20707D5D3F80C217B
:1087A00042F00102C3F80C21D3F80C31B0FA80F08A
:1087B000400912B0BDE8F081012487E7A9881C3583
:1087C00055F8140CC1F30B014FF0E4FC55F8043CD0
:1087D0001B68834218BF012481E7274A5A6002F1CF
:1087E00088325A60DB68D9078BD58FE7224AC3F8F5
:1087F000042102F18832C3F80421D3F80C3185E753
:10880000B7F8048002A904A88DF80D50C8F30B082E
:108810001C3708F10603ADF8083037F81C3CC3F3E9
:108820000B021B0BADF80A2006228DF80C3056F017
:1088300043F8062202A92046FEF7CAF8044657F874
:10884000141C424604A856F037F8204657F8141C6A
:108850004246FEF7BDF804466AE70120A9E700BFDB
:10886000000002082C330A0828860B08908F0B089A
:1088700000000408002000522301674570B5244C15
:10888000FFF756F994F88438013B012B2ED9D4F820
:10889000B83801221F4E03F2DC53154684F8202914
:1088A000C4F8B838FFF706FFC0B13378B12B15D143
:1088B000FEF7ADF890B194F884380022013B84F8BB
:1088C0002029012B1CD9144B012100221B6884F89C
:1088D000D11884F82129C4F8B83870BD032D01D00F
:1088E0000135DFE705200DF019F8E4E708F0AEFCEC
:1088F0000A4B0222034484F8A828C4F8A438C6E727
:1089000008F0A4FC0223C4F8A40884F8A838DAE725
:10891000A852002400000208581E002460E316003C
:1089200001230B4A10B50B4C82F8C836A374FFF72D
:10893000A5FFFFF70DFD41F20242FF230E20A4F830
:10894000D82884F8DA38BDE8104016F0F3BB00BF31
:10895000241D0020A852002490F88730F7EE002A4A
:10896000DFED695A002103EE903A90F88B3006EE65
:10897000103A90F88930F8EEE33A04EE103A90F8A5
:108980008A30B8EEC66A04EE903A90F88D3063EE05
:10899000A57A03EE903A26EE256AB8EEC44AF8EEC0
:1089A000E44AF8EEE33A26EE276A24EE254A64EE1E
:1089B000A54A63EEA53A24EE064A64EEA74A63EEA2
:1089C000A73AF0B5514D062600F1660EA5F10C0C44
:1089D000B7EE005A06FB01F290F88670AC1802441C
:1089E000F0EE456A15E0012904F1060402F10602E1
:1089F000EED190F8883007EE903A90F8903006EE7D
:108A0000903AF8EEE77AF8EEE66A27EEA55A66EEB7
:108A1000A56A237866EE867A07EE103AB8EEC77A32
:108A200027EE277AFDEEC77A17EE903A66EE847A43
:108A3000FA2BA8BFFA2323EAE3731372637807EED5
:108A4000103AB8EEC77A27EE277AFDEEC77A17EE0E
:108A5000903AFA2BA8BFFA2323EAE37353725CF827
:108A6000213007EE903A002BF8EEE77A49DDA37843
:108A700007EE103A90F88C30B8EE477A03EE103AD1
:108A8000B8EEC33A37EE677A23EE253A87EE272A07
:108A9000B0EE627AA2EE037A64EEA77A66EEA36A7B
:108AA00067EE857A27EE877AFDEEE77ABDEEC77A24
:108AB00017EE103AFA2BA8BFFA2323EAE373937256
:108AC00017EE903AFA2BA8BFFA2323EAE3730EF8C5
:108AD00001300131A38807EE903AF8EEE77A67EEAD
:108AE000A67AFDEEE77A17EE903AB3F57A7FA8BF43
:108AF0004FF47A738F4223EAE3739381BFF673AF27
:108B0000F0BDB7EE007AC7E70AD7233C583A0A0807
:108B100090F88E306BB3B0F85A308BB190F88F204C
:108B2000642102EB8203C3EB0313B3FBF1F3A0F860
:108B30005A30962312FB03F3B3FBF1F3A0F85C3039
:108B400043884BB190F88F30642203EB8303C3EB6F
:108B50000313B3FBF2F34380B0F846304BB19622D7
:108B600090F88F3013FB02F36422B3FBF2F3A0F80A
:108B70004630704790F821304BB3438B83B190F867
:108B80002230FA22642113FB02F203EB8303B2FBCF
:108B9000F1F2B3F57A7F4283A8BF4FF47A738383EF
:108BA000838843B1FA2290F8223013FB02F3642247
:108BB000B3FBF2F38380C3884BB190F8223003EB10
:108BC0008303B3F57A7FA8BF4FF47A73C3807047ED
:108BD00070B50B4C002504F5247694F8863013B15B
:108BE0002046FFF7B9FE20460135FFF791FF3046DA
:108BF000FFF7C0FF042D04F1A404EED170BD00BF47
:108C000004540024034B53F8E00C08B106F0E6BF0F
:108C1000704700BFA063002408B50B460549024613
:108C200051F8E00C28B10449FEF7F8F9BDE8084016
:108C3000E8E708BDA06300248D670408024B0146E5
:108C400053F8E00CFDF7A4BDA063002408B504466A
:108C50000848FFF7F3FFFFF7D5FF074BD86F16F073
:108C6000E7F90CF057FC012C01D150F05FFFFAF747
:108C70005DFA00BFE5EE0A08A85200240048DDE7CF
:108C80008EFA0A080CB4C30607B500D561B905A968
:108C900004980191FFF7C0FFFFF7F0FF012003B038
:108CA0005DF804EB02B070470020F8E708B5FFF765
:108CB000C5FFBDE80840E1E710B504460348FFF7EB
:108CC000BDFF2046BDE81040F0E700BFF1EE0A0806
:108CD0000848002408B5FFF7EFFFFFF793FF064BA6
:108CE00003F8DC4C5C6283F8284029F017FE20462C
:108CF000FFF7ACFFF6EE0A08A0630024034B014621
:108D000053F8E00C08B106F055BF7047A06300248B
:108D10000CB407B510F020000BD079B92320FFF771
:108D2000EDFF05A904980191FFF776FFFFF7A6FF75
:108D3000012003B05DF804EB02B070470020F8E7B3
:108D40000FB407B504A951F8040B0191FFF764FFB4
:108D500003B05DF804EB04B07047154B1B6870B5A9
:108D60002BB30025134E1448FFF7A0FFFFF74AFF6F
:108D7000FCF720FAFCF750FA044640B1132016F035
:108D8000D9F9FFF77BFF0D48BDE870408EE730460C
:108D9000FFF7D6FF782D06D80135FFF733FF6420A3
:108DA0000CF01CFCE6E72546FFF768FFF5E770BD11
:108DB000201E00247A330B081DEF0A0837EF0A083B
:108DC0000FB407B504A951F8040B0191FFF724FF74
:108DD000FFF754FF03B05DF804EB04B070472DE9D2
:108DE000F041037903F0E002402A50D004D85AB190
:108DF000202A29D0BDE8F081602A4BD0802AF9D101
:108E000082794179254812E003F00703052B16D833
:108E1000DFE803F0101510150309D0F805102048FD
:108E2000BDE8F041CCE7D0F8052051421D48BDE82F
:108E3000F041C5E7B0F80720B0F80510F6E7B0F943
:108E40000720B0F90510F1E746790024164D1748C0
:108E500005EBC605FFF7F2FE012395F84477A7421C
:108E600002D8BDE8F04109E7D5F840674FEA840829
:108E700056F824204AB113B90D48FFF7DFFE56F823
:108E800008100C48FFF75CFF00230134E7E7417945
:108E90000948C5E70948BDE8F04191E78CEF0A08A9
:108EA0003DEF0A0853EF0A082C330A086AEF0A0854
:108EB000F6F20A0899030B087BEF0A08A3EF0A08E9
:108EC0002DE9F04387B0224EFCF764F902698389EB
:108ED00000250188044602928268DFF888800192AA
:108EE00042881C4FDFF88090009242681A48FFF7D2
:108EF00067FF15B94046FFF7D9FE3B689D4212DA7D
:108F00003378052B21D809EB8303D3F8E828B388FD
:108F10002946013511480093063636F8043CFFF720
:108F20004FFF062DE5D14FF0A1FF81884388CB1A72
:108F3000616803FB01110591FCF7B4F9059902463C
:108F4000074807B0BDE8F0433AE70022DFE700BF7B
:108F5000DC2A0024CC2A0024BBEF0A0825F00A08EA
:108F600034F00A0819F00A082C330A0802490348A9
:108F700001F500610EC923E700E0F11F51F00A0876
:108F800010B5752104462DF071FA01460948FFF726
:108F900017FF1A2120462DF069FA01460648FFF70F
:108FA0000FFF1B2120462DF061FA01460348BDE862
:108FB000104005E765F00A0878F00A088BF00A0807
:108FC00038B50C4D95F8EF0310F0FD0405D10A48B3
:108FD000FFF7F6FE2046FFF7D3FF95F8EF33013B8E
:108FE000012B06D80548FFF7EBFE0120BDE838400D
:108FF000C6E738BDA85200249EF00A08A9F00A0866
:10900000714B42F201011A68B1EB124F4FEA124361
:109010002DE9F04F93B000F0D38042F20302934267
:1090200000F0D08041F20302934214BF09230A23C7
:10903000664A674E116806EB8303664A664C6748CA
:10904000674DDFF8F481DFF8C091B1FBF2F2D3F89D
:109050000019FFF775FE628D4FF47A730A20B2FB98
:10906000F3F103FB1122B4F92C3092B2B2FBF0F20F
:109070005C48FFF7A5FE5C4A5C495D48FFF760FE6F
:10908000FFF7FCFDA97C5B4A06EB81015A4B5B486C
:10909000D31AD1F84819B5F88220FFF791FE584845
:1090A000FFF7CCFD94F82E105648FFF749FE5648BE
:1090B000FFF7C4FD94F82F105448FFF741FEFFF767
:1090C000DDFD5348FFF7BAFD00210A4695F80B3441
:1090D0004F1C0B4113F0010F08D012B14846FFF7A7
:1090E000ADFD39464046FFF72BFE0122072F3946DA
:1090F000ECD1484F97F86A1507F5EC7307F13C027D
:10910000012918BF134693F8DC30032B02D04248E4
:10911000FFF716FE414B97F86A15A3F5CE720129A9
:1091200018BF134693F8DC30012B02D13C48FFF7FF
:1091300007FE3A4B97F86A15A3F5CE72012918BFBE
:1091400013461B695B7B012B02D93648FFF7F8FDFC
:10915000DFF8E890FFF792FD4FF00008236B09F16C
:10916000200A039359F8041B002969D0012303FA4C
:1091700008FB039B1BEA030F1FD01BF01F0F1CD023
:10918000294B5AF8282013F8080052F82020B8F18B
:10919000000F06D02548CDE90412FFF74FFDDDE9A9
:1091A00004122348FFF7CCFDBBF1020F05D197F85D
:1091B000ED1611B11F48FFF7C3FD08F10108D1E713
:1091C0000B2335E70C2333E70010005CD0030024A9
:1091D0002C330A0840420F00A0630024BCF00A08A8
:1091E000A8520024CFF00A08F8FF01200008000070
:1091F000F0F00A08000004080000020814F10A0850
:1092000043F10A0855F10A085DF10A085FF10A08FE
:1092100067F10A08241D002080F10A08FC1E0020C6
:1092200088F10A088DF10A08D8040024F6F20A0829
:1092300095F10A089BF10A0877F10A087C3C0A08B4
:10924000FFF71CFD95F87E1ED5F8802E06EB8101F8
:109250007C48137AD1F88419527AFFF7B1FD7A4924
:109260007A48FFF76DFD7A497A48FFF769FDFFF705
:1092700005FD794B794819684FF47A73B1FBF3F126
:10928000FFF75EFD07A8FEF723FB38B107A90AA880
:1092900055F03EFC0AA97248FFF752FDFFF7EEFCBD
:1092A000D4F8BC20002A00F0888007EE902ADFED79
:1092B0006D6AB8EEE77AC6EE877AFDEEE77A17EECA
:1092C000903AB4F8340858B107EE900ADFED656AB9
:1092D000F8EEE77A86EEA77AFDEEC77A17EE900AE7
:1092E000E16B59B107EE901ADFED5E6AF8EEE77AAE
:1092F00086EEA77AFDEEC77A17EE901AB7F82877B0
:10930000642FCDE9000139465748A8BF6421FFF713
:1093100057FD94F8363894F8372806EB8303B4F8F1
:1093200038185248D3F89839FFF74AFD504B514846
:10933000198889B2FFF744FDFBF72CFF016921B1C1
:1093400082684D48120DFFF73BFD4C48FFF776FC55
:10935000D5F8E4351B0660D594F86438032B8CBF30
:1093600047484848FFF76AFC95F80035022B26D19C
:109370004548FFF763FC94F86438042B44D843480D
:10938000FFF75CFC94F87438002B44D006EBC30361
:10939000D3F8F0193E48FFF7D3FCFFF76FFC3D48C8
:1093A000FFF74CFC3C4FD5F81C490125002C38D167
:1093B000FFF764FC13B0BDE8F08F134681E702208D
:1093C00013F0ACFC074608B93448D2E73AF02CF960
:1093D00097F9041006EB80000131D0F8AC29304831
:1093E000FFF7AEFC95F80335012B04D12D48FFF7AC
:1093F00025FC2D48BDE7BB792C4806EB8303D3F849
:10940000AC19FFF79DFCF4E795F802350BB9284835
:10941000B6E72848B4E72849BCE72848FFF70EFC20
:10942000BBE794FAA4F33846B3FA83F305FA03F2E0
:1094300006EB8303D3F8241A24EA0204FFF780FC26
:10944000B4E700BF9FF10A08B1F10A08D2F10A0897
:10945000E0F10A0823340B08581E0024E6F10A083C
:1094600000F20A080024744913F20A0859F20A08A3
:109470004821002480F20A088FF20A08AAF20A089A
:10948000B0F20A08BCF20A08CCF20A0899350B08B7
:1094900014F30A0830F30A0820F30A08D2F20A0883
:1094A000DCF20A08F0F20A08F5F20A0815FD0A08CB
:1094B000F9F20A0809F30A08B4F00A0824F30A08C2
:1094C0002DE9F04FDFF8748199B098F80730002B40
:1094D00000F0978050480025504EDFF864B1FFF748
:1094E000E5FB2F46DFF85C91DFF85CA10BA9E8B241
:1094F00017F0CCFA9DF83430002B53D0139C54B1A4
:1095000007EE904A9FED460AF8EE677A80EE270A4A
:1095100057F0A6FA04460B9A29465846FFF710FC66
:10952000109A002A6FD002FB04F04FF47A73B0FB5C
:10953000F3F30993DDF848C0BCF1000F65D00CFBD4
:1095400004F142F21073B1FBF3F1082D98F80730E3
:1095500018BF7F18002B5AD017984FF47A7E0A2331
:10956000079015980690169805901198B0FBFEFE8E
:10957000CDF810E00998B1FBF3FE03FB1E11CDE915
:1095800002E10999B1FBF3F103FB1100BCFBF3F31A
:10959000CDE9001021465046FFF712FC0023B362CC
:1095A000C6E90D3301354036202D9FD198F807309C
:1095B00023B31C4C4FF47A731B48D4F87818D4F8B2
:1095C0007C28B1FBF3F3D208D4F88018FFF7F8FB3E
:1095D0000A221648B7FBF2F102FB1172FFF7F0FB0B
:1095E000134B1B78432B06D1D4F88428D4F8881861
:1095F0001048FFF7E5FB0023C4F8803819B0BDE838
:10960000F08F0D4867E7099294E761469DE7214690
:109610004846FFF7D5FBC1E746F30A08D4630024A8
:109620008096184BA0630024EDF30A080DF40A0895
:10963000B01E002431F40A08A4F30A08A85200243A
:10964000AEF30A0835030B08BDF30A0813B5294821
:10965000FFF7F4FA284B93F85134002B48D02748F1
:10966000FFF724FB20F0F6FE80B1254B254893ED53
:10967000280A8DED010AFFF7E1FA234B9DED010A5F
:10968000B3F834383BBB2148FFF710FB204C21488E
:10969000B4F8C417FFF754FB94F8C03713B31E484F
:1096A000FFF704FBB4F8C8171C48FFF749FB94F810
:1096B000C237CBB11848FFF7F9FAB4F8C617184803
:1096C000FFF73EFB94F8C13783B1134802B0BDE801
:1096D0001040FFF7EBBA57F0C3F981B21148FFF71A
:1096E0006FFBD3E71048DBE70F48E4E70E48EDE7F0
:1096F0000E48EBE75BF40A08A852002471F40A084C
:109700005024002078F40A08A063002492F40A0888
:10971000241D0020A1F40A08C1F40A08D1F40A08A3
:10972000EBF40A089CF40A08CAF40A08543C0B0833
:109730000EB403B503AA52F8041B0192FDF788FD8D
:10974000074B53F8E03C2BB9064B0749D3F884008C
:10975000FDF71EF802B05DF804EB03B0704700BFE0
:10976000A0630024A85200248EFA0A082DE9F047CD
:1097700098460B7981460F4603F0E0041646402CCC
:1097800031D10024674DDFF8A081DFF8C09122E0DD
:109790003B7903F00703013B042B04D8DFE803F017
:1097A00006080B0E2000315D28460AE03157FBE722
:1097B00036F81410F8E736F91410F5E756F82410C7
:1097C0004046FFF7BDFA7B79013BA34202DD4846E4
:1097D000FFF734FA01347B79A342D9DCBDE8F08786
:1097E00056F82410E0E703F00703052B58D8DFE80C
:1097F00003F0030C141619313578602C5ED045D86F
:10980000002C66D0202C7CD0E8E796F90050602C24
:1098100054D03BD8002CF5D148E03588EDE7B6F9B7
:109820000050F4E7D6F800A0202C554669D02BD87C
:10983000002CD3D151463C48FFF782FAD7F80510E7
:109840008A4518D8B8F1000FC8D03848BDE8F047AD
:10985000FFF776BA202C356853D015D8002CBDD12F
:1098600029463048FFF76CFAD7F80510A94202DB09
:109870004B42AB42E6DDFFF701FA2B463A68484619
:109880002B49BDE8F04753E7602C17D0802CA5D1B9
:109890003178284B2848002914BF31461946D5E7AE
:1098A000202C2DD007D8002C98D12546B7F905409B
:1098B000B7F9076011E0602CE8D100257B7945FA03
:1098C00003F3DB07BDE8F0474CBF1C481C48FFF71B
:1098D00037BAB7F80540B7F8076029461148FFF7CF
:1098E0002FFAAC42C7DCAE42C5DBB8F1000F3FF443
:1098F00075AF324621461348BDE8F047FFF720BA5E
:1099000000257A79104B03EBC20393F84427954264
:10991000B1DAD3F8403753F82500BDE8F047FFF738
:109920008DB900BF343B0B0850EF0A080BF50A084D
:1099300011F50A0806340B0899030B08B8EF0A085A
:10994000543C0B0807FE0A082C330A085DF10A088C
:1099500013B50446084601920091FCF7ABFF02469E
:109960002046DDE9001302B0BDE81040FEE60EB46B
:1099700003B503AA52F8041B0192FDF769FC054BDD
:109980000549D3F88400FCF703FF02B05DF804EB4F
:1099900003B07047A85200248EFA0A080246014913
:1099A000E5E700BF2BF50A08F8B50C460646084661
:1099B000FDF7B0FE20210546204657F04AFF044639
:1099C00018B93046BDE8F840E8E7114F114E3B7832
:1099D00032789A4201D0FBF721FD0F4B20461D60E3
:1099E00055F00EFA012201462046FBF7B9FC3B7800
:1099F00032789A4201D0FBF711FD204655F000FA6B
:109A00002A4601460548BDE8F840FFF7D9B900BF2E
:109A10001C1E0024D42A0024181E002442F50A0823
:109A20002DE9F0410D4688B006460846FDF772FE66
:109A300020210446284657F00CFF20B9304608B0D4
:109A4000BDE8F041AAE7FDF765FE2246054601465E
:109A50000F48FFF7B5F985B1202D2A466946204603
:109A600028BF2022E846FBF7F5FC00270646B74250
:109A700008DBAD1B3444002EEDD1FFF7FFF808B032
:109A8000BDE8F08118F8010B0137FFF737F9EEE771
:109A900058F50A0810B504460748FFF707F9FBF721
:109AA0006FFD20B10548BDE81040FFF7FFB8204624
:109AB0000349BDE810405AE770F50A087AF50A082C
:109AC00082F50A08154BD3F8683B2DE9F0410446AE
:109AD00088B0F3B11A6804A91846D56A6A46A8473F
:109AE000064688B104AC6D460027DFF83C8001379C
:109AF00035F8022B34F8021B4046FFF761F9BE42ED
:109B0000F5DC08B0BDE8F08105492046FFF72FFFDE
:109B1000F7E7044908B0BDE8F04128E7A85200245F
:109B2000A3F50A08BBF50A0889F50A0813B5044627
:109B30000846019155F064F9024670B10D2804D130
:109B40000199094857F0ABFE38B1074B2046074A48
:109B5000074902B0BDE8104009E70349054802B0D3
:109B6000BDE81040FFF72CB968AC0A08C2F50A0836
:109B7000CDF50A08F7F50A0813B504460846019121
:109B800055F03EF90199024668B1042803D109480D
:109B900057F085FE38B1074B2046074A074902B007
:109BA000BDE81040E3E60349054802B0BDE81040B7
:109BB000FFF706B960AC0A0805F60A08CDF50A08F1
:109BC00015F60A082DE9F04300279BB00646084623
:109BD0000C4655F015F905461C22394602A8019796
:109BE00057F030FD25B3402D07D040232A46384991
:109BF00030461BB0BDE8F043B9E60DF1040804F1AE
:109C0000400902222146684657F05DFE00231022DB
:109C100009A968468DF80270FDF7D8FC099B0DF183
:109C20000202934222D1023408F8010BA145E8D187
:109C300000213D220AA8099157F004FD002D3AD0D9
:109C4000244C257DD5B1202204F1180101A857F03C
:109C5000CFFC98B104F1180109A8FDF7D5FB09ABB9
:109C60001D4A30461D49FFF782FE04E01A7830464F
:109C70001B49FFF77CFE1BB0BDE8F08394F88030F1
:109C8000CBB9C5B901AD174C0FCD0FC495E80F0086
:109C900084E80F00144B012209A8A4F1100183F8F5
:109CA0008C28FDF7B1FB1148FFF706F809A9104809
:109CB000FFF786F8DFE70C4B93F88C381BB9054BA0
:109CC0001B7D002BF2D0074909A8FDF79DFBEDE7AE
:109CD00028F60A08A852002466F60A08CDF50A08F4
:109CE0004AF60A08C0520024A063002470F60A084D
:109CF0007FF60A082DE9F74F394F834608460D468F
:109D000055F07EF8D7F8E0950446B8B9354D0126F0
:109D1000354F3648FEF792FF55F8041B49B106FA55
:109D200004F313EA090F02D03846FFF709F80134AB
:109D3000F2E703B0BDE8F04FFEF7A0BF02462C49A2
:109D40002846FDF7F3FB78B9264C2A4D2A48FEF742
:109D500075FF54F8041B0029EBD00B78002BF8D0CA
:109D60002846FEF7EDFFF4E72B782D2B11D10135B6
:109D7000013C4FF0010A1B4B002653F8048BB8F14D
:109D8000000F09D12A461D49584603B0BDE8F04FDF
:109D9000EDE54FF0000AEEE72246414628460193E2
:109DA000FDF7C4FB019BC0B90123B340BAF1000F1A
:109DB0000DD029EA03031248C7F8E035FEF73EFF4D
:109DC00041460C4803B0BDE8F04FFEF7F9BF49EA41
:109DD00003030C48C7F8E035F0E70136CDE700BFD4
:109DE000A8520024B83D0A0896F60A088CF60A081C
:109DF000A9F30A0820F30A089AF60A08A5F60A0841
:109E0000B6F60A08BFF60A082DE9F74F814608465C
:109E10000E461746984654F0F3FF0446E8B9404D05
:109E20004048FEF78DFF204612F00AFD3B681842BD
:109E300006D0204612F016FD01462846FEF780FFA8
:109E40000134182CEFD13B6813B93748FEF7F6FE02
:109E500003B0BDE8F04FFEF711BF0246334930466C
:109E6000FDF764FB0546A8B92C46314D3148FEF795
:109E7000E5FE204612F0E4FC10EA080F06D020466A
:109E800012F0F0FC01462846FEF75AFF0134192C67
:109E9000EFD1DDE733782D2B2AD10136013C0125A6
:109EA00048F080734FF0000A0193504612F0DAFC3C
:109EB0002246834601463046FDF738FB18BB504624
:109EC00012F0BEFC019B03421DD09DB1BAF1180FE8
:109ED00002D03B6840EA03081748C7F80080FEF745
:109EE000ADFE5946124803B0BDE8F04FFEF768BF1B
:109EF0000025D5E7BAF1180F02D03D6825EA000524
:109F00000E483D60EBE70AF1010ABAF1190FCCD116
:109F100032460B49484603B0BDE8F04F27E500BF85
:109F20001FF30A08C7F60A08D1F60A08A9F30A08B7
:109F300020F30A089AF60A08B6F60A08BFF60A08D5
:109F4000A5F60A0840F20223004A5DE7845900247E
:109F50006FF07F43004A57E77C59002410B5044650
:109F60002BF068FE20B920460449BDE81040FEE40D
:109F70000348BDE81040FEF723BF00BFD8F60A082B
:109F8000E7F60A0870B5054608461646FDF7C2FB17
:109F90000D4B044693F89025904205D201460B489C
:109FA000FEF70EFF204670BD2EB1FF2803D10848F2
:109FB000FEF706FFF6E7013A064928464FF0FF3460
:109FC000FFF7D5FCEEE700BF241D0020F2F60A08DB
:109FD00003F70A0816F70A082DE9F04F074691B073
:109FE00082480E46824DFEF7EBFE00238149402455
:109FF000062285F894383046012391F89015C5F86B
:10A0000090D885F895480BF047FA0A200BF0E6FA4D
:10A0100095F894380C2BDAB240F2E4809DF80C509D
:10A02000FE2D30D0FF2D0BBF15240F240126002656
:10A03000944240F0D780611E6846C9B240F0DAFF12
:10A0400004F140030DEB030414F8413C834240F05B
:10A05000C48006F1FF389DF80D305FFA88F8B8F13A
:10A06000010F12D903F01F075C0961376248FEF740
:10A07000E5FD022E6AD0013C042C65D8DFE804F02F
:10A080000B5E606462000226D2E79DF80E701D46EA
:10A090009DF80F40EAE759486C464FF0000ADFF898
:10A0A000B891FEF703FEDFF8B4B15548FEF7C6FDE0
:10A0B0000AF1010A14F8011B4846FEF741FEBAF105
:10A0C0000C0F49D1FEF7DAFD022E4FD064223B4639
:10A0D0004C48B5FBF2F102FB1152C9B2D2B2FEF705
:10A0E0006FFEB8F1010F71D8474A484B9DF8101028
:10A0F0004748002914BF11461946464DFEF760FE39
:10A100009DF81110444B4548002914BF19462946B3
:10A11000FEF756FE022E59D19DF812404048FEF738
:10A120008DFD4CB3FF2C37D00A223E48B4FBF2F130
:10A1300002FB1142D2B2FEF743FE20E03A48ABE701
:10A140003A48A9E73A48A7E73A48A5E700230DF1BE
:10A150001F008DF83F309FE7374B03FB0AF2B2F147
:10A16000553FA5D85846FEF769FDA1E73A4629466E
:10A170003248FEF725FEB7E72846FEF797FD9DF823
:10A1800013402F48FEF75AFD44B1FF2C21D0214641
:10A190002C48FEF715FE04E02B48EEE71D48FEF7BD
:10A1A00085FD0DF1130500241A4E274FDFF8688056
:10A1B00015F8013F7BB1FF2B0CBF3A4642462146C2
:10A1C00001342248FEF7FCFD042CF1D111B0BDE8AA
:10A1D000F08F1D48E3E73246F1E71D493846FFF7A7
:10A1E000C6FBF3E71B48FEF761FDEFE75CF70A08E3
:10A1F000A0630024241D00206DF70A0878F70A08E0
:10A200009EF70A08B0F70A083CF70A0845F70A085B
:10A21000E7F70A084CF70A08D8040B08FEF70A0803
:10A2200005F80A0819F80A087FF70A0887F70A08E4
:10A230008FF70A08B4F00A08ABAAAAAACCF70A0852
:10A2400021F80A08343B0B0850F70A0831F80A08CD
:10A250003CF80A084CF80A08D8EE0A0806340B083D
:10A260002DE9F84F07460C46DFF8A480DFF884900C
:10A27000DFF8A0A0204654F0C3FD064660B91D4B90
:10A280001D4893F820241D4B03EB8203D3F8041BD5
:10A29000BDE8F84FFEF794BD024641462046FDF763
:10A2A00045F960B1DFF85CB000255BF8041BB1B97B
:10A2B000224638461249BDE8F84FFFF758BB114C0B
:10A2C000114D1248FEF7BAFC54F8041B19B1284688
:10A2D000FEF736FDF8E7BDE8F84FFEF7CFBC324693
:10A2E00020460135FDF722F90028DED1544689F8D1
:10A2F0002054BFE7A852002455F80A082C330A0856
:10A30000A5F60A08343E0A0820F30A089AF60A0855
:10A31000A9F30A0890FA0A0838B50D460446052242
:10A3200019492846FDF702F968B9184B93F88820B7
:10A3300022B9012183F8892083F888101448BDE8E8
:10A340003840FEF7B3BC032212492846FDF7EEF869
:10A35000A0B90E4D95F8883063B195F889304BB1AE
:10A360000D492046FFF703FB002385F8883085F868
:10A37000893038BD0948FEF799FCF5E720460849C1
:10A38000BDE83840FFF7F3BA1C040B08A8520024BC
:10A390005FF80A0881050B0875F80A08ACF80A0886
:10A3A000C0F80A08F8B5174C054694F888307BB118
:10A3B00094F8893063B11449FFF7D9FA2846134954
:10A3C000FFF7D5FA002084F8880084F88900F8BDEA
:10A3D0000F4E96F88C7897B1207D0028F7D10D4D5F
:10A3E00006F698040FCD0FC495E80F0084E80F001F
:10A3F000012386F8D3380BF079FD3846E7E70120D2
:10A40000E5E700BFA852002475F80A08CFF80A084B
:10A41000A0630024C052002408B5FFF7C3FF50B169
:10A42000054B01229A74FEF729FA0448FEF744FC12
:10A430000020FEF70BFC08BDA8520024EDF80A0826
:10A4400008B5034610462AB1DB0600D511B1FEF768
:10A4500033FC002008BDF8B50D4E054696F8803057
:10A4600093B9F8BD25B12388C3F30B039D4204D0F3
:10A47000A288D4E9020157F071F81C34BC42F1D330
:10A48000002386F88030ECE7024C034FF6E700BF6C
:10A49000A852002428860B08908F0B082DE9F04F56
:10A4A000164685B01A468246019130460021334C4B
:10A4B000FFF7C6FF4FF0000906F0100305460293B0
:10A4C000FEF7A0FB2379019A03F01803934203D00F
:10A4D000002A48D1182B46D14FF00D0B274B0BFB10
:10A4E0000933B3F80900FCF7CFF980462046FBF7A3
:10A4F000E4FF0746D8E90221024401442046FBF765
:10A5000095FF80F001012A460390C9B23046FFF75B
:10A5100097FF0546DDE9022302B123BB174A0BFB77
:10A5200009FB52F80BB0B2060FD573B9594614485F
:10A530000393FEF705FCD8F808202146039B5046FC
:10A540003A44FFF713F9FEF799FB59460D48FEF719
:10A55000F7FBD8F80C20002321463A445046FFF779
:10A5600005F9FEF78BFB09F1010940F265230D3473
:10A570009945A5D105B0BDE8F08F00BFC04C0A08D1
:10A58000F4F80A08F5F80A080149FFF7F0B900BF26
:10A59000FFF80A0838B50C46054615492046FCF771
:10A5A000A1FF30B9FEF714FB1248BDE83840FEF7B2
:10A5B0007DBB11492046FCF795FFA0B90F4A82F8F0
:10A5C000E20182F8EA0182F8860282F88E0282F8BD
:10A5D0002A0382F8320382F8CE0382F8D60382F887
:10A5E0000D040748E1E72846BDE83840CCE700BF46
:10A5F0000EF90A0814F90A082FF90A08A8520024CB
:10A6000037F90A082DE9F043064687B008460C469C
:10A6100054F0F6FB082844D1671E03AD07342946E1
:10A620003A46A84612F8010FFCF756FF01F8010B55
:10A63000A242F7D10023DFF880908DF8143017F88C
:10A64000010FFCF749FF05F8010BC1B24846019123
:10A6500057F0FFF820B10199284657F0FAF828B1D1
:10A660003046FFF791FF07B0BDE8F083A742E6D17F
:10A67000104940462BF068FA0E4808230E4910F89E
:10A68000012B013B11F8014B02F118026A4402F858
:10A690000C4CF4D103A909488DF81430FEF790FB57
:10A6A000E1E70028E8D0304607B0BDE8F043FFF707
:10A6B00075B900BFD85600245CBC0A0853F90A08D3
:10A6C0002DE9F74F4FF0000B064601AA08462E4928
:10A6D0005D4656F079FF01270446DFF8BC80DFF8BD
:10A6E000BC90DFF8A4A01CBBBBF1000F28D1274C05
:10A6F000002D44D029462648FEF762FB94F88030AE
:10A700000BB904F0BDFCFCF751F9002384F8893043
:10A71000FEF75EFA15B12846FFF79DFE9FB1304661
:10A72000FFF740FE78B1FEF7A9F80020FEF78EFA99
:10A73000BBF1000F0AD02046FCF7ECFF85B2C5B98B
:10A740003046FFF721FF03B0BDE8F08F41462046B9
:10A75000FCF710FF80B949462046FCF70BFF0028A4
:10A76000EED05F4601AA5146002056F02DFF044668
:10A77000B9E74FF0000BF5E74FF0010BF2E70548A2
:10A78000FEF79AFABFE700BF1FFE0A08A85200248E
:10A7900063F90A0886F90A085AF90A0853040B08EB
:10A7A00007B5009313460A460249FFF7E0F803B0E5
:10A7B0005DF804FB9CF90A0820B10078B0FA80F03B
:10A7C00040097047012070472DE9F34106460846CD
:10A7D000FFF7F2FF0D46074670B1002401A920469D
:10A7E00001344BF0FFFC01463046FFF7EDFF122C21
:10A7F000F4D102B0BDE8F0810846FCF78BFFC4B28B
:10A80000112C72D8681C3D4DFBF7D4FF8046E8B987
:10A810003B4B03EB440393F8D4188A1E5142514139
:10A82000374B03EB440393F8D428AA5C002955D096
:10A8300093F8D538192040F2EE2100FB031321468E
:10A84000304802B0BDE8F041FEF7BABA01782846B8
:10A8500056F0FFFF78B1032C2B49A0EB050394BF02
:10A860000022012202EB42020A4452FA83F393F8D7
:10A87000747B032F04D1304602B0BDE8F04183E67B
:10A880004046FBF797FF08B3022FF4D1FCF742FFD5
:10A8900040F6CA0280B21A4B904203EB4403A8BFB1
:10A8A000104640F2EE229042B8BF10461922A0F2A4
:10A8B000EE20B0FBF2F083F8D508BB1E5942594197
:10A8C0000F4B03EB440383F8D478A9E7022FF4D1AC
:10A8D000304602B0BDE8F041FFF760B821460B48B2
:10A8E00002B0BDE8F041FEF76BBA11233A460849C1
:10A8F000304602B0BDE8F04152E700BF7CBE0A0816
:10A90000A0630024B5F90A082C330A08C5F90A081F
:10A91000D2F90A082DE9F04F024691B008460B46DD
:10A92000FFF74AFF044628B1104611B0BDE8F04FCA
:10A93000FFF734B84FF0FF3227462646DFF8E082B3
:10A94000DFF8E092DFF8E0A2CDE90820A24AD26F5A
:10A9500092F83810CDE90E02CDE90C10CDE90A00CD
:10A9600007AA9E49184656F02FFE054604944DB995
:10A97000089A0C9FBA4262D19948FEF721FA11B0A9
:10A98000BDE8F08F062F12D8DFE807F0041E232859
:10A99000454C510051462846FCF7ECFD78B14FF488
:10A9A0008060012412F0BAF990F90430089307AAE4
:10A9B0008A490020013756F007FE0546D7E72846AA
:10A9C000FCF7A8FE0890F2E72846FCF7A3FE0990E2
:10A9D000EDE72846FCF7E5FD0A90E8E7284654F045
:10A9E0000FFA4146024605902846FCF79FFD18B332
:10A9F000059A49462846FCF799FD06460028D6D018
:10AA00002846FCF787FE04280646D0D9014675483B
:10AA1000FEF7D6F9B3E72846FCF77CFE00230C903E
:10AA20000F93C4E72846FCF775FE0D90BFE7284654
:10AA3000FCF7B7FD0E90BAE701230493B7E7DFF800
:10AA4000EC8151B2434613F9010B884208D001351D
:10AA50000C2DF8D1002101316348FEF7B1F98EE7E2
:10AA600001216248FEF7ACF900237AB218F9011B04
:10AA70008A4200F00C8101330C2BF7D13A460121B8
:10AA8000E9E7A7F1140253425341059308AD0023AF
:10AA900003F10108EB68A3BB95F900B0584612F02A
:10AAA00009F9D5F804A020B1D0F80090B9F1000F51
:10AAB0005ED1BAF1000F19D14FF461434FF0010A92
:10AAC0006B60AB680BB90323AB600023D5F804902F
:10AAD0005846029319462A7ACDE900921A4614F094
:10AAE00029FAE86028B94146414891E74FF0000A49
:10AAF000E7E74A464146BAF1000F37D03D48FEF736
:10AB00001FF9B8F1020F05F110054FF00103BFD195
:10AB1000059BDDF83C800B9D53B13748FEF7C6F826
:10AB2000D8F800301B6A1BB12A4634494046984782
:10AB3000049B002B4ED03249324B142F18BF1946BC
:10AB40003148FEF73DF9142F09D1049B03B936B102
:10AB50002B68DB691BB132462C4928469847002CEC
:10AB600066D10022414628464BF0F0FA2848C6E755
:10AB7000C5F80C90BAF1000F25D041462548524641
:10AB8000FEF7DEF85146484602F07EFED5F808A0F2
:10AB9000BAF1000F0FD099F8042092450BD053461C
:10ABA00041461D48FEF7CCF8D9F800305FFA8AF12B
:10ABB00048469B699847D9F82C30002BA1D0002338
:10ABC000C9F82C309DE7D9F8082041461348FEF714
:10ABD000B7F8DBE70B49B3E7A85200241FFE0A08C9
:10ABE00010FA0A08F8F90A0854FB0A0829FA0A08B0
:10ABF00035FA0A0851FA0A0808FB0A0889D8040835
:10AC0000DAF90A0890FA0A0831FB0A08CD67040845
:10AC100075FA0A0891FA0A08E3FA0A08BEFA0A085D
:10AC2000F2F90A08D3F60A08E7F90A080C380A0804
:10AC30001C4F0026DFF874904FF0030A05F09CFDCE
:10AC400005200AF0CBFC99F89035B34289D917F862
:10AC500001BBBBF1000F15D058460AF0B5FF044602
:10AC600080B1584605F0D6FC08B1A0F806A0012135
:10AC70000490F7F777FBA379049813F0010F03D042
:10AC8000F6F7F0FE0136DEE7F6F7E6FEFAE73A46BB
:10AC900002210548FEF794F8099B002B3FF4F1AE22
:10ACA0000023F2E6EC29002429FA0A08241D0020DA
:10ACB00010B5044608460B46FFF77EFD28B903226F
:10ACC00008491846FCF732FC28B90748FDF7F4FF9D
:10ACD0000120FDF7BBFF20460449BDE81040FEF708
:10ACE00046BE00BF66FB0A086AFB0A08C0F80A08ED
:10ACF0002DE9F74F05460846FFF75EFD0B46044673
:10AD000018B9334A92F8F87827B9284603B0BDE855
:10AD1000F04F39E42646DFF8C880DFF8C89001AA72
:10AD2000DFF8C4A018462B4956F04EFC10B905F0C8
:10AD300031FD08E056B9012201462846FFF722F905
:10AD4000421C04461BD103B0BDE8F08FFCF7E2FCC7
:10AD50002F28834636D80FB105F00EFDBBF1060F44
:10AD600014D01D4901235FFA8BF291F89015E0B2DF
:10AD70000AF092FB002759464846FEF721F801AA3F
:10AD800014490020013656F01FFCCFE7DAF8E4350D
:10AD90001B0113D5FF2C0FD0E1B22846FFF71CF999
:10ADA000E8E701372846FFF717F90B4BF9B293F89C
:10ADB00090258A42F5D8DDE70027F6E70748FDF73A
:10ADC00075FFD7E72F2241462846FEF7D0FDD6E78C
:10ADD000A06300241FFE0A08241D0020D8F60A08DC
:10ADE0009DFB0A088CFB0A08A85200242DE9F04FAD
:10ADF000064685B008460B46FFF7DEFC044628B140
:10AE0000304605B0BDE8F04FFEF7C8BD03AA304993
:10AE10001846274656F0D8FBA0460546DFF8C090F6
:10AE2000DFF8C0A0DFF8C0B05DB92A4B3A46A1B246
:10AE3000D86F4EF00FFC68BB27493046FEF797FDF0
:10AE400028E0B8F1000F06D0B8F1010F25D0304648
:10AE5000FEF7A4FD1EE0284653F0D2FF4946024605
:10AE600001902846FCF762FB50B3019A51462846F0
:10AE7000FCF75CFB30B3019A59462846FCF756FBB9
:10AE800010B3019A28461549FCF750FBF0B1304643
:10AE9000FFF77AFB05B0BDE8F08FBB1E29463046B0
:10AEA0005A425A41FFF76EF8421C0446F2D003AAF8
:10AEB0000749002008F1010856F086FB0546B3E774
:10AEC0004746F4E70127F2E70227F0E70427EEE719
:10AED0001FFE0A08A8520024C9FB0A08C6FB0A087C
:10AEE000BDFB0A08C0FB0A08C3FB0A082DE9F743AB
:10AEF00080460846FFF760FC0B46054628B14046F1
:10AF0000FEF74CFD03B0BDE8F08301AA2D491846B9
:10AF10002F4656F059FB2E460446DFF8A8907CB920
:10AF2000022DECD1A7F57A73B3F57A7F21D94FF4CE
:10AF3000FA634FF47A7224494046FFF731FCE1E7A7
:10AF40004DB1012D10D001AA49460020013556F01F
:10AF50003BFB0446E3E7012221464046FFF712F897
:10AF6000431C0646EFD1CDE72046FCF7D3FB07464E
:10AF7000E9E7164DB8B2D5F8CC365B689847FF2E96
:10AF8000BCEEC00A124B0BD1F8EE407A95F8902532
:10AF9000A24212DC10EE101A0E48FDF711FFB1E7C5
:10AFA000F8EE407A03EB860310EE102A31460A4889
:10AFB000C3ED007AFDF704FFA4E70134E3EC017A66
:10AFC000E6E700BF1FFE0A08D7FC0A08241D002080
:10AFD0009C6C0024F4FB0A08E7FB0A08F8B5074656
:10AFE0000846FFF7E9FBC8B11F4BDE6A0136304661
:10AFF000344611F037FC0546F0B90134192CA8BFCE
:10B000000024204611F02EFC0546A8B9B442F4D124
:10B0100038461649BDE8F840FEF7A9BC0846FCF7DB
:10B0200079FB044611F01EFC054628B9214610485C
:10B03000BDE8F840FDF7C4BE0B4BDC6214F044F8E9
:10B040002A4621460B48FDF7BBFE182C09D80A48B2
:10B050000C2101FB040090F87C0BBDE8F84014F0D3
:10B0600069B80020F9E700BFB404002403FC0A0813
:10B0700017FC0A082DFC0A082C330A0838B50446C8
:10B08000114D0846FFF798FB68B1104B93F900107B
:10B090004B1C06D10E4B19790E48BDE83840FDF720
:10B0A0008FBEC9B2F8E70846FCF734FB032804D882
:10B0B000C0B2FDF773FA2946E3E7204603220649AA
:10B0C000BDE83840FEF753BC90FA0A08B4040024E7
:10B0D000A852002446FC0A0856FC0A0838B5044663
:10B0E000114D0846FFF768FB68B1104B93F901104A
:10B0F0004B1C06D10E4B59790E48BDE83840FDF780
:10B100005FBEC9B2F8E70846FCF704FB032804D881
:10B11000C0B215F00FFF2946E3E720460322064997
:10B12000BDE83840FEF723BC90FA0A08B4040024B6
:10B13000A852002442FC0A0851FC0A08444B2DE99D
:10B14000F74FDFF824A105461A7988468AF80020CF
:10B150005A7993F880308AF801200BB903F090FFF8
:10B1600000263C4CFBF722FCB1460D23394A4146F0
:10B17000734352F803B05846FCF7FCF9002841D05D
:10B18000B9F1000F01D0FDF779FD59463248FDF7BE
:10B19000D7FD002221462846FEF7DAFBFDF76EFDBB
:10B1A000237903F01803082B45D0102B48D02046F4
:10B1B000FDF715FE274A0D2303FB0623B3F809000C
:10B1C000FBF762FB0746D8B12046FBF776F9009003
:10B1D000D7E90221024401442046FBF727F978B958
:10B1E000594601901D48FDF7ABFD019AB968284604
:10B1F0001346009A0A442146FEF7B8FAFDF73EFDD1
:10B2000009F10109013640F265230D349E42ACD1AB
:10B210000020FFF720F9FF238AF800308AF8013078
:10B22000B9F1000F11D142460D49284603B0BDE8DF
:10B23000F04FFEF79CBB0B492846FFF71FFFB6E710
:10B2400008492846FFF74AFFB1E703B0BDE8F08F91
:10B25000A8520024C04C0A08F9F80A0871FC0A0830
:10B26000A5F60A0890FA0A08B40400242DE9F74F5D
:10B27000074608460E4653F0C3FD044620B1012898
:10B2800025D132782A2A22D1B24E00254FF00D0B5B
:10B29000DFF8E092B24640F26528AF48FDF706FDC0
:10B2A0000BFB05F3484601355AF80310FDF748FD3E
:10B2B000221E3146384618BF01220D36FEF748FBE4
:10B2C000FDF7DCFC4545EBD103B0BDE8F08F3D2137
:10B2D000304656F0BEFA002800F0368101460A4694
:10B2E00011F8014D202CFAD0921B0130814610F844
:10B2F000011B2029FAD05FFA82FA4FF00008DFF82C
:10B3000054B20D235246304603FB08F10BEB010407
:10B310005BF801100091FCF709F90546002857D1A8
:10B320000099084653F06CFD824551D1267906F00C
:10B33000E001402900F0CB800ED8002956D020290A
:10B3400000F09D8038468549FEF711FB204603B08A
:10B35000BDE8F04FFDF743BD602900F091808029E2
:10B36000F0D1484653F04CFDE3790546A679DB075A
:10B370000CD52046FBF79EFA0378014633B12A46E6
:10B38000484656F08CFA002840F0D880002D00F096
:10B39000D580AE42C0F0D2800D23204603FB08B317
:10B3A00093F805A0FBF786FA3246002156F04AF9D9
:10B3B000AA452CD82A466A49484656F070FA30B356
:10B3C0002046FBF777FA2A46494656F0C7F81EE0B2
:10B3D00008F1010840F26523984592D1324661494F
:10B3E000384603B0BDE8F04FFEF7C1BA06F00703D8
:10B3F000042B1CD10B460A224846FCF7E7F8D4F888
:10B400000530014683429DD32046FBF769FA0D23A0
:10B41000554803FB08F85BF80810FDF791FC002283
:10B420002146384603B0BDE8F04FFEF791BA052B30
:10B430000FD101230A224846FCF7C8F8D4F805309A
:10B4400001468342FFF67EAF5B4283423FF77AAF0D
:10B45000DAE74846FCF75EF9B4F80550B4F807108F
:10B4600016F0050FAAB28BB201D02AB20BB29042ED
:10B47000FFF668AF98423FF765AF0146C4E76579CC
:10B480003A4A002602EBC505B246334695F84427F2
:10B490000092009AB24202D9BAF1000F03D0002BF9
:10B4A0003FF450AFB3E7D5F8401751F8260060B12C
:10B4B00049460193FCF716F8019B30B94FF0010A99
:10B4C00031462046FBF70CFA53460136E1E706F019
:10B4D00007066379013E0093009BAB4297DD484627
:10B4E000814610F8013B202BFAD02046FBF7E2F909
:10B4F0008246042E04D8DFE806F0031010161F0061
:10B500004846FCF707F90AF8050048462C2156F092
:10B51000A0F9013500F10109DEE74846FCF7FAF829
:10B520002AF81500F1E700230A2200214846FCF71B
:10B530004DF84AF82500E8E70123F5E732460C49C3
:10B540003846FEF714FAFDE63146384603B0BDE84A
:10B55000F04FF3E5C04C0A0881FC0A08CFFC0A084A
:10B5600006340B08A5F60A08C4FC0A082C330A089E
:10B5700094FC0A08F9F80A082DE9F04F914689B0C1
:10B580000C461A46002180464D46FEF759FF00271B
:10B590000646DFF8E0B0B9F1000F69D0294606226F
:10B5A000204656F025F800283246404613BF0121B8
:10B5B00000214FF0010A4FF0000AFEF741FF064656
:10B5C000287814F0E7FF079010B3687914F0E2FFD1
:10B5D000079B4FF461714FF0190C5B79EA78079380
:10B5E000AB781CFB021295F801E01CFB03132979D0
:10B5F00000B14079CDF804E0CDE90232079B5A460C
:10B60000CDE90410009351463B464046FDF780FBD0
:10B61000207814F0BFFF079010B3607914F0BAFFE0
:10B62000079B4FF461714FF0190C5B79E278079337
:10B63000A3781CFB021294F801E01CFB0313217990
:10B6400000B14079CDF804E0CDE90232079B5A46BB
:10B65000CDE90410009351463B464046FDF712FBEE
:10B66000013706340635142F95D109B0BDE8F08FA7
:10B67000CA46CDE7DDFC0A082DE9F041064686B052
:10B6800008460F46FFF798F8054638B100235C4995
:10B6900001201A4606B0BDE8F0416DE70846FCF708
:10B6A00039F81328044600F3A28006268DF81750B7
:10B6B000544D4643781CFBF77DF8074670B1FCF704
:10B6C00029F8C0B214F07CFF40B1AB19027983F8BD
:10B6D0003C269DF8173001338DF817303846FBF7BC
:10B6E00069F8074668B1FCF715F80D2809D8062354
:10B6F00003FB045383F83D069DF8173001338DF8A2
:10B700001730DFF8FC80B11C0DF1170238464144B8
:10B71000FCF704F8FBF74EF8074668B1FBF7FAFFB1
:10B72000012809D8062303FB045383F840069DF83B
:10B73000173001338DF817303846FBF73BF880B1EE
:10B74000FBF7E8FFC0B214F03BFF50B106230279CB
:10B7500003FB045383F841269DF8173001338DF81D
:10B7600017309DF817200623042A2FD103FB04531A
:10B770000022A3F840261FF031FF06234FF4617624
:10B7800003FB045595F83C0614F004FF95F83F269A
:10B7900095F83E761923804695F8410613FB076716
:10B7A00013FB026614F0F6FE4379214698F8052053
:10B7B000039395F8403614480097CDE9016395F856
:10B7C0003D36FDF7FDFA06B0BDE8F081052A05D14A
:10B7D00003FB0453002283F84126CCE7062ACAD093
:10B7E000002308EB060248F806309380C3E71323D2
:10B7F0002A460649304606B0BDE8F041FEF7D0BF04
:10B80000E4580024A8520024DDFC0A08F6FC0A08CB
:10B810002DE9F04F174689B01A460C4600218146A3
:10B820003D46FEF70DFE3A4E07F190038046DFF8E5
:10B83000E8B0079394F904100023364A92F90800FF
:10B84000884260D001330C320C2BF7D10C35079BAA
:10B850000C349D42EED109B0BDE8F08F29460C2290
:10B86000204655F0C5FE00284246484613BF012138
:10B8700000214FF0010A4FF0000AFEF7E1FDEA79DE
:10B8800095F90430804606EB820251464846D2F8CC
:10B89000AC2904922A7A06EB8202D2F8AC290392F0
:10B8A000AA7906EB8202D2F8AC2902926A7906EBF9
:10B8B0008202D2F8AC2901922A6800925A46FDF71A
:10B8C00027FAE279514694F90430484606EB8202A1
:10B8D000D2F8AC290492227A06EB8202D2F8AC2983
:10B8E0000392A27906EB8202D2F8AC290292627925
:10B8F00006EB8202D2F8AC290192226800925A46E5
:10B90000FDF7C0F9A2E7002FA8D1BA46D9E700BFDA
:10B910002C330A08F8570024FCFC0A082DE9F043F0
:10B9200080468BB00846FEF747FF38B100234D49EB
:10B9300001201A460BB0BDE8F04369E7CDE90700E6
:10B94000099008464D1CFBF7E5FE44B2204611F075
:10B9500069F90646002843D08DF820400124284686
:10B96000FAF728FF054638B1013400230A22E4B271
:10B970001946FBF72BFE07900027DFF8F0902846CA
:10B98000FAF718FF054618B3FBF7C4FE3649002244
:10B9900051F804CBD3B2604503D00132102AF7D15D
:10B9A000002309EB8302D2F8AC29904210D1022F78
:10B9B0001DD0032F20D05A1E012FD2B212D00B2A35
:10B9C00003D88DF821300134E4B20137042FD6D1E9
:10B9D000052C17D840460BB0BDE8F043FDF7DEBF9D
:10B9E0000446BCE7042AF0D88DF82230EBE7052B9B
:10B9F000EBD88DF82430E6E79A1E0D2AE5D88DF8AD
:10BA00002330E0E707AB9DF8232003CB30601868B4
:10BA1000164B7160002103EB8202B0600846D2F839
:10BA2000AC2904929DF8242003EB8202D2F8AC29C1
:10BA300003929DF8222003EB8202D2F8AC290292F5
:10BA40009DF8212003EB8203094AD3F8AC39019316
:10BA5000079B00939DF92030FDF714F90BB0BDE86A
:10BA6000F08300BF10570024D83C0A082C330A0882
:10BA7000FCFC0A082DE9F04F8BB00C46002107466C
:10BA800008921A46FEF7DCFC0026089D4FF01909C3
:10BA90004FF46178DFF8A4B00990089B002B49D0DF
:10BAA00029460A22204655F0A3FD0028099A384667
:10BAB00013BF012100214FF0010A4FF0000AFEF7E9
:10BAC000BFFC2A890990334606925146EA883846D7
:10BAD00005922A790492EA780392AA7819FB0282E5
:10BAE00002926A7819FB028201922A7800925A46E1
:10BAF000FDF70EF922893346013651460692384643
:10BB0000E2880A35059222790492E2780392A278BB
:10BB100019FB02820292627819FB0282019214F8E8
:10BB20000A2B00925A46FDF7ADF81E2EB5D10BB088
:10BB3000BDE8F08FDDF820A0DCE700BF19FD0A08A2
:10BB40002DE9F04380468BB008460F46FEF734FEE1
:10BB5000044638B10023654901201A460BB0BDE800
:10BB6000F04387E70846FBF7D5FD1D28054600F39F
:10BB7000B3800A268DF827404643781CFAF71AFE50
:10BB8000044630B1FBF7C6FD9DF8273001338DF830
:10BB900027302046564CFAF70DFE074668B1FBF7F2
:10BBA000B9FD0D2809D80A2303FB054383F81C09B6
:10BBB0009DF8273001338DF82730DFF83091711C64
:10BBC0000DF1270238464944FBF7A8FDFAF7F2FDCC
:10BBD000074668B1FBF79EFD222809D80A2303FB1C
:10BBE000054383F81F099DF8273001338DF827306E
:10BBF0003846FAF7DFFD074668B1FBF78BFD0D28E5
:10BC000009D80A2303FB054383F820099DF8273050
:10BC100001338DF827309DF82730062B0CD00023F8
:10BC200009EB0602404649F8063053601381FDF7E0
:10BC3000B5FE0BB0BDE8F0830A260023384606FBAC
:10BC40000546A6F82239A6F82439FAF7B3FD0746C7
:10BC500040B1FBF75FFD9DF82730A6F822090133BC
:10BC60008DF827303846FAF7A5FD58B1FBF752FD9D
:10BC70000A2303FB0543A3F824099DF82730013369
:10BC80008DF827301B4B4FF0FF324FF461705A6034
:10BC90000A2202FB0542B2F824390693B2F822398F
:10BCA000059392F82039049392F81F3903931923CE
:10BCB00092F81E1913FB0101029192F81D1913FB52
:10BCC000010300210193084692F81C390A4A0093A7
:10BCD0002B46FCF7D7FFACE71D2322460749404619
:10BCE0000BB0BDE8F043FEF75BBD00BFBC6C0024A9
:10BCF000A0630024B404002419FD0A08F6FC0A0815
:10BD00002DE9F04F804691461F460C4616464FF0EF
:10BD1000000BDFF820A12DED088B95B094ED008A83
:10BD2000B5EE408AF1EE10FA7DD0D4ED019A94ED93
:10BD3000029AD4ED038AB9F1000F49D0D6ED00BACA
:10BD400096ED01BAB4EE6B8AD6ED02AA96ED03AA7F
:10BD5000F1EE10FA6CD1F4EE4B9AF1EE10FA67D1D5
:10BD6000B4EE6A9AF1EE10FA62D1F4EE4A8AF1EE7C
:10BD700010FA0CBF012100213A460D46404681F0E1
:10BD80000101FEF75DFBB0EE6B0A074611A8FAF75A
:10BD90008BFCB0EE4B0A07900EA8FAF785FCB0EECC
:10BDA0006A0A06900BA8FAF77FFCB0EE4A0A0590E3
:10BDB00008A8FAF779FC0599069A079B0390404674
:10BDC000029129460192524600935B46FCF7A0FF80
:10BDD000B0EE480A11A8FAF767FCB0EE690A05460A
:10BDE0000EA8FAF761FCB0EE490A06900BA8FAF724
:10BDF0005BFCB0EE680A059008A8FAF755FC069BB4
:10BE0000059A0021039040460292524610341036A3
:10BE1000CDE900535B460BF1010BFCF733FFBBF19F
:10BE2000080F7FF47BAF15B0BDEC088BBDE8F08F39
:10BE30000021A1E73CFD0A082DE9F74F07460D4612
:10BE4000DFF894A1DFF894B12846FEF7B5FC06466A
:10BE500038B10023594901201A4603B0BDE8F04F1C
:10BE60004EE7052251462846FBF760FB60B9534B6D
:10BE700000221A601A611A621A631A641A651A6635
:10BE80001A6703B0BDE8F08F04224D492846FBF73E
:10BE90004DFB04462846002C44D1FAF78BFC804623
:10BEA0000028EED052F0ACFF464BC2B253F8049BD0
:10BEB000B9F1000F07D12A464349384603B0BDE81F
:10BEC000F04FFDF754BD494640460134CDE900230B
:10BED000FBF72CFB0646DDE900230028E6D1374AB4
:10BEE000034600211546013342F8101B082BFAD1F6
:10BEF0000BEBC404D4F8D8C0BCF1000F03D094F805
:10BF0000D4E0764505DB49463048314DFCF758FF13
:10BF10009AE70CEB061305EB061401360FCB84E809
:10BF20000F00EEE7FBF7F6FB072804463DD828464E
:10BF3000FAF740FC064658B3FAF79CF91F4B012567
:10BF400003EB041383ED000A3046FAF733FC064690
:10BF500038B1FAF78FF9194B013503EB041383ED70
:10BF6000010A3046FAF726FC064638B1FAF782F99C
:10BF7000124B013503EB041383ED020A3046FAF746
:10BF800019FC38B9384603B0BDE8F04FFDF706BDDF
:10BF90000546D9E7FAF76EF90848032D00EB0414BB
:10BFA00084ED030A3FF455AFECE707233246094915
:10BFB000384603B0BDE8F04FFEF7F2BB145C002436
:10BFC00050FD0A08343E0A08A5F60A0855FD0A087D
:10BFD00090FA0A08F6FC0A08F2F90A082C330A0853
:10BFE0002DE9F74F92460C461A46002181465646E7
:10BFF000FEF726FA00258046DFF864B0BAF1000F9C
:10C000002CD031460422204655F0F2FA0028424650
:10C01000484613BF0121002101270027FEF710FA2F
:10C02000738880465A46019339463AF82530484687
:10C0300000932B46FCF76CFE63885A463946484607
:10C040000193043634F8043B00932B460135FCF78A
:10C0500019FE042DD2D103B0BDE8F08F5746EBE7AF
:10C060005FFD0A082DE9F34105460846FEF7A4FBEB
:10C070000C46074638B10023334901201A4602B066
:10C08000BDE8F041ACE731492046FBF72BFA034607
:10C0900068B92D4A4FF47A704FF4FA610133108079
:10C0A00051800432042BF9D102B0BDE8F081204662
:10C0B000FBF730FB0328064641D82046FAF77AFB07
:10C0C000074670B1FBF726FB4FF0010804463846DF
:10C0D000FAF770FB48B9284602B0BDE8F041FDF719
:10C0E0005DBC40F2EE248046F1E7FBF713FBB8F1AC
:10C0F000000FF0D0A4F2EE2240F2DC539A4203D8B3
:10C10000A0F2EE229A420AD940F6CA0340F2EE2289
:10C110000F49284602B0BDE8F041FEF741BB0D4B88
:10C1200000210D4A03EB8603A3F8484AA3F84A0A04
:10C130003346CDE900400846FCF7A4FDB4E70323ED
:10C140003A460649E5E700BFE86D0024F2F90A081F
:10C1500070FD0A08A06300245FFD0A08D2F90A08EE
:10C160002DE9F04F8FB08946174600211A46064642
:10C170000024FEF765F90DF1240B0546DFF86CA0ED
:10C1800059F82430594602A8029349F08FFF57B35B
:10C1900057F824303046029A039393422A4613BF3D
:10C1A000012100214FF001084FF00008FEF748F987
:10C1B00004A9054603A849F079FF04A9234652467D
:10C1C000009130464146FCF7A3FD23460134524618
:10C1D00041463046CDF800B0FCF754FD202CCFD1BD
:10C1E0000FB0BDE8F08FB846EFE700BF7EFD0A084C
:10C1F000F0B5074689B008460E46FEF7DDFA05465B
:10C2000038B10023194901201A4609B0BDE8F040B1
:10C21000A6E70846FBF77EFA1F2804461DD83046DD
:10C22000FAF7C8FA0146204637F082FB78B103AE30
:10C230000E48314600EB840049F038FF23460C4A93
:10C24000294628460096FCF71DFD09B0F0BD38468A
:10C2500009B0BDE8F040FEF797B91F232A4605490B
:10C26000384609B0BDE8F040FEF79ABAF86D0024F0
:10C270007EFD0A08F6FC0A082DE9F04F924685B0CB
:10C280000C461A46002181465546FEF7D9F800268D
:10C290008046DFF86CB0BAF1000F2FD02946042297
:10C2A000204655F0A5F900284246484613BF012113
:10C2B000002101270027FEF7C3F8EB7880465A4695
:10C2C00002933946AB78484601932B880093334656
:10C2D000FCF71EFDE3785A4639464846029304357A
:10C2E000A378019334F8043B009333460136FCF7FE
:10C2F000C9FC102ECFD105B0BDE8F08F5746E9E755
:10C3000088FD0A08F0B5074685B008460E46FEF7D8
:10C3100053FA054638B100231C4901201A4605B0DE
:10C32000BDE8F040A8E70846FBF7F4F90F280446FB
:10C3300023DC3046FAF73EFA0146204637F070FA21
:10C34000A8B104F12002124B2946284603EB8203D0
:10C3500093F85B2A029293F85A2A0192B3F8583A5A
:10C360000C4A00932346FCF78DFC05B0F0BD38461F
:10C3700005B0BDE8F040FEF707B90F232A4606498D
:10C38000384605B0BDE8F040FEF70ABA786E0024E2
:10C39000A063002488FD0A08F6FC0A082DE9F04F86
:10C3A00087B014461A46054603910021FEF748F867
:10C3B0004FF000080646DFF820B106234FF00009D1
:10C3C00003FB08F7C037039BDB5D0493002C7FD091
:10C3D000E35D2846049A05939A42324613BF012131
:10C3E00000214FF0010A4FF0000AFEF729F8059BE3
:10C3F00006465A4651462846CDE900934346FCF787
:10C4000087FC049B5A46514628460137CDE90093E4
:10C4100009F101094346FCF735FCB9F1060FD2D109
:10C4200008F10108B8F1060FC7D1E427DFF8A8B07A
:10C43000039BA7F1E40913F807A0002C4AD0E35DA1
:10C44000324628469A45049313BF012100214FF03C
:10C4500001084FF00008FDF7F3FF049B06465A461B
:10C4600041462846CDE900930623FCF751FC0137ED
:10C470000623194A41462846CDE9009AFCF702FCFA
:10C48000EF2FD5D1039B93F8EF70ACB194F8EF8008
:10C4900032462846474513BF0121002101240024CC
:10C4A000FDF7CEFF00230C4A2146009328460723C0
:10C4B000CDF80480FCF72CFC0023074A21462846CF
:10C4C000009307230197FCF7DDFB07B0BDE8F08F71
:10C4D000A24696E7A046CAE79AFD0A08F0B50546C7
:10C4E00087B008460B46FEF767F9044638B10023CB
:10C4F0001C4901201A4607B0BDE8F0404EE703AEE4
:10C50000194F02AA1849184655F05EF8B8B1032C25
:10C5100004D12846FDF742FA07B0F0BDFBF7FAF860
:10C5200002AA46F8040B39460020013455F04CF8B5
:10C53000ECE7324621460D48FCF742FCECE7032CC1
:10C54000E7D1059BDDE903461A4601933146E0B287
:10C5500037F0B0F9019B0028EBD12846FEF714F81C
:10C56000DAE700BFF86D00241FFE0A089AFD0A08EA
:10C570002DE9F04F0F46164689B04FF00009B84636
:10C580003446DFF83CB11A4600210546FDF758FF56
:10C590000790002E7CD021460C22404655F028F80A
:10C5A0000028079A284613BF012100214FF0010AF5
:10C5B0004FF0000AFDF744FF94F90B2007904B461B
:10C5C0000492514694F90A2028460392B4F90820AF
:10C5D0000292B4F906200192B4F9042000925A465E
:10C5E000FCF796FB98F90B204B4609F101095146DF
:10C5F0000492284698F90A200C3408F10C0803929A
:10C6000038F9042C029238F9062C019238F9082CDA
:10C6100000925A46FCF736FBB9F1080FB9D1002455
:10C62000DFF8A0900C2303FB04FA9EB34FF0000840
:10C63000012356F80A2003FA08FB57F80A30534042
:10C640003BEA030314BF0121002112EA0B0F08D0BB
:10C6500023464A462846CDF800800791FCF758FB50
:10C66000079957F80A301BEA030F06D023464A46BB
:10C670002846CDF80080FCF705FB08F10108B8F169
:10C680000E0FD5D10134082CCCD109B0BDE8F08F04
:10C69000B246A7E7B046012357F80A2003FA08F389
:10C6A000134207D023464A4601212846CDF8008090
:10C6B000FCF7E8FA08F10108B8F10E0FEBD1E1E759
:10C6C000AEFD0A08C6FD0A08F0B506468BB008465E
:10C6D0000D46FEF771F8044620B300233F490120C0
:10C6E0001A460BB0BDE8F04042E72D2B03D0A3F172
:10C6F0003002092A4BD8052C05DD30460BB0BDE8C9
:10C70000F040FDF74BB92846FBF704F80AAB621C72
:10C7100003EB440424F80C0C15F8013F303B092BC3
:10C72000FAD914462B78002BDFD1062CE5D1BDF8C1
:10C730001C20BDF91C30072ADFD8BDF91E10A1F559
:10C74000FA7292B2B2F5FA6F1AD8BDF92040A4F588
:10C75000FA7292B2B2F5FA6F12D8BDF92270B942EC
:10C760000EDCBC420CDBA1420ADCBDF924C00CF19A
:10C77000640292B2C82A03D8BDF92650112D11DDEA
:10C78000174930460BB0BDE8F040FDF7F0B8202B5C
:10C7900002D101352246C4E730460BB0BDE8F04077
:10C7A000FDF7F2BE0C200F4A6DB200FB0322A2F887
:10C7B0004C1BA2F84E4BA2F8507B82F852CB82F869
:10C7C000535B00910021084A0846CDE903C5CDE935
:10C7D0000147FCF757FA0BB0F0BD00BFE86E00242C
:10C7E000DBFD0A08A0630024AEFD0A082DE9F04F26
:10C7F00089468DB0164600211A4607460024FDF7EB
:10C800001FFEDFF8DCA00546C4EBC40309EB0302FE
:10C8100059F80300918840F3074892790890ADF8E1
:10C8200024108DF82620B8F1000F53D0002E54D0DC
:10C83000F218F0589188937907220A9008A8ADF869
:10C840002C100AA98DF82E3054F0D2FE00282A466A
:10C85000384613BF012100214FF0010B4FF0000BB0
:10C86000FDF7EEFD9DF82E300546524606935946DB
:10C870009DF92D30384605939DF92C3004939DF891
:10C880002B3003939DF92A3002939DF829300193B0
:10C890009DF8283000932346FCF73AFA9DF826309D
:10C8A00052465946384606939DF9253005939DF921
:10C8B000243004939DF82330CDE902839DF8213084
:10C8C00001939DF82030009323460134FCF7DAF9F8
:10C8D000102C99D10DB0BDE8F08FB346DEE700BF54
:10C8E000F1FD0A082DE9F04F06468DB00D469C4F2C
:10C8F000DFF8A082DFF8A092284652F081FA0346C2
:10C9000030B90246974901200DB0BDE8F04F6DE700
:10C91000052239462846FAF709FE0446C8B9924D61
:10C920000146702205F6A83054F08CFEC5F8484B3D
:10C93000C5F8544BC5F8604BC5F86C4BC5F8784B3F
:10C94000C5F8844BC5F8904BC5F89C4B0DB0BDE8BD
:10C95000F08F042241462846FAF7E8FD044638BB2A
:10C960002846F9F727FF82460028EFD052F048FA10
:10C97000DFF828B202465BF8041B39B92A467B4926
:10C9800030460DB0BDE8F04FFCF7F1BF5046CDE9A1
:10C990000012FAF7CBFD019A40B92046744D27F0FA
:10C9A00091F900994846FCF70BFAA5E70134E2E754
:10C9B000072270492846FAF7B9FD074600287AD1C0
:10C9C0002021284654F045FF044670BB6A4D6B4851
:10C9D000FCF7B6F9214601342846FCF7B1F90E2CD4
:10C9E000F8D10024DFF8B891654FFCF747F9DFF87C
:10C9F000B4810C260025DFF8B0A1214666434846E5
:10CA0000FCF79EF90123F2595E48AB400135134211
:10CA100014BF41465146FCF793F90E2DF2D1013473
:10CA2000FCF72CF9082CE4D190E704AC564D03AA8E
:10CA3000554954F0C9FD002848D0022F11D1049A5D
:10CA4000072A07D805990D2904D80378722B13D02B
:10CA50006E2B22D0082300224C493046FDF7A0FE61
:10CA600074E7FAF757FE03AA44F8040B294600209E
:10CA7000013754F0A9FDDEE70C203B4B00FB0233ED
:10CA8000012000FA01F1D3F8480B0843C3F8480B22
:10CA900038493046FFF726FF58E7334B0C2000FBA0
:10CAA0000233012202FA01F1D3F8482B22EA0102F3
:10CAB000C3F8482BECE72846002404AD324F03AA04
:10CAC000314954F081FDA8B1082C03D13046FCF760
:10CAD00065FF3BE7FAF71EFE03AA45F8040B39464B
:10CAE0000020013454F070FDEDE729493046FCF791
:10CAF0003EFF2BE7082CE9D1049B0F2BF5D8DDF87E
:10CB000014E0BEF1070FF0D8DDF818C0BCF10D0F2E
:10CB1000EBD8079F07F16402C82AE6D8089DFF2DCD
:10CB2000E3D809986428E0D80A996429DDD88842B6
:10CB3000DBDA0B9C032CD8D8C3EBC3020A4B13449B
:10CB400083F8AD1B83F8A8EB094983F8A9CB83F8D8
:10CB5000AA7B83F8AB5B83F8AC0B83F8AE4B98E70A
:10CB6000F2F90A08486F0024A0630024A5F60A0819
:10CB700090FA0A080EFE0A0816FE0A089A030B0825
:10CB8000E86E00241BFE0A081FFE0A0821FE0A08A0
:10CB9000DBFD0A0850FD0A0855FD0A08343E0A0864
:10CBA000343B0B08D9FD0A082C060B082DE9F04F81
:10CBB00089B000260C46002107921A460746B24665
:10CBC000FDF73EFC4FF01909079D4FF46178DFF83F
:10CBD00094B00690079B3BB329460622204654F0AA
:10CBE00007FD0028069A384613BF012100214FF0A7
:10CBF000010A4FF0000AFDF723FC6A7906903346DC
:10CC000019FB02825146384605922A7919FB0282A5
:10CC10000492EA780392AA7802926A7801922A78BA
:10CC200000925A46FCF774F8627933460136514651
:10CC300019FB0282384606350592227919FB0282D9
:10CC40000492E2780392A27802926278019214F838
:10CC5000062B00925A46FCF715F80A2EBAD109B0F5
:10CC6000BDE8F08F27FE0A082DE9F04F80468BB013
:10CC700008468946FDF7A0FD074638B1002355490F
:10CC800001201A460BB0BDE8F04F8FE7524C084622
:10CC900094F84E3894F864B794F865A70793FAF7B8
:10CCA00039FD0928054600F38B8006268DF827708C
:10CCB000464309F10100F9F77DFD074658B1FAF73F
:10CCC00029FD0D2807D8A31983F8800B9DF827307C
:10CCD00001338DF827303846F9F76CFD074668B107
:10CCE000FAF718FD834509D3062303FB054383F8B0
:10CCF000810B9DF8273001338DF827303846F9F73E
:10CD000059FD074668B1FAF705FD504509D80623D5
:10CD100003FB054383F8820B9DF8273001338DF820
:10CD200027303846F9F746FD074670B1FAF7F2FCAE
:10CD3000079B834209D3062303FB054383F8830B38
:10CD40009DF8273001338DF82730DFF88890311DAA
:10CD50000DF1270238464944FAF7E0FC9DF82730E8
:10CD6000062B0BD0002309EB0602404649F806309B
:10CD70009380FCF713FE0BB0BDE8F08F03FB054476
:10CD80004FF46171192394F8852B13FB021205925D
:10CD900094F8842B13FB02130021104A04930846D5
:10CDA00094F8833B039394F8823B029394F8813B7D
:10CDB000019394F8803B00932B46FBF763FFDAE77F
:10CDC00009233A46064940460BB0BDE8F04FFDF74F
:10CDD000E7BC00BF285E0024A852002427FE0A08F2
:10CDE000F6FC0A082DE9F04F144689B00F461A46A2
:10CDF00000210646FDF724FB0546002C00F0D580F7
:10CE000022783B789A42024630460DBF4FF0010827
:10CE10004FF0000801210021FDF712FB23780546A1
:10CE2000994A41463046FBF773FF3B784146964AA4
:10CE30003046FBF727FF002C00F0B98062783046BF
:10CE40007B789A422A460DBF4FF001084FF0000848
:10CE500001210021FDF7F4FA637805468B4A41462B
:10CE60003046FBF755FF7B784146884A3046FBF752
:10CE700009FF07F1CA0304F1CA0B4FF0020904933A
:10CE80004FF0000A822305933B78534500F39180CD
:10CE9000002C00F0F28097F8EA30304694F8EA204F
:10CEA0009A422A460DBF4FF001084FF000080121B9
:10CEB0000021FDF7C5FA94F8EA300546744A414668
:10CEC0003046FBF725FF97F8EA304146704A304676
:10CED00007F1EC09FBF7D6FE002C00F0D08004F13E
:10CEE000EC034A4604F1FC014FF001089A4633F87E
:10CEF00002CB32F8020B844518BF4FF000088B427A
:10CF0000F5D188F001012A463046C9B2FDF798FAFA
:10CF1000082105465046FAF757FA5E4A034641464D
:10CF20003046FBF7F5FE97F8EA104846FAF74CFA58
:10CF3000584A034641463046FBF7A4FE002C00F059
:10CF4000A0804FF0FC094FF0010807EB090104EB4A
:10CF50000900FAF7C7FA09F10409002818BF4FF0D1
:10CF60000008B9F58E7FF0D188F001012A463046DD
:10CF7000C9B2FDF765FA082104F1FC00F9F74EFC8F
:10CF8000454A034641463046FBF7C2FE97F8EA1091
:10CF900007F1FC00F9F742FC3F4A034641463046A0
:10CFA00009B0BDE8F04FFBF76DBEA0463DE7A046D7
:10CFB00059E7059B3B440693002C5CD0059B0698E3
:10CFC000234419460793FAF78DFA049B1A789BF8C5
:10CFD00000309A424CD1B0FA80F84FEA58184B46CC
:10CFE00009F11002F85AE15A0233884218BF4FF093
:10CFF00000089342F6D188F001012A463046C9B2B2
:10D00000FDF71EFA627804EB090105469BF818004B
:10D01000FAF7ACF902909BF8003041461F4A3046BF
:10D020000193079B00930AF10103FBF771FE049B38
:10D0300007EB09017A780AF1010A187E0BF1010B5E
:10D040000793FAF793F9079B4146049A09F11009EF
:10D05000029030461B7801320193069B04920093A4
:10D0600053460E4AFBF70EFE059B093305930BE76B
:10D070004FF00008B3E7A046D9E7A04623E7A04653
:10D0800051E7A04682E700BF40FE0A0852FE0A08A8
:10D0900080FE0A0898FE0A08AFFE0A0867FE0A0822
:10D0A0002DE9F04F8FB004460846B04902AA54F06B
:10D0B0008BFA064640B903460246AD494120FFF7C8
:10D0C00091FE0FB0BDE8F08FAA49FAF70BFA0746B8
:10D0D00020BB02AAA54954F077FAFAF71BFB0828EF
:10D0E000054606D908233A46A3492046FDF758FBD2
:10D0F000E7E7A24C94F86437834202DC84F8645773
:10D10000DFE7064604F264773146384630F01CFA11
:10D11000013694F86437B342F6DCEFE798493046BD
:10D12000FAF7E0F90546E0B902AA904954F04CFA42
:10D13000FAF7F0FA0828064603D908232A46914947
:10D14000D3E78E4C94F86537834202DC84F8656738
:10D15000B7E728460135314648F080FF082DF8D161
:10D16000F4E789493046FAF7BDF9074600BB02AA41
:10D170007E4954F029FA0028A3D0FAF7CBFA082800
:10D18000054603D908233A468049AEE77B4C94F81C
:10D190004E38834209DD014604F2647030F01EFA15
:10D1A000294604F2647030F027FA84F84E5888E774
:10D1B00077493046FAF796F9054618BB06AE6F4B2D
:10D1C000DFF8A8910146B0461022304693F84E7819
:10D1D00054F038FABD4202AA80F20E81494600207E
:10D1E00054F0F2F910B93A466A490EE1FAF792FAA8
:10D1F000013528F8020BEDE7674C96E80F0084E84C
:10D200000F005EE765493046FAF76CF905460028DD
:10D210003BD15A4B0DF11808074693F84E984646F5
:10D220004F4502AA51494FF0000080F2F28054F0BD
:10D23000CBF9014610B94A465949E6E0B2464FF0EB
:10D24000000B0322304654F03EFB304651F0D8FD2F
:10D25000584502D801370436E2E79AF800000BF18E
:10D26000010BFAF739F90AF8010BEEE74A464D4986
:10D27000CBE0414620460135043408F1040803227E
:10D2800030F04CF9AF42F4D11BE747493046FAF78A
:10D2900029F90546002840F0AC80384F02AA3349EE
:10D2A00097F8648754F090F900283FF40AAFFAF732
:10D2B00031FA461E01D4B04503DC434601223B4906
:10D2C00013E72A4902AA002054F07EF901460028FB
:10D2D0003FF4F7AE4FF000080DF10C09082203A847
:10D2E0008DF81480CDE9038854F0EDFA03A851F0CD
:10D2F00087FD40451CD802AA1C49002054F064F95F
:10D3000000283FF4DEAE90F800A04FF0000897F838
:10D310006597DFF8A8B04D4502AA14494FF0000008
:10D320007EDA54F051F9024658B94A4620496CE079
:10D3300099F8000008F10108FAF7CEF809F8010B96
:10D34000D4E7002D40D11378303B092B3CD9194943
:10D350000192FAF7C7F8019A90B310465946FAF7C6
:10D36000C1F8019A002838D013494EE01FFE0A0880
:10D370000C5A0024C6FE0A08CCFE0A08A852002453
:10D38000D7FE0A08E0FE0A08EEFE0A08FAFE0A08BE
:10D390000CFF0A08FBFF0A08F85A002436FF0A08A7
:10D3A0001B000B0842FF0A0860FF0A0865FF0A0815
:10D3B0003B000B08C2EE0A0878FF0A0871FF0A0852
:10D3C0004FF001084FF0FF3510460192FAF7A2F92D
:10D3D0000028019A03DA214917E0A846F2E70EABCC
:10D3E00003EB4503013523F8200C94E74A461C491A
:10D3F0000BE032461B4908E01B49002054F0E4F8DA
:10D4000000283FF4F9AE3A4618492046FCF7AFFA37
:10D4100057E654F0D9F800287FF428AF144C31E7D0
:10D4200054F0D2F80028E1D106EBC600114C0822D6
:10D4300003A982303744204430F070F85046FAF7A0
:10D440004BF887F82E0804EB061006A96A00023094
:10D4500054F084F887F8468833E600BFADFF0A0829
:10D46000C2FF0A08E5FF0A081FFE0A0818FF0A089B
:10D47000085B00240C5A00242DE9F04F0F4691461A
:10D4800089B0002187EA09099846139A06460025C3
:10D49000FCF7D6FF6FEA09030446DFF88090069395
:10D4A00028460FF0CDF9129B184230D0069BDFF8CA
:10D4B00070B0034014BF4FF0010A4FF0000A04930C
:10D4C00010EA0703284614BF4A465A4605930792B6
:10D4D0000FF0C8F94346079A514603900090304632
:10D4E000FBF716FC049B22463046B3FA83F1490948
:10D4F000FCF7A6FF039B059A04460093514643465A
:10D50000002A14BF5A464A463046FBF7BBFB01359A
:10D51000182DC5D109B0BDE8F08F00BF4AFD0A083B
:10D5200060000B0837B504460846019151F068FCCD
:10D530000199054602462046F9F7F8FF70B9625D89
:10D540001046F9F7B3FF00B932B901352C44204633
:10D5500001340378202BFAD003B030BD0020FBE764
:10D560000329F0B5054685B00C46164614D80B4F76
:10D570003970FBF783FB0A492846FDF77FFD2246F9
:10D58000084901A8F9F798FE01AB32460821284660
:10D59000FCF784FFFF233B7005B0F0BDB40400240A
:10D5A00090FA0A0846FC0A080329F0B5054685B03A
:10D5B0000C46164614D80B4F7970FBF75FFB0A49EF
:10D5C0002846FDF78BFD224608496846F9F774FEA8
:10D5D0006B46324610212846FCF760FFFF237B7024
:10D5E00005B0F0BDB404002490FA0A0842FC0A0811
:10D5F00010B5114B86B0114904460493104B1148E5
:10D600000393114B114A0293114B0193114B009359
:10D61000114BFBF795FBFBF731FB10491048FBF76B
:10D62000CFFB3CB10F4A1049104806B0BDE810408E
:10D63000FBF7C6BB06B010BDA7000B0871000B08B6
:10D64000AC000B087C000B08B6000B0867000B0849
:10D65000BF000B08E0F10A08B3520024CB000B080E
:10D66000D3000B0868AC0A0860AC0A08E4000B0899
:10D670000120BDE7224BB0F5FA6F1A680346A8BF38
:10D680004FF4FA63B3F57A7FB8BF4FF47A73D204DC
:10D6900016D540F2DC52904215D040F2DB5207EE34
:10D6A000903A9042F8EE677A1FD8DFED166A9FED48
:10D6B000167A77EEE67A9FED150AA7EE870A70478D
:10D6C000B0F57A7F02D89FED120A704707EE903AC4
:10D6D000DFED106A9FED107AF8EE677A9FED0F0A82
:10D6E00077EEE67AA7EE870A7047DFED0D6A9FEDC9
:10D6F0000D7A77EEE67A9FED0C0AA7EE870A70475F
:10D700008C58002400007A44D62000C000E08244F7
:10D710000000000000407A446610004000004042D3
:10D7200000A0BB44D62000400000834410B58446CE
:10D730004FEA810E102312F4004F4FEA420214BF49
:10D740000E240724013B92B2CCF80040F444F2D1FD
:10D7500000EB81128C010351122042F8213010BDE0
:10D7600010B584464FEA810E0424130B013C4FEAA6
:10D77000021203EB430392B203F11803CCF800301A
:10D78000F444F2D100EB01130A018450062043F85F
:10D79000214010BD704700BF704700BF034B00EB36
:10D7A000400003EBC000407C704700BFB810002071
:10D7B0002DE9FF471E46C368044689469246BDF8D8
:10D7C0003070DDF834804BB3CBB20D2B24D81A4A1D
:10D7D000D556BAF1FF3F23D023683146174A384661
:10D7E000CDE9005AC04752465FFA89F12079F4F733
:10D7F00053F9024600B10288D3B23146384603934A
:10D80000C2F30323120B02932368CDE900520C4AA2
:10D81000C04704B0BDE8F0870025DAE74D1CD8E723
:10D820007B06F6D423683146064A3846C4460C9532
:10D8300004B0BDE8F047604744AC0A0811010B088A
:10D840001E010B0842010B08002353224370027093
:10D850008370C370704700BF704700BF704700BF40
:10D860000020704701207047704700BF704700BF1D
:10D87000704700BF704700BF9FED010A704700BFAF
:10D88000000000000020704703681B6918470B4B1D
:10D89000002130B593F9002001315D780433092A65
:10D8A000C8BF1E3A092900EB0204E57213F8025CB6
:10D8B000855413F8012CA275ECD130BDE46B0A0835
:10D8C000002383700370C37043707047D0F82C310D
:10D8D00093B1D0F8C82112685368D0F844219A4215
:10D8E00010B405D2C0685DF8044B1044C01A7047EC
:10D8F000D01A5DF8044B7047D0E907239A4201D350
:10D90000D01A7047C0681044C01A7047D0E9093275
:10D91000934212D3A3EB020CD0F830310169A3B1CA
:10D92000D0F8C421481E126853689C44604502D94F
:10D93000A0EB0C0070470020704701690B44A3EB7B
:10D94000020CD0F83031002BEAD1481EA0EB0C00BD
:10D95000704700BFD0F8303113B190F8E001704744
:10D96000D0E90903181AB0FA80F04009704700BFE7
:10D97000D0F82C21034610B472B1D0F84421C1680C
:10D980005C69881A013A205C08BF0A465DF8044BBE
:10D99000C0B2C3F844217047006A5C69411C205C36
:10D9A000DC68C0B2A14238BF0A465DF8044B1A6277
:10D9B000704700BFD0F8E43103B11847704700BF8B
:10D9C000F8B590F8F931012B1CD0002A164619DD64
:10D9D00005460F460269436AD41AA8693946B4421B
:10D9E0001844A8BF34462246361B53F0B7FD686A78
:10D9F0002A6927440444002EB4FBF2F302FB1343CC
:10DA00006B62E9DCF8BD00BF38B5D0F8E4310446FC
:10DA10000D460BB19847B8B1636AA269D554636AE1
:10DA200021690133D4F830218B4228BF002363627F
:10DA300022B12046BDE83840F5F7F4B9D4F85021BA
:10DA4000136843F08003136038BD00BF002308490A
:10DA500001E0152B09D003EB4302013311F802C09A
:10DA60000A448445F5D1104670470020704700BF36
:10DA70004C21002408B3B1FA81F35B09E9B14FF0FE
:10DA8000100C10B50E4C4FF0010E224604E001338D
:10DA9000572B10D092F804C0604502F11C02F6D159
:10DAA0000EF1010C71455FFA8CFEF0D1C3EBC3039C
:10DAB00004EB830010BD002010BD0020704700BFA4
:10DAC000C81C0A082DE9F0411E4688B0030990469B
:10DAD0000E9F00F00F04403349B30793FFF7CAFFCE
:10DAE000C2790546079B41463046CDE90042144ABB
:10DAF000B847C8B12868F4F7B9F8A9796A7911F07C
:10DB0000020FDFF84CC04FEA92020E49ED7908BFD0
:10DB100061460132079B0094CDE90102CDE903156E
:10DB2000094A00213046B84708B0BDE8F081074AED
:10DB300041463046BC460E9408B0BDE8F04160470F
:10DB400051010B08B9EF0A0863010B0885010B08A6
:10DB500090FA0A082DE9F04F184F884601F109099B
:10DB600001253B8804339EB218F8014BB4464FF0B0
:10DB7000000EACF1040305FA0EF29BB222401146EE
:10DB800002B1818903F1010B00EB830A1FFA8BF3C9
:10DB9000CAF814109C45F2D10EF1010E0CF1040CE0
:10DBA000BEF1080F1FFA8CFCE3D12036C845B6B28F
:10DBB000DAD100233B80BDE8F08F00BF147E002443
:10DBC0002DE9F04FDFF8949083B00F4601F106087D
:10DBD000B9F80230012500210B339BB2019317F8ED
:10DBE00001EB4FF0000C019A0126A2F10B039BB24E
:10DBF00006E0013384899BB2CBF81440934209D0EC
:10DC000000EB830B002EF4D10133CBF814609BB2F0
:10DC10009342F5D10433BCF1090F00EB8303596043
:10DC200010D0BCF1080F0BD005FA0CF313EA0E0F5D
:10DC300014BF012600260C320CF1010C92B2D4E77D
:10DC40000026F8E7019C474504F17804A3B201934C
:10DC5000C5D1A9F8021003B0BDE8F08F147E0024EE
:10DC60002DE9F8430B46067B282200211F78044645
:10DC70004FF00008FF43C0E90566C0E90766C0E948
:10DC80000966C0E90B66C0E90D663C30FFB253F08F
:10DC9000D9FC4FF0140E4FF0050C47FA0CF2734606
:10DCA00002F00102002A424414BF4FF019094FF05C
:10DCB0000A091CF001055FFA82F80EEB090018BF93
:10DCC000354680B2591C04EB83028BB255619842F1
:10DCD000F8D10CF1FF3CCE44BCF1FF3F1FFA8EFEA1
:10DCE000DBD118F0010F734614BF19250A250EEB7E
:10DCF000050080B2591C04EB83028BB2566183424B
:10DD0000F8D1AE44084900221FFA8EFE0EF101033D
:10DD10000EF1040E9BB204EB8E0E8B80CEF8042025
:10DD20002361BDE8F88300BF147E002470B5094C60
:10DD3000A36873B10546002606E099681A681E7349
:10DD4000A1609047A36823B15A681846AA1A002A0E
:10DD5000F3DA70BD147E002470B5204C2378012BBB
:10DD600000D070BD1E4B1B68002BFAD01D4D2B68D8
:10DD700028465B6898470028F3D01B4B1B4E1A6857
:10DD8000338892889A4219D3194900222846096893
:10DD90004968EA622A6803FB01F1D368984733882F
:10DDA000144A013352683380002ADAD0116893880C
:10DDB0004A69134218BF1B048B6170BD0D4B0022D2
:10DDC0005B682270002BCCD00B491A6809789B88BD
:10DDD000890748BF1B04936170BD00BFD82A002487
:10DDE000201E0024241E0024D02A0024D62A002429
:10DDF000C82A0024601E00246C1E0024944B1B685B
:10DE0000D90600D47047F0B5924CE3692DED028B32
:10DE100087B013B104F10C009847236A002B70D02F
:10DE20008D4894ED188A9847C21C054675D0002885
:10DE300077DA431C00F0FF806FF001031A46A362FB
:10DE4000864E4FF609213368EB1A03FB03F38B422E
:10DE500000F386808249A1FB031343F3CF0394F8B8
:10DE60007D00411C04EB4000A0F88030CBB2052BB4
:10DE700084F87D3000F08D8094F88A303560002B76
:10DE800000F09480B4F88200B4F88030B4F88410C4
:10DE90000344B4F8860094F834600B44B4F8881056
:10DEA00003440B441BB2B3F5FA4F1946A8BF4FF415
:10DEB000FA4121EAE171A18746B9002A06DDB3F5EE
:10DEC000167F7EDB01231E4684F83430654B1878BC
:10DED0001B2848D01C2838D1E76A634DA36B002F5C
:10DEE0002A806E80AB802EDD002A2CDDB1F5167FF6
:10DEF00029DA002E00F0A7809A42ACBF002301234C
:10DF000022E04FF0FF3357491A460878A3621B28D6
:10DF1000E36202D1544D6A80AB8007B0BDEC028B46
:10DF2000F0BD636E514904EB830201330968052B90
:10DF300090662163636652D094F87C30002B53D1F5
:10DF40000246A2627CE70023EB80D4ED097AB4EEAE
:10DF5000E78AF1EE10FA0FD54FF0FF33E362DCE70A
:10DF60004FF4C8537BE7D4ED097A3F4DB4EEE78A0E
:10DF7000E980F1EE10FA14D4002A66DB07EE902A4D
:10DF8000F8EEE77A67EE887AFDEEE77A17EE903AD8
:10DF9000BDE70023356084F87D30012384F88A30A2
:10DFA00070E74FF0FF310B46E162B4E74FF6FF73C5
:10DFB00094F834604FF0FF31A387002E86D1002AF9
:10DFC00084DDA36B9A423CDD02EB820328480026E5
:10DFD000C3EB0313A0FB03035B09A36376E70022F3
:10DFE0000123626684F87C30224F01AE0FCF0FC64A
:10DFF00002993B688842336002DC0B4601461846B2
:10E00000DDE90432934202DC16461A463346834267
:10E01000A8BF03468A42B8BF0A460399994202DB69
:10E0200018460B4601469342A8BF13468B42B8BF21
:10E030000B461A4685E70D4B0246A0621B68236318
:10E04000FEE6002642E701237EE74FF0FF335EE75E
:10E05000D0630024147E0024207E002418050024B0
:10E06000CDCCCCCCB01E0024B41E0024581E0024FD
:10E070001F85EB517C7E00242DE9F04F3E4C87B08C
:10E080000A4600210646FCF7DBF905903B4A237857
:10E09000608802EB8303D3F874A1F8F7F5FB83687B
:10E0A000C1680493364B1A78002A4BD0DDF81080F3
:10E0B0000491002721796279049B07FB012213F860
:10E0C0000290B8F1000F3FD018F802504D45059A64
:10E0D000304607F1010713BF012100214FF0010B6A
:10E0E0004FF0000BFCF7ACF905907DB305F00F0283
:10E0F0002D0953465946403502923046214ACDE912
:10E100000075FAF705FEB9F1000F2AD009F00F02E9
:10E110004FEA191953465946029209F14002304616
:10E12000CDE90072174AFAF7ADFDA279012A38BF8E
:10E130000122BA42BEDC0834134BA342A6D107B079
:10E14000BDE8F08F9046B4E74546BFE7B8F1000F51
:10E15000D9D053460D4A594630460097FAF7D8FDB4
:10E16000D1E77306E1D45346084A59463046009732
:10E17000FAF788FDD9E700BF086C0A08E46B0A08C3
:10E180002853002497010B08586D0A08AD010B08AD
:10E1900038B50C4B0C4603EBC0050B4895F8242012
:10E1A00003EB8203D3F87411FAF7CAFD95F82A300D
:10E1B00033B1611C0548C9B2BDE83840FAF7C0BDAB
:10E1C00038BD00BFE46B0A0899030B08333B0B080A
:10E1D00002460846531C05D1044B1A681B790A6095
:10E1E0000B7170470249F9F767B800BF4C010B0883
:10E1F000343B0B0810B501311446FFF73BFC28B93E
:10E20000064B1A681B792260237110BDC279204623
:10E210000349BDE81040F9F74FB800BF4C010B08A7
:10E220005E010B082DE9F041154686B08846194677
:10E230006A1CBDF830600D9F26D0030900F00F0462
:10E24000184A30464033CDE900450593B847C0B180
:10E25000EAB2D8F8000098F805100F2A11D82A461B
:10E26000F3F76CFC68B1028801783046059B039196
:10E27000C2F30321120B02910021CDE900420A4AA8
:10E28000B84706B0BDE8F0817306FAD4030900F080
:10E290000F00064ABC460C904033304606B0BDE83D
:10E2A000F0416047C1010B08D3010B08FC010B08CA
:10E2B0002DE9F04F704D0A460021824605F1900B82
:10E2C0002DED028B8BB0FCF7BBF8814600266B4B23
:10E2D0001C78AB7AB34200F391801035AB45F5D191
:10E2E00040F21620F8F7D0FAD0E902530CB12C46D0
:10E2F0001D460DF1100B002715220021584653F042
:10E30000A1F92E78002E41D069783046FFF7B2FB94
:10E3100095F9023008EE100A5A1C029353425341F9
:10E32000002C00F0A580002214F802C0A018B4450B
:10E3300040F09A8090F90280029A424540F0928023
:10E3400042788A4208BF0123012203F001030BF83F
:10E3500007204A4683F0010150460393FCF770F80A
:10E36000039B81464CB1464A18EE101A3046CDE95F
:10E3700000A24246FFF756FF039B424A18EE101ACE
:10E380003046CDE900A2029AFFF74CFF0137033572
:10E39000152FB6D16CB304F13F06394FDFF8E48096
:10E3A0001BF8013B02930BBB2078F8B194F90220D3
:10E3B00001321BD06178FFF75DFB05464A4601211B
:10E3C0005046FCF73DF894F90220029B294681460D
:10E3D0002078CDE900A7FFF725FF2078029B4FF0BA
:10E3E000FF322946CDE900A8FFF71CFF0334B442F1
:10E3F000D6D10BB0BDEC028BBDE8F08FE888F8F702
:10E4000043FAD0E902230CB114461A46297A6B7AF2
:10E4100006FB013312F903800CB3E756B8454A46B0
:10E4200050460DBF01230023012100210293FCF778
:10E4300007F8029B814644B1114A31462846CDE98E
:10E4400000A23A46FFF7B4F9029B0E4A314628462D
:10E450000136CDE900A24246FFF7AAF937E74FF0AF
:10E46000FF37DBE700236FE703323F2A7FF45CAF1F
:10E470004FF0FF386DE700BF1C050024285300242F
:10E48000118D0408858C04082DE9F04F07468BB0E8
:10E4900040F216200391F8F7F7F9039A0446002199
:10E4A0003846FBF7CDFF3F4A0646D4E902531478BD
:10E4B0000CB12C461D461522002104A853F0C2F8C9
:10E4C00005F13F03039395F80090B9F1000F30D0A8
:10E4D00095F801A0002C63D022460023117849450D
:10E4E00057D1283392F8018001226B4403F8182C8D
:10E4F000D0453246384613BF012100214FF0010BB1
:10E500004FF0000BFBF79CFF064654B1B8F1000F2B
:10E5100007D0254B5A464146484600933B46FFF7F5
:10E52000D1FA224B5A465146484600933B46FFF7E4
:10E53000C9FA0335039B9D42C5D13CB3651C0DF15F
:10E5400010084034DFF86090DFF860A018F8013B55
:10E55000CBB915F8013CB3B116B13046FAF7ACFBB4
:10E5600029783B4615F8010C0022CDF800900026D2
:10E57000FFF7A8FA002215F8010C3B461146CDF82A
:10E5800000A0FFF79FFA0335A542DFD10BB0BDE82D
:10E59000F08F01330332152BA0D14FF00008A7E70D
:10E5A000A046A5E728530024118D0408858C040893
:10E5B00008B5294B1B68DB041ED5B5EE400AF1EE09
:10E5C00010FA26D0DFED257AB4EEE70AF1EE10FA64
:10E5D0001FD49FED237AB4EEC70AF1EE10FA2AD8C1
:10E5E00070EE677A9FED1F7A9FED1F0AA7EE870AEC
:10E5F00052F036FA80B208BDDFED187AB4EEE70AC1
:10E60000F1EE10FA0BDA9FED190A52F029FA80B2F6
:10E6100008BD9FED170A52F023FA80B208BD70EED4
:10E62000677A9FED147A9FED140AA7EE870A52F0DD
:10E6300017FA80B208BDDFED117ADFED116A70EED6
:10E64000677A9FED107AA7EEA67AB0EE470A52F0ED
:10E6500007FA80B208BD00BF8C5800240000404279
:10E6600000E0824466BEFFBE0060BB4400007A4406
:10E670000080BB4438DFFF3E00407A440000834402
:10E6800066BEFF3E00A0BB448D4B1B6813F0200309
:10E6900070B52DED048B37D08A4C94F88B3013F085
:10E6A000020300F0BF80D4ED267AB4F89C30F8EE77
:10E6B000E77AC4ED237A002B40F0E380DFED828A15
:10E6C00094F8C020012312F0010225D094F8C12053
:10E6D000002A00F0CB8094ED339AB1EE499A002BDA
:10E6E00040F0BA8094ED378ADFED788A784B1E7857
:10E6F0000E2E07D19FED770A28EE000A52F0B0F9EE
:10E70000754B9880012331E0DFED6F8A6D4C94F8F2
:10E71000C02012F00102D9D194F8C11000297CD197
:10E7200094ED317ADFED6D6AD4ED337A27EE267AF7
:10E73000F1EE677A84ED317AC4ED327A63B101216A
:10E7400094F8D420D4F88C308A4284F8C210C4F8EB
:10E75000D03018BFC4F8C8305D4B1E780E2E00F0C4
:10E760009D809FED5A8A0023B0EE489A94ED397A45
:10E77000D4ED3A6A38EE478AD4ED387AA6EE887A34
:10E7800037EE676A84ED397AE6EE867AC4ED387A38
:10E79000C4ED377A0BB1C4ED327A94ED3D7AD4ED05
:10E7A0003B6AF0EE475A9FED4E5A77EEE66AC4EDAB
:10E7B0003B7AF0EE477A94ED3E6A94ED3C0AD6EE51
:10E7C000855AE6EE257A37EEC07AC4ED3D7AA6EE9C
:10E7D000070A84ED3C0A52F043F902B282EAE2737E
:10E7E000A3EBE2739BB2092B34D9002AACBF0A38E1
:10E7F0000A3005B20E2EA4F8FC5016D0242E09D1F2
:10E80000DFED347A94ED320A20EE270A52F028F92F
:10E81000314B5880BDEC048B70BD84F8C22084F865
:10E82000C1207DE7DFED288A71E7DFED2D7A2A4CE4
:10E8300068EEA78A9FED270A29EE000AFDEEE88A16
:10E8400018EE903A238052F00BF9E5806080BDEC21
:10E85000048B70BD0025CDE794F8C23073B194ED00
:10E86000238AD4ED347A38EE678A3FE794ED319A03
:10E87000012284ED339A84F8C1202EE794ED378A83
:10E8800034E707EE903ADFED166A9FED167AF8EE60
:10E89000E77AC6EEA78AC8FEC78A11E7D4ED237AC5
:10E8A00000239FED117A0C4A67EE877A9FED078A65
:10E8B000B0EE489AFDEEE77A17EE901A918055E790
:10E8C000D0630024147E00249A99993E0000000031
:10E8D000B01E0024CDCCCC3DB41E0024CDCC4C3F8A
:10E8E0000000C8426666663F0AD7233C6E4B1B7821
:10E8F0002DE9F04F87B0002B00F0CF806B4D4FF02B
:10E9000000086B48A968FAF75BFA69686948FAF782
:10E9100057FA694B6948DFF8DCA1D3E90031C91A1D
:10E92000674BD3F80021B1FBF2F2FAF749FAFAF794
:10E93000A5F96448FAF7BAF96348FAF7B7F9634BEF
:10E940005FFA88F41B78A34221D8614C0025614FFF
:10E95000FAF794F92646013556F8041B3846FAF7BB
:10E96000EFF9162DF7D101255A4EFAF787F923460C
:10E970006168013530461B680434C91AFAF7E0F9BA
:10E98000162DF4D107B0BDE8F04FFAF777B9524B26
:10E9900014264FF03C0B671C03EB840306FB045664
:10E9A00093ED000A52F05CF896F81EE081B2B6F8DA
:10E9B0000E901EF0010F80B214BF52222D221EF0C5
:10E9C000020F0490504614BF54232D231EF0040F51
:10E9D00007EE903A14BF56232D231EF0080F009324
:10E9E00017EE903A14BF4FF0430C4FF02D0C1EF071
:10E9F000800FCDF804C014BF4FF0530E4FF02D0E12
:10EA0000B1FBFBF10591642101FB09F1CDE902E1C4
:10EA10003946FAF795F9B37FDB073AD55C232F4ADD
:10EA20006343D118D05891ED010A70B1B8EE400A95
:10EA3000DFED2B7A20EE270A07EE900AF8EE677AD0
:10EA400080EE270A52F00CF800B2642290FBF2F13B
:10EA500002FB11022348FAF773F91421224808F146
:10EA6000010801FB075701FB0454F988628A0491ED
:10EA7000218B02F0030392080391E18A0291A18B9A
:10EA80000191A18A009119214B43218AFAF798F943
:10EA900055E71648FAF7D2F8DFE7154807B0BDE8A2
:10EAA000F04FFAF703B900BF04000020581400200B
:10EAB00010020B0820020B08701C002037020B0804
:10EAC000147E002464020B08C0020B08B42200204C
:10EAD0000415002070030B08E43600207811002094
:10EAE00000401C4639030B084E030B0845030B0876
:10EAF00074030B081C030B082DE9F84F06460C465F
:10EB00001E4D3A274FF00008DFF87890DFF878A024
:10EB10002046FBF751FED5F800B048B921465846CB
:10EB2000F8F728FD20B921466868F8F723FD80B181
:10EB30005846FAF783F8696811B15046FAF700F9B8
:10EB4000A96811B14846FAF7FBF84FF00108FAF747
:10EB500095F8013F05F11005DAD12046FBF72CFEB0
:10EB600048B9B8F1000F06D1224630460449BDE845
:10EB7000F84FFAF7FCBEBDE8F88F00BFC86E0A0870
:10EB80009C030B0896030B0890030B088160F3F7B6
:10EB900015BF00BF0171F3F711BF00BFF8B590F8C2
:10EBA000F931012B6BD0D0F830310446002B67D0FF
:10EBB000EFF31185502383F31288D0F830311B68AE
:10EBC00003F00103002B57D1D0F8D021D0F8D41195
:10EBD0000A4302F02102212A4ED0D0E909218A42BB
:10EBE0005AD054D9531A9BB2A262002284F8E02171
:10EBF000D4F8D021202A3FD1A26951183CD0B3FAD1
:10EC000083F25209002B37D094F8CC01012833D07D
:10EC10002120A4F8A6314FF0010CC4F8D821C4F883
:10EC2000D001D4F8C401C4F8A011A4F8A43184F828
:10EC3000CCC100283AD0234E90F834E0C663224E6F
:10EC4000E64502650664214EC6640CD090F8356036
:10EC5000D4F85071664580F834C021D04FF4006379
:10EC600080F834204365102100222023C4F8D811F5
:10EC700084F8CC21C4F8D031EDB285F31188F8BD09
:10EC8000D0F85021136843F080031360F8BD006989
:10EC90001A46431A9BB2A7E7012380F8E031EBE75D
:10ECA00007F1280242F06AFA0028DCD1D4F850318A
:10ECB00000224021196284F8CC219A6842F0800237
:10ECC0009A60D9E7A1D20808C5D2080801D308087C
:10ECD0002DE9F041CF4CA36820469847002800F06A
:10ECE0009380B4F90E30A17D06EE903AB4F910305D
:10ECF000092907EE103AB4F91230F8EEE66A07EE89
:10ED0000903AB8EEC77A4FF00103F8EEE77AC4ED17
:10ED1000126A84F8543084ED137AC4ED147A75D0F5
:10ED2000BD4D04F1480027F055F9AA8DAB6A002AC1
:10ED300077D1BA4A1268520700F1AE80B3F90020C9
:10ED400094ED126A06EE902AB3F90220B3F904306A
:10ED500007EE102AF8EEE66A07EE903A2B88B8EE36
:10ED6000C75A94ED137AF8EEE75AD4ED147A76EE9A
:10ED7000666A37EE457A77EEE57AC4ED126A84ED7D
:10ED8000137AC4ED147AFBB3D5ED024AD5ED085AD7
:10ED900076EEE46A95ED055A95ED033A77EEE57A5D
:10EDA00037EE457AD5ED063AE6EE834A95ED094A07
:10EDB000F0EE656A95ED016AA7EE235A95ED047AA7
:10EDC000E4EE276AD5ED077A34EEC62AC5ED024A8D
:10EDD00075EE472A85ED055A76EEE75AC5ED086AC5
:10EDE000F0EE466AA2EEA37AE4EE257AE3EE026A3A
:10EDF00085ED047A84ED137AC5ED016AC4ED126ADB
:10EE0000C5ED077AC4ED147ABDE8F081824D04F1B6
:10EE1000200104F1480027F077F8AA8DAB6A002A98
:10EE200087D0B2F5C87F00F0A9807D49002694ED17
:10EE3000127A0020D1ED416A012AD4ED137AF8EE5E
:10EE4000E66A94ED146AA66476EE876A91ED427ADA
:10EE5000B8EEC77AFDEEE66A37EE277AD1ED437A4F
:10EE6000C1ED416AF8EEE77A1880BDEEC77AE66434
:10EE700077EE867A81ED427A5880FDEEE77A266554
:10EE8000C1ED437A988000F09A80013AAA85634ADE
:10EE9000126852077FF552AF614EB6F81021322A40
:10EEA0002DD0002A40F0868096F82E21002A3FF4CB
:10EEB00045AF06F590705B4F4FF0000C07C887FB1D
:10EEC000028ED21786F82EC1C2EB2E12A689921B93
:10EED0009A8087FB0062C017C0EB221087FB0127D6
:10EEE000C91701221880C1EB271159804E4BA3F896
:10EEF0000EC0C3F80A20F9F713FDAB6A1EE71A68C3
:10EF0000DFED4A7AC6F81421B3F90420A6F81821D7
:10EF1000454AD268C6F81C2194ED127A00200021DF
:10EF200077EE877AA0641980B6F81021FDEEE77AB3
:10EF3000322AC6ED487A7BD096ED497A012AD4ED83
:10EF4000137AB8EEC77AD4ED146AE064598037EECC
:10EF5000277AD6ED4A7A2065F8EEE77A9980BDEEF9
:10EF6000C77A77EEA67A86ED497AFDEEE77AC6EDA6
:10EF70004A7A6ED0013AA6F8102195E7D4ED126ACC
:10EF8000002094ED137A0021D4ED147AFDEEE66AA8
:10EF9000BDEEC77A224EFDEEE77AA064C6ED416A67
:10EFA000198086ED427AE0645980C6ED437A206587
:10EFB00099806AE7D6ED487AF8EEE77AACE717EE83
:10EFC000907ADFF860C016EE906A17EE101AC83714
:10EFD000C836C8314FEAE77E8CFB0787CEEBE717D0
:10EFE000B4F80CE0A7EB0E079F808CFB06E7F61742
:10EFF000C6EBE7161E808CFB016CC917C1EBEC1148
:10F000005980094BC3F80A20D881F9F789FCAA8DE9
:10F01000AB6A3AE7F4230020BC2300208C5800247C
:10F02000147E00241F85EB51C85800240000000006
:10F0300094ED137AD4ED147ABDEEC77AE064FDEE58
:10F04000E77A5980206586ED497A9980C6ED4A7A3B
:10F0500090E70B2086F82D2186F82C1110F06AF825
:10F06000AB6AD6F81421D6F81C111A60B6F918212B
:10F070009A80024AD160B6F810217BE7C858002474
:10F0800038B5074C074DAC4203D3074B01221A7029
:10F0900038BDA288D4E9021052F060FA1C34F2E7BD
:10F0A00028860B08908F0B08285300242DE9F04F79
:10F0B0000C4695B00546344920461746FEF732FA0D
:10F0C000064600284FD131492046FEF72BFA064666
:10F0D00000284AD12E492046FEF724FA0646002889
:10F0E00045D12C492046FEF71DFA0646002840D19E
:10F0F00020462949FEF716FA0028064612BF0824C2
:10F10000264601240FB144F0100424493046FEF78E
:10F1100009FA80B344F02004214B1B780BB9FFF7A8
:10F12000AFFFF7F743FC14F0090F00F049831D48C7
:10F13000F9F7C2FD0020FEF75BFA14F48073069322
:10F140003CD11948F9F7B8FD1848F9F7AFFD04F0BC
:10F150001803182B05D11648F9F7AEFD1548F9F735
:10F16000A5FD01232BE00124CCE70224CAE70424F7
:10F17000C8E78124C6E710493046FEF7D3F90028D6
:10F18000CAD044F48074C7E7CF030B08D6030B083A
:10F19000DE030B08E4030B08ED030B087DF90A08F6
:10F1A00028530024F6030B08FE030B0816040B0873
:10F1B00022040B084A040B08F1030B0800230593F3
:10F1C000F9F75CFDBC4904F01008BC48F9F7F8FDFC
:10F1D000BB49BC48F9F7F4FD04F48473082B07D14C
:10F1E000B9492846F9F7C2FEB7492846FAF7EAFCBA
:10F1F00014F0800308930ED1B44B204693F83021CD
:10F2000003F59873002AB24A06BF01211346002174
:10F21000B04AF9F737FDB0492046FEF72DFFAF4958
:10F220002046FFF731F9AE492046FFF741F8AD4BD4
:10F23000D3F800B0AC4B1B680493B8F1000F40F05A
:10F24000FD814646A948F9F737FDA94B4FF0000963
:10F25000DFF860A307930393049B6BEA03030A930D
:10F26000039B53F8047B0393002F40F0E981049B38
:10F27000DFF844A363EA0B030993079B53F8042BBD
:10F2800003920793002A40F005829A4B20469A4A3F
:10F290009A49FCF7BDFA089B002B40F0A382DFF8E7
:10F2A0001CA32046DFF818B39AF800209BF8003022
:10F2B000DFF810939A42924A13BF012100210127DF
:10F2C0000027FBF7BDF89BF8003039460646013BA6
:10F2D0008C4A204659F82330F9F71AFD9AF8003085
:10F2E0003946894F013B874A204659F82330F9F7C0
:10F2F000C9FCD7ED007A854A2046F5EE407AF1EE5A
:10F3000010FA0CBF01210021F9F7BCFC33463A4644
:10F310007F492046FCF7F4FC7E4B7F4A20467F491C
:10F32000FDF726F9B8F1000F05D07D4B93F90230B7
:10F33000002B00F0DF817B48F9F7BEFC7A48F9F733
:10F34000B5FC0023764A20467849FDF74FFA784B02
:10F350006FF07F42774F784E2046019300923A68D3
:10F360003168FEF789F840F20222744B2046009281
:10F370000193BA68B168FEF77FF8B8F1000F40F06A
:10F38000BB816F48F9F798FC42466E4808266E49E3
:10F390000127DFF834C210F8013B11F8019B03F19B
:10F3A000500EEE440EF8209C1CF801EB0EF1500AB2
:10F3B000EA440AF8109C2FB1A3EB0E0EDEF1000711
:10F3C00047EB0E07013EE6D187F0010120468DF89C
:10F3D0003860FBF735F810AB5C4A394620468DF8AB
:10F3E0004860F9F795FC0CAB584A39462046F9F7C6
:10F3F00049FC574B574A20465749FCF7B1FE574B3B
:10F40000574A20465749FCF737FF574B514A204689
:10F410005149FCF7C3FF554B554A20465549FCF767
:10F42000ABF8554B554A20465549FCF723FB554B45
:10F43000554A20465549FCF7D3FD554B554A2046C1
:10F440005549FDF7CFFC554B554A20465549FDF728
:10F45000ADFBB8F1000F40F051815348F9F72CFC97
:10F46000524F4FF0000BDFF86481414602223846CC
:10F4700052F0BEF8002897F800A0204614BF0121E2
:10F480000021039A0CBF4FF001094FF00009FAF771
:10F49000D7FFBAF1020F039040F0338198F80120B2
:10F4A0004FF0190A40F2EE23494620461AFB023279
:10F4B0003F4B01928CE000BF5A040B08F7F50A0895
:10F4C00068040B0815F60A0890FA0A08147E00244E
:10F4D00006340B086D040B087A040B0884040B082F
:10F4E00089F10A08E87B002488580024B0030B083F
:10F4F000B83D0A08A1040B081057002430770024F7
:10F50000BE030B08A8040B08145C0024B1040B080C
:10F51000E879002421FE0A08E86E002430700024F7
:10F52000486F0024B8030B08C0040B08BC6F00240C
:10F53000CD040B087C5900247C7C0024D4040B08E7
:10F54000C4030B08887D00245CBC0A0853F90A0830
:10F55000C3F60A08F86D002494700024E0040B0838
:10F56000786E002414710024DB040B08E6040B08F9
:10F57000E458002488730024EA040B08BC6C0024BF
:10F580009C710024F3040B08E86D002488710024AA
:10F59000FB040B080C5A0024C877002404050B0850
:10F5A000285E0024E87A0024C8030B08CC720024EB
:10F5B0007CBE0A088A040B0896040B084C7D0024C4
:10F5C000C8560024343E0A08D8560024746C00241F
:10F5D00098F800209A5C5B460092864AF9F798FBFF
:10F5E0007A7840F2EE21844B20461AFB02124946FB
:10F5F00001923A789A5C5B4600927E4AF9F742FBA8
:10F600000BF1010B023708F10208BBF1120F7FF476
:10F610002CAF7A4B224600212846FAF73FFF2307FA
:10F6200000F18580764E224628463178FDF798FF16
:10F63000224671782846FDF7B7FFB7E0714E04E621
:10F640003B7823B301230A9A204603FA09F31A40B0
:10F650000B930CBF0121002109923246FAF7F0FE0C
:10F66000049B0646204663EA0B020B9B1A423B466C
:10F67000524614BF01210021F9F74AFB09993B4684
:10F6800052460039204618BF0121F9F7FBFA09F16B
:10F690000109E5E5039B1B7853B34FF00109049B77
:10F6A00009FA07F913EA090F0BD06BEA0303524674
:10F6B000204613EA090F039B14BF01210021F9F72B
:10F6C00027FB1BEA090F13D0099B3246204613EA99
:10F6D00009090CBF01210021FAF7B2FEB9F10001BE
:10F6E0000646039B524618BF01212046F9F7CAFA85
:10F6F0000137C2E5444B25E6444A46E6444B0393B2
:10F70000AEE698F8002049463B4B20469A5C5B46A3
:10F710000092404AF9F7FCFA3A78374B49462046BE
:10F720009A5C5B4600923B4AF9F7ACFA68E700271F
:10F73000F9B2013722462846FDF712FF042FF7D110
:10F740002F4FDFF8F4803B7888F80030069B33B900
:10F750003148F9F7B1FA31492846FBF78FFCFF230E
:10F7600088F80030F1B2013622462846FDF71CFF2A
:10F77000042EF7D17B782A4C2370069BA3B9294825
:10F78000F9F79AFA25492846FBF7A8FC2648F9F725
:10F7900093FA2648F9F752FAFF232370002015B098
:10F7A000BDE8F04FFAF757BEFF232370059B002BEF
:10F7B000F4D01F48F9F780FA1E48F9F777FAEDE719
:10F7C000A10706D50E4B224628461978FDF7C8FE3C
:10F7D000E4E76207E2D50A4B224628465978FDF74E
:10F7E000E3FEDBE7054B224618212846FAF756FED2
:10F7F000DCE700BFB5F90A087CBE0A08CF030B0896
:10F80000CC7D0024B0030B08B8030B08C4030B081D
:10F81000C8030B08C5F90A0808050B0890FA0A087E
:10F82000B50400242B050B0852050B0855040B08E2
:10F8300065050B087B050B08B4040024002235E4A1
:10F84000012233E4224B30B583B09A7901906AB338
:10F8500093F82630DFED1F6A07EE903A1E4B1F4CDF
:10F86000F8EEE77A1D7886EEA77A84ED187ADDB196
:10F870001B4BDDED017AB3F85E31F8EE670ADFED80
:10F88000197A00EE103A60EEA70AB8EE400AF7F7D0
:10F8900025F904F12003002103EBC50219600833A8
:10F8A00003ED010A9A42F9D103B030BD0E4A126845
:10F8B0001201F9D593F82630DFED066A07EE903A8B
:10F8C000064BF8EEE77A86EEA77A83ED187AEBE737
:10F8D000E429002455555540B4220020E436002088
:10F8E000147E0024BD3786358C580024A54B1B7828
:10F8F000002B00F0B2802DE9F04FA34E83B096F8B4
:10F900000491B9F1010F02D003B0BDE8F08F9F4B15
:10F910009F4F1B6893F83450002D6ED09D4B0022F2
:10F92000DFED9D6ABE4697ED187A904693F800B0D9
:10F9300040F6FF7A67EE266A9FED986A3346984C48
:10F94000019200971CE000F47061B1F5006F00F0C7
:10F95000B38000F29380B1F5806F00F0DB80B1F5E9
:10F96000C06F7BD1C0B24CF0080C988283F81EC0E7
:10F97000013214330EF1040E0234D2B2AA422AD05C
:10F9800093F81EC09889BCF1010FDCD1504500F0FE
:10F99000D080C0F30801400A01FA00F081B20029CA
:10F9A00000F0BF807F4F80B2BBF12D0F07EB5101FC
:10F9B000B1FBF0F000F0D7804FF6FF718842D7D04E
:10F9C00007EE900A0199F8EEE77A014480B20191BE
:10F9D00067EEA67AB3E0009FB8F1000F0DD0DDED21
:10F9E000017AB8EE677A07EE908AF8EE677A27EE2A
:10F9F000267AC7EE276AC7ED196A6B4BDFED6B6A93
:10FA00001878C7ED1A6A10B3694A97ED185A5E491B
:10FA100002EB8000A2F14803CC89083353ED037A4E
:10FA2000143107EE104A53ED025AB0EE676AB8EE91
:10FA3000C77A97EE056AE5EE867AE2EC017A9042A3
:10FA400043ED037AC6FEE76AE6D1C7ED1A6A0223E0
:10FA500086F8043103B0BDE8F08F7047B1F5007F40
:10FA600031D14CF0020CC1B283F81EC093F81FC014
:10FA700019828C45BFF47CAFD87779E7B1F5406F38
:10FA800013D0B1F5606F06D1C0B26CF07F0C9883D3
:10FA900083F81EC06CE7B1F5206F14D1C0B24CF0F2
:10FAA000200C188383F81EC062E7C0B24CF0400CF3
:10FAB000588383F81EC05BE7C0B24CF0100CD882AC
:10FAC00083F81EC054E7504546D0C0F30801400AF1
:10FAD00001FA00F081B221B3324F80B2BBF12D0F99
:10FAE00007EB5101B1FBF0F049D04FF6FF718842AE
:10FAF0003FF43EAF07EE900A0199F8EEE77A014431
:10FB000080B2019167EEA67A4CF0010CD88183F89F
:10FB10001EC017E0C0B24CF0040C588283F81EC01F
:10FB200026E7BBF12D0F7FF423AF4FF0FF3121808B
:10FB30001EE7BBF12D0FF0EE467A08D00020D881E9
:10FB400083F81E9008F10108CEED007A10E74FF01F
:10FB5000000100202180F2E7BBF12D0FF0EE467A84
:10FB600008D00020D0E74FF6FF71208088423FF494
:10FB7000FFAE25E74FF0000100202180C4E7208080
:10FB8000B3E700BF0400002058140020F023002039
:10FB9000E4360020B01E0024000070420000000087
:10FBA000B41E0024C0270900B4220020FFFF7F7F7D
:10FBB0005037002010B5437B04468268581C6073A0
:10FBC000D154627B237B934200D802B910BD2368D5
:10FBD000D4E9010198470023637310BD427B42B111
:10FBE000036810B50446D0E9010198470023637308
:10FBF00010BD704730B58BB04FF0010C044605685E
:10FC0000009100218DF80CC08DF820C00991CDE93C
:10FC10000123CDE90411CDE90611EFF3118C102376
:10FC200083F3128803681B6A0BB36846029B024683
:10FC30001BB1D3691432002BFBD12B6A6BB19968CD
:10FC400039B9934209D0196829B15B6899680029CC
:10FC5000F7D01433F3E7C3E900405FFA8CFC8CF370
:10FC600011882268136A002BFCD10BB030BD5FFAFB
:10FC70008CFCC5F820D08CF3118851F05DFEF0E7C4
:10FC800030B40568EFF3118C102383F312880368F6
:10FC90001B6AEBB18B6804460A461BB1D369143268
:10FCA000002BFBD12B6A6BB1986838B9934209D00D
:10FCB000186828B15B6898680028F7D01433F3E718
:10FCC000C3E900415FFA8CFC8CF3118830BC7047AB
:10FCD0005FFA8CFC29628CF3118830BC51F02CBE89
:10FCE00030B593B0002304468DF807100DF10601DE
:10FCF0008DF8062001220DF107058DF814308DF8DE
:10FD000028208DF83C200B930E9310930295CDE99B
:10FD10000332CDE90631CDE9083200220023016823
:10FD2000CDE90C23EFF3118C102383F312880368C1
:10FD30001B6A0BB302A8049B02461BB1D3691432A1
:10FD4000002BFBD10B6A6BB1996839B9934209D08A
:10FD5000196829B15B6899680029F7D01433F3E773
:10FD6000C3E900405FFA8CFC8CF311882268136AA7
:10FD7000002BFCD113B030BD02AB5FFA8CFC0B62E0
:10FD80008CF3118851F0D8FDF0E700BF30B593B087
:10FD900004460DF10705089200228DF8071009931B
:10FDA000012100238DF814200B920E9210920491E1
:10FDB0008DF828108DF83C100168CDE90252CDE98C
:10FDC00006220022CDE90C23EFF3118C102383F3DC
:10FDD000128803681B6A0BB302A8049B02461BB17E
:10FDE000D3691432002BFBD10B6A6BB1996839B916
:10FDF000934209D0196829B15B6899680029F7D046
:10FE00001433F3E7C3E900405FFA8CFC8CF31188EC
:10FE10002268136A002BFCD113B030BD02AB5FFA2D
:10FE20008CFC0B628CF3118851F086FDF0E700BF6B
:10FE300030B5002395B0012204468DF81C300DF139
:10FE400007050D93109312930B928DF830208DF8C7
:10FE500044208DF8071004950168CDE90532CDE9FD
:10FE600008330DF10F0300220A930023CDE90E237E
:10FE7000EFF3118C102383F3128803681B6A1BB302
:10FE800004A8069B02461BB1D3691432002BFBD198
:10FE90000B6A6BB1996839B9934209D0196829B1D5
:10FEA0005B6899680029F7D01433F3E7C3E9004091
:10FEB0005FFA8CFC8CF311882268136A002BFCD14A
:10FEC0009DF80F0015B030BD04AB5FFA8CFC0B62DF
:10FED0008CF3118851F030FDEEE700BF0246074B6E
:10FEE00002209A4208D801335B0840009A4280B24F
:10FEF00002D2FF28F8D97047704700BF7FF0FA029E
:10FF0000013905292DD81B4B4FF0280C02460CFB5C
:10FF100001FC10B403F5B074634464444FF0010C69
:10FF2000046003F5B07480F888C093F8600102287B
:10FF300019D0C9B2104809014158C3F8641171B110
:10FF40000221604683F860114FF48071A18102F1B3
:10FF500010014C32C3E95E125DF8044B704700207B
:10FF6000FAE70020704793F86D216046624483F8F9
:10FF70006D21F1E7147E00248C2100242DE9F04F3F
:10FF8000934F85B0DFF858924FF0010B4FF0000807
:10FF9000904E0AE008F101080BF1010B283709F136
:10FFA0000509B8F1060F00F0FB803B78022BF1D178
:10FFB00099F90320511C00F0F680D2B294465FFA02
:10FFC00088F10F2A6BD88448002403E00134033001
:10FFD0002A2C64D00378002BF8D145788D42F5D1D6
:10FFE0007D4804EB44047D4D044402EB4200A478B8
:10FFF00005F8204005EB8000756884604068A842E1
:020000040805ED
:1000000000F04B81B56AA84200F06581F56CA8420A
:1000100000F06981356FA84200F06981D6F89450EC
:10002000A84200F07281D6F8B850A84200F084814E
:10003000D6F8DC50A84200F07B81D6F80051A842E7
:1000400000F08381D6F82451A84200F07981D6F8D7
:100050004831984200F08E81D6F86C31984200F019
:100060008381D6F89031984200F0A781D6F8B43158
:10007000984200F09C81D6F8D831984200F0A981CE
:10008000D6F8FC31984200F0AA81D6F82032984286
:1000900000F0998116F8083C002B00F092800132A4
:1000A000D2B262458DD90023019399F90420531CE3
:1000B0007DD0D2B296465FFA88F10F2A68D84648BA
:1000C000002403E0013403302A2C61D00378012B93
:1000D000F8D145788D42F5D13F4804EB44040444FF
:1000E00002EB4200A5783D4C04F8205004EB800060
:1000F000746885604068A04274D0B46AA04200F081
:10010000EE80F46CA04200F0F680346FA04200F064
:10011000F780D6F89440A04200F0FB80D6F8B840B3
:10012000A04200F00081D6F8DC40A04200F0F6804A
:10013000D6F80041A04200F01281D6F82441A04236
:1001400000F00781D6F84841A04200F01F81D6F8A0
:100150006C31984200F01481D6F89031984200F04A
:100160002081D6F8B431984200F01581D6F8D83104
:10017000984200F04681D6F8FC31984200F03B816D
:10018000D6F82032984200F0308116F8083C93B13E
:100190000132D2B2964590D20023C7E90433F9E682
:1001A00005B0BDE8F08F4FF00F0C002207E74FF0CD
:1001B0000F0E00227FE7132306F807BC06F8083C61
:1001C000E6E7142306F807BC06F8083C67E700BF1B
:1001D000747F0024400100246C1A0A088000002467
:1001E000AC5C00244FF0000C6346E2460AEBCA0008
:1001F0000AF1010A06EB8000047F029400F11C045E
:100200000394029C002CC3D1037206EB0C03039AE7
:100210007B611323C56080F81DB050461370F1F761
:10022000DFFC019B002BB7D07869F1F785FB3869BB
:10023000F1F782FB3B697A68D968BB695962402152
:100240005C60996002F120019C631960C3E903447A
:10025000C3E90544C3E90744C3E90A44C3E90C44BC
:100260007B698BB1D9683032FB6959621C629C632F
:10027000C3E90024C3E90244C3E90444C3E90644D2
:10028000C3E90A44C3E90C440023504660491A46B6
:10029000F1F7BAFC01233B737CE61D469E460EEB4C
:1002A000CE0A0EF10100019006EB8A0090F81CA026
:1002B00000F11C0EBAF1000F7FF4F1AE03721423AB
:1002C0003544C46080F81DB08EF8003001983D615F
:1002D000F1F786FCE9E6012324259E46DFE74FF08F
:1002E000240C9A4682E7022348259E46D7E703233B
:1002F0006C259E46D3E702234FF0480C9A4675E7DB
:1003000003234FF06C0C9A4670E7042390259E4619
:10031000C5E704234FF0900C9A4667E706234FF099
:10032000D80C9A4662E705234FF0B40C9A465DE775
:100330000623D8259E46B2E70523B4259E46AEE7A0
:100340004FF490754FF0080EA9E70723FC259E4651
:10035000A5E74FF4907C00234FF0080A46E70723F7
:100360004FF0FC0C9A4641E702234FF4B4754FF06E
:100370000A0E94E74FF4A27501234FF0090E8EE7A1
:1003800002234FF4B47C4FF00A0A2FE74FF4A27C0B
:100390004FF0090A2AE74FF4D87C04234FF00C0AE7
:1003A00024E74FF4C67C03234FF00B0A1EE74FF4FB
:1003B000D87504234FF00C0E71E74FF4C675032374
:1003C0004FF00B0E6BE74FF4077507234FF00F0E3E
:1003D00065E74FF4EA7505234FF00D0E5FE74FF424
:1003E000FC7506234FF00E0E59E74FF4077C0723E8
:1003F0004FF00F0AFAE64FF4FC7C06234FF00E0A8A
:10040000F4E64FF4EA7C05234FF00D0AEEE600BF58
:10041000F90E0000036810B59B6804469847012256
:10042000FF236273A37310BD036810B504461B68F5
:1004300098470121236820469B689847E37B013356
:10044000E37310BDF0B583B004460D461646089F11
:10045000019338464EF0D4FC216828443246E672B7
:10046000A07220468E692946019BB44603B0BDE8C0
:10047000F040604703689B6A184700BF03685B6DE4
:1004800003B11847704700BF0368DB6C03B118471E
:10049000704700BF002310B5C373044642748A6CD2
:1004A000016003730AB11946904723680121204671
:1004B0009B689847FF2123680122A173DB6C62735C
:1004C0001BB12046BDE81040184710BD2DE9F04F84
:1004D0004C484FF0010A4C494FF002094B4B4FF08A
:1004E000040808271026202540244FF0800EDFF84E
:1004F00020C130F8022F12F0010F03D01960083329
:1005000023F804AC12F0020F03D01960083323F86B
:10051000049C12F0040F03D01960083323F8048CF4
:1005200012F0080F03D01960083323F8047C12F08E
:10053000100F03D01960083323F8046C12F0200F59
:1005400003D01960083323F8045C12F0400F03D085
:100550001960083323F8044C12F0800F03D019609F
:10056000083323F804EC12F4807F05D04FF4807B2D
:100570001960083323F804BC12F4007F05D04FF44F
:10058000007B1960083323F804BC12F4806F05D097
:100590004FF4806B1960083323F804BC12F4006F29
:1005A00005D04FF4006B1960083323F804BC12F433
:1005B000805F05D04FF4805B1960083323F804BCDA
:1005C00012F4005F05D04FF4005B1960083323F884
:1005D00004BC12F4804F05D04FF4804B19600833EF
:1005E00023F804BCD20B05D04FF400421960083345
:1005F00023F8042C01F5806161457FF47AAFBDE8F2
:10060000F08F00BFFE1B0A0800000258EC210024F6
:10061000001C025810B50409013C062C16D80D4ADE
:1006200000F00F0332F8141041FA03F212F0010245
:100630000ED001209840013808404FF00DF9064BCC
:10064000064A1B5D184402EBC00010BD002010BD1F
:10065000104610BD001C0A08101C0A08EC210024DA
:10066000F8B50C4F97F8343093B10B4C0025A668C1
:1006700001353079FFF7CEFF20B194F8DC10F27924
:10068000F1F72CFB97F8343004F5B474AB42EEDC90
:100690000120F8BD801C00203C05002038B50C4628
:1006A00005460078FFF7B6FF611C0446C9B210B1D9
:1006B0004123C171837120466978F1F753FEAB780D
:1006C00020461BB1BDE83840F1F7C6B9BDE8384057
:1006D000F1F7C8B92DE9F041FFF79CFF0C4B054637
:1006E00000241F680B4EBC4201DBBDE8F08104EB27
:1006F0004403F05C03EB0608FFF78CFF854204D14E
:1007000021464046BDE8F041C8E70134EBE700BFB1
:10071000005D0024D05C0024054B53F8203033B139
:100720001A689B8851690B4218BF1B04936170477C
:10073000601E00240E4B012210B40E4C93F800C032
:1007400002FA00F354F8200003EA0C0351B1003B15
:1007500018BF012318B1016882883BB18A615DF836
:10076000044B7047B3FA83F35B09F3E71204F5E730
:100770006C1E0024601E002410B5054C23681B6904
:1007800098472368002283F836209A6310BD00BF83
:10079000F023002010B5084C236893F8352012B1DF
:1007A000DB68984700B910BD044A0121236812682C
:1007B00083F836109A6310BDF0230020581E0024E1
:1007C0000D4A0E4B12889B8C07EE902A9FED0C6A07
:1007D000DFED0C6AB8EEE70A07EE903A9FED0A7A71
:1007E000F8EEE77A60EE277A67EE867AA7EEA67AC9
:1007F00027EE870A704700BFD86B0024E429002445
:100800000AD7233C3F89B6B6FCA9713F2DE9F84FC2
:10081000C14C804694F8C030DB072DED028B7CD5AF
:10082000BE4B94F85052BE4E1F88012D62D0022D4F
:100830003BD0002D47D094ED998AF37B33B1B38937
:1008400023B1B84B1B78002B40F0038194F8511270
:10085000A94238BF2946337A632B07D8022D00F00E
:10086000188194F85C22002A40F02A81AE4BB0EE49
:10087000487ADFEDAE6A1970B07BD4E99D231A4443
:10088000D4F87C32D31AC4F87C2207FB03F307EEBA
:10089000903AF8EEE77AA7EEA67A84ED997A0028E6
:1008A00070D1BDEC028BBDE8F88FB4F85432BB4276
:1008B000C1D29F4B012594ED998A1B6884F8505250
:1008C000C4F86832B9E7B4F85632BB421ED3984B2D
:1008D000D4F868121A68F37D521A03EB830303EB12
:1008E0008303B2EB830FA6DB012594ED998A84F88C
:1008F0005052A2E7B4F85832BB4280F0B680B4F848
:100900005232BB4202D2002584F85052884B94EDFB
:10091000998A1B68C4F868328FE794F85052DFF860
:10092000FC91EB1E012B39D9B9F80800C0F30B007C
:100930004EF092FF092840F3DB80794EB9F8007041
:10094000F3889F4203D33288BA42BFF46EAFB7EB4D
:10095000430F3FF76AAF0323DFED767A714A84F8DD
:100960005032B0EE678A84F851320023C4ED997A90
:100970001370A4F85232A4F85432A4F85632A4F8F2
:100980005832ACE0012900F0AC80022989D107205F
:10099000BDEC028BBDE8F84F0EF0CCBB604EB9F851
:1009A0000070F3889F4202D33288BA4203D2B7EB79
:1009B000430F40F38F80B9F80800C0F30B004EF0EE
:1009C0004BFF092840F3BE800023357D84F8503268
:1009D00084F85132002D00F0B880524A2946157033
:1009E0001D46554889B2DFED535A90ED345AC0ED9B
:1009F0003A5AFFF7E5FEC5EE007AB288738812FB1B
:100A000001F213FB01F3717C92B2B7EE007A9BB254
:100A10008A42A4F85222A4F85432C7FEC77AC7FE0D
:100A2000A57AC0ED357AC0ED367A40F2D280521AFE
:100A300092B28B42A4F8562240F2C9805B1A9BB254
:100A4000A4F85832642384F85D320023C4F860327D
:100A5000EBE610F0E9F900284ED1022329469D4229
:100A600084F8513238BF1946F5E6314BD4F8681294
:100A70001A68337E521A03EB830303EB8303B2EB52
:100A8000830FFFF6D8AE022594ED998A84F8505270
:100A9000D3E694F85C0298B90122C4F860828046DB
:100AA00084F85C22C3F16403244A08FB03F382FB4D
:100AB0000302DB17A3EBA253643384F85D32D5E65F
:100AC000D4F860021E4AA8EB00089045EADB84F8DF
:100AD0005D32CBE6032D40F0838094ED998A0325A7
:100AE000ABE6BDEC028B0820BDE8F84F0EF022BB50
:100AF000B9F800700A4E98E6337C834207D301238D
:100B000029469D4284F8513238BF1946A3E6002396
:100B1000294684F851329EE6147E0024D86B0024C6
:100B200090580024D76B0024D66B0024ACC527371F
:100B3000581E002400000000B42200206BCA5F6B26
:100B400080969800032DC8D075E63388294ADFF8CF
:100B5000B0A01268B7FBF3F3013392F96C20082BB5
:100B600028BF0823D9B28AF80010002A3FF439AF11
:100B70009A423FF436AF204A92F800E00EF10102AB
:100B800002F0030296453FF42CAF4FF0FF3C4FF0CC
:100B9000A40B09E018B93CEA2C0C28BF944601329A
:100BA00002F00302964516D014480BFB020090F9A0
:100BB0006C008342EED194465FFA8CF0F7F7EEFCBE
:100BC0009AF80010B9F8007094F8505209E7002321
:100BD00036E700222DE7BCF1FF3F3FF402AFEBE721
:100BE000B9F80800C0F30B004EF036FE09283FF7B5
:100BF000A5AE20E6C4560024AC52002404540024C0
:100C0000D76B0024F8B5114E0124114D522716F868
:100C1000010BFFF7FFFC0022202118B1C47187717E
:100C2000F1F75CF815F8010BFFF7F4FC4FF0530CEB
:100C30000022402120B1C47180F806C0F1F74EF8BF
:100C40000134E4B2052CE2D1F8BD00BF7C79002468
:100C50007079002438B50C4614F8011B41B10546E3
:100C60002B6828461B68984714F8011B0029F7D108
:100C700038BD00BF03681B68184700BF03682DE933
:100C8000F0415F6A1FB13B46BDE8F041184704469A
:100C90000D46164600E023689B6820469847B04200
:100CA000F9D3002E08DD2E442368204615F8011BD9
:100CB0001B689847B542F7D1BDE8F08103685B68CF
:100CC000184700BF03689B68184700BF0368DB68CC
:100CD000184700BF03685B69184700BF03689B6A39
:100CE00003B11847704700BF0368DB6A03B11847B8
:100CF000704700BF03682DE9F04116469A6A044622
:100D00000D460AB1904723685F6A5FB132462946B3
:100D10002046B8472368DB6AC3B12046BDE8F041EE
:100D2000184723689B6820469847B042F9D3002EA5
:100D3000F0DD2E442368204615F8011B1B689847F8
:100D4000B542F7D12368DB6A002BE6D1BDE8F0811C
:100D500070B504460E461546236820469B689847A2
:100D6000A842F9D32A4631462046BDE87040C1E783
:100D70002DE9F843D0F8E8510446C24F95F800C079
:100D800017F91CE05FFA8EF30F2B40F2AD80D0F81C
:100D90003001002851D0BC4E7368984200F05E814B
:100DA000B36A984200F01981F36C984200F05C81BC
:100DB000336F984200F05C81D6F89430984200F08E
:100DC0005981D6F8B830984200F05881D6F8DC3016
:100DD000984200F06581D6F80031984200F06681B3
:100DE000D6F82431984200F06381D6F84831984211
:100DF00000F06281D6F86C31984200F06181D6F83B
:100E00009031984200F06281D6F8B431984200F0F7
:100E10005F81D6F8D831984200F06081D6F8FC3175
:100E2000984200F05F81D6F82032834200F05C8166
:100E300016F8083C002B00F0A280D4F82C31002BCF
:100E400050D0914E7268934200F00A81B26A9A4281
:100E500000F0A680F26C934200F00481326F93425E
:100E600000F00481D6F89420934200F00581D6F872
:100E7000B820934200F00481D6F8DC20934200F0C1
:100E80001181D6F80021934200F00E81D6F824217A
:100E9000934200F00F81D6F84821934200F00E8172
:100EA000D6F86C21934200F00D81D6F89021934240
:100EB00000F00A81D6F8B421934200F00B81D6F8F5
:100EC000D821934200F00881D6F8FC21934200F02B
:100ED0000781D6F82022934200F0088116F8083CDA
:100EE000002B54D0BDE8F883684B00211E461A46FB
:100EF00003E0013103322A293ED010780428F8D1CA
:100F000050786045F5D101EB4101614A0EEB4E008E
:100F10003144897802F8201002EB80025068916019
:100F2000C4F83811C4F8300107EB4C0797F90120D9
:100F300001323FF42EAF002204E0013203332A2AAB
:100F40003FF427AF19780529F7D159786145F4D1D5
:100F500002EB42024E4B0EEB4E0E3244927803F8F7
:100F60002E2003EB8E0EDEF80430CEF80820C4F8F5
:100F70003421C4F82C310CE7D4F83001D4E70B232A
:100F80000CF1010C06F8083C06F807CC55E72B7865
:100F90000C22013306F8082C06F8073CBDE8F8835C
:100FA000012303EBC3032A7806EB830101329B0084
:100FB000087FD2B2002895D1F058364B4A77984234
:100FC0000CBFA020A1200C230B7749F00BFD6B6810
:100FD0002433C4F84C31BDE8F883012303EBC30389
:100FE0000CF1010C06EB83089F0098F81C305FFAA7
:100FF0008CFC002B7FF421AF0B23F059DFF8949089
:1010000088F81DC048450CBFA020A12088F81C30DE
:1010100049F0E8FCF05995F8316048450CBFA02034
:10102000A12049F0DFFC1C4BB109B8F91600C8F843
:101030001030C8F8184049F0A5FCB8F91630002B5C
:1010400007DB03F01F0101225B098A40134941F8C5
:1010500023206B682833C4F84831EEE60023BDE74F
:1010600000239EE702239CE70223B7E7032398E7C8
:101070000323B3E70423B1E7042392E70523ADE795
:1010800005238EE72C790024400100246C1A0A08FD
:101090008000002400000240990B040800E100E0F9
:1010A00006239BE706237CE707237AE7072395E7D8
:1010B000082393E7082374E709238FE7092370E7E0
:1010C0000A238BE70A236CE70B236AE70B2385E7E8
:1010D0000C2383E70C2364E70D2362E70D237DE7F0
:1010E0000E235EE70E2379E70F2377E70F2358E7F8
:1010F000154B1B885BB9154A154B12781B688AB1D2
:101100007BB11A689B8800B91B0493617047114B2F
:10111000D3F894222AB150B9D3F88022106083F812
:101120009102704780F00100002BEAD1F9E7B3F893
:1011300098C20121084AD3F88002B2FBFCF20A41AE
:10114000026083F891127047A25C0024A85C00241E
:10115000A45C0024147E002440420F0038B540F007
:101160002DFF0D490D4DD1F8FC20A5FB00500C4C76
:1011700042F080720B4B800CC1F8FC204FF06042B3
:101180000949C4F80001C2F8B01F00225A601A6869
:1011900042F001021A6038BD00ED00E083DE1B431F
:1011A000147E0024001000E055CEACC530B4EFF33F
:1011B0001183102282F312880B4C4FF0E0210B4870
:1011C00000252268DBB2013222608A69C0F89C22C5
:1011D000C0F8A0520A6983F31188054A13680133E5
:1011E00030BC1360704700BF581E0024147E0024DA
:1011F0004421002410B4EFF31181102383F31288EB
:101200004FF0E0220F4894691369DB0303D50123F3
:10121000C0F8A03294690C4BC9B21B68D0F8A02268
:1012200081F31188D0F800114FF47A701A4400FB52
:1012300001F31B1B5DF8044BB3FBF1F300FB023021
:10124000704700BF147E0024581E0024244B5B68A6
:10125000C3F3080330B4EBB9EFF31183D3B9214CD6
:101260004FF0E02C204A1368DCF8180011688B421C
:10127000F9D1D4F89C128842F5D8D4F800414FF443
:101280007A7101FB04F2101AB0FBF4F030BC01FBE0
:1012900003007047EFF31183102282F312884FF09E
:1012A000E022104C95691169C90303D50121C4F8E6
:1012B000A01295690C4ADBB21268D4F8A00283F33D
:1012C0001188D4F8001110444FF47A7202FB01F334
:1012D0005B1BB3FBF1F330BC02FB0030704700BF77
:1012E00000ED00E0147E0024581E00242DE9F04F8C
:1012F000F24C054694F8A472022F2DED048B93B0A6
:1013000040F0FC8119F0DAF894F8C030D80700F109
:10131000B68219F007FE94F8C030DB0700F1B981FE
:1013200094EDC84AE649BDEEC44AD4EDC94A94EDED
:10133000CE5AFDEEE44AD4EDCA5A14EE103ABDEE90
:10134000C55AFDEEE55A94EDCC6AB3F5FA6FD4EDCB
:10135000CB6ABDEEC66A94EDCF7AA8BF4FF4FA63AC
:10136000FDEEE66ABDEEC77AD4EDCD7AB3F57A7FAD
:10137000D4EDD03AFDEEE77A94EDD14AB8BF4FF400
:101380007A73A3F57A73C3EBC3135B00A1FB03234A
:101390009B097F3B8DF83C3014EE903AB3F5FA6F21
:1013A000A8BF4FF4FA63B3F57A7FB8BF4FF47A73EE
:1013B000A3F57A73C3EBC3135B00A1FB03239B0963
:1013C000C3F17F038DF83D3015EE103AB3F5FA6F97
:1013D000A8BF4FF4FA63B3F57A7FB8BF4FF47A73BE
:1013E000A3F57A73C3EBC3135B00A1FB03239B0933
:1013F0007F3B8DF83E3015EE903AB3F5FA6FA8BFFB
:101400004FF4FA63B3F57A7FB8BF4FF47A73A3F55C
:101410007A73C3EBC3135B00A1FB03239B097F3BE0
:101420008DF83F3016EE103AB3F5FA6FA8BF4FF4BF
:10143000FA63B3F57A7FB8BF4FF47A73A3F57A7382
:10144000C3EBC3135B00A1FB03239B097F3B8DF818
:10145000403016EE903AB3F5FA6FA8BF4FF4FA6336
:10146000B3F57A7FB8BF4FF47A73A3F57A73C3EB01
:10147000C3135B00A1FB032317EE102AB2F5FA6F2A
:101480004FEA9313A8BF4FF4FA627F3BB2F57A7F1D
:101490008DF84130B8BF4FF47A72A2F57A72C2EB80
:1014A000C2125200A1FB023217EE903AFDEEE37A2F
:1014B000B3F5FA6F4FEA9212A8BF4FF4FA637F3A7E
:1014C000B3F57A7F8DF84220B8BF4FF47A73A3F555
:1014D0007A73C3EBC3135B00A1FB032317EE902ABF
:1014E000FDEEC47AB2F5FA6F4FEA9313A8BF4FF43A
:1014F000FA627F3BB2F57A7F8DF84330B8BF4FF484
:101500007A72A2F57A72C2EBC212530017EE902AD9
:10151000B3F5FA3FB4BF00230123B2F5FA6FA8BFB9
:101520004FF4FA62B2F57A7FB8BF4FF47A72A2F53F
:101530007A72C2EBC2125200B2F5FA3F01DB43F0FD
:101540000203D4EDD27AFDEEE77A17EE902AD4EDBD
:10155000D37AB2F5FA6FFDEEE77AA8BF4FF4FA62DC
:10156000B2F57A7FB8BF4FF47A72A2F57A72C2EB05
:10157000C2125200B2F5FA3F17EE902AD4EDD47A97
:10158000A8BF43F00403B2F5FA6FFDEEE77AA8BFF7
:101590004FF4FA62B2F57A7FB8BF4FF47A72A2F5CF
:1015A0007A72C2EBC2125200B2F5FA3F17EE902ADD
:1015B000D4EDD57AA8BF43F00803B2F5FA6FFDEE7B
:1015C000E77AA8BF4FF4FA62B2F57A7FB8BF4FF45A
:1015D0007A72A2F57A72C2EBC2125200B2F5FA3FE9
:1015E00017EE902AD4EDD67AA8BF43F01003B2F5D7
:1015F000FA6FFDEEE77AA8BF4FF4FA62B2F57A7F90
:10160000B8BF4FF47A72A2F57A72C2EBC2125200DE
:10161000B2F5FA3F17EE902AD4EDD77AA8BF43F07F
:101620002003B2F5FA6FFDEEE77AA8BF4FF4FA6235
:10163000B2F57A7FB8BF4FF47A72A2F57A72C2EB34
:10164000C2125200B2F5FA3F17EE902AA8BF43F03B
:101650004003B2F5FA6FA8BF4FF4FA62B2F57A7F91
:10166000B8BF4FF47A72A2F57A72C2EBC21252007E
:10167000B2F5FA3F134AA8BF63F07F03D2F8CC1249
:101680008DF8443092F89C32032B02D1002940F0AF
:10169000C7840023DFF838801E4684F8A4320A4B42
:1016A0001B78002B3CD1FFF7D1FD084BC5F101059C
:1016B000BA001B682844DD690CE000BF147E0024DA
:1016C000D34D6210002B0024EC23002004250020C1
:1016D000B01E002404EB8703D3F8D034E9094FEAA5
:1016E000A31CBCEBD51F01D08B0199118842224469
:1016F00040F3D9808001C2F8D00411E001236C4A84
:101700009F4282F88C3023D10FF0A4FF0223DFF830
:10171000C8811E4684F8A432664B1B78002BC2D0C9
:1017200098F80030472B07D104EB8703624AD3F8BF
:10173000D0349B1122F8173004EB8603D3F8D03451
:101740009B11C4F8DC3413B0BDEC048BBDE8F08F02
:1017500094F8A532002B40F08A8094F8A632002B32
:1017600097D0002384F8A632544B1E78002E40F008
:10177000B980534B1B689D4240F2BB8094F8A7325E
:10178000002B00F01E854F4A9FED4F8ADFF84C91E9
:101790009346DFF84081DFF848A1CDE9017517468F
:1017A0000FE029467B6858469847032E43DD0136F3
:1017B00094F8A73209F10409AAEC010A9E4280F2CA
:1017C0005482072ED8F83030D4BF18F80650F5B23E
:1017D000002BE6D07B68584629469847B8F81A206F
:1017E00004EB4503B8F81C00B3F8F0329A4200F25B
:1017F000378207EE900A07EE103AF8EE677AB8EEF5
:10180000477AC7FEC77A012303FA05F1D8F83030CA
:10181000194205D0D4F8183313F4807F00FE270A4C
:10182000BCEEC00A032E10EE103A9BB200EE103A46
:10183000B8EE400ABBDCB5EE400AF1EE10FAB6D0C5
:10184000B9F8003006EE903AB9F80230F8EE666A60
:1018500007EE103AB8EE477A30EE660A37EE667A4F
:1018600060EE087A87EE870A30EE080A9FE7154A8D
:10187000D36810469847002384F8A5326DE7134BD0
:101880001B68002B3FF405AF11491A6809789B8843
:10189000C907DFF8448058BF1B04936100231E462C
:1018A00084F8A432FBE6013BC2F8D03438E700BF2D
:1018B000E4360020EC230020B41E0024505B0024FA
:1018C0004C5B00242C5B002400007A44601E002442
:1018D0006C1E0024D8560024B01E0024E86D00249D
:1018E000BC800024C74A1268954284BF06F1FF36C7
:1018F0001E70C54ADFF860831369002B00F0B380C7
:1019000098470646FFF7A2FCD4F81424831BB21AAA
:10191000049300F0A880C4F81464C4F81824D4F820
:101920001C340499EB1A9942B8BF134698F800206A
:10193000DFEDB66A3E2AC4F81C544FF6DC7200F0A4
:101940008D829A4240F2B631A8BF1A468A42B8BF89
:101950000A4607EE902AD31AB8EEE77AB3FA83F371
